:10A1BF0020466F726D6174616765204C6F674361F4
:10A1CF0072642E2E2E20004E4520746F75636865C5
:10A1DF007A205041532027206C61204C6F674361D8
:10A1EF007264202100005F00204D656E7520707233
:10A1FF00696E636970616C200020456E7472612610
:10A20F006E656D656E74200020456E747261266EEA
:10A21F00656D656E74205374616E646172642000A5
:10A22F0020456E747261266E656D656E7473207055
:10A23F006572736F2E204C43200020456E7472613F
:10A24F00266E656D656E747320706572736F2E2048
:10A25F0000204E6F7576656C20656E747261266E88
:10A26F002E20706572736F2E204C432000204E6F8E
:10A27F007576656C20656E747261266E2E20506542
:10A28F0072736F2E2000204E6F7576656C20656E91
:10A29F00747261266E656D656E74204C43200020CC
:10A2AF004E6F7576656C20656E747261266E656D86
:10A2BF00656E74200020442A66696E697220656E8F
:10A2CF00747261266E656D656E74206475722A6591
:10A2DF00200020442A66696E697220656E7472616F
:10A2EF00266E656D656E742E2064697374616E637E
:10A2FF006520002052617070656C204C6F67436160
:10A30F0072642000204D2A6D6F6972652000204312
:10A31F006F6E66696775726572200020436F6E6697
:10A32F0069672C206D2A6D6F697265200020436F5D
:10A33F006E6669672E2046432000204365696E7460
:10A34F0075726520414E5420002050726F707269F3
:10A35F002A742A73200020436F65662E2053696785
:10A36F006E616C2000204269656E76656E756520A2
:10A37F0000204175207265766F69722000204C6F46
:10A38F006743617264200020522A73756D2A204C36
:10A39F006F67436172642000205574696C69746142
:10A3AF0069726573204C6F67436172642000204DA2
:10A3BF006F6469662E20646F6E6E2A6573204C6F12
:10A3CF006743617264200020442A662074656D70B3
:10A3DF007320706173736167652000456666616302
:10A3EF006572206D2A6D6F697265203F0045666644
:10A3FF0061636572206465726E2E20732A616E63CD
:10A40F0065203F0050617373657220656E206D6F1C
:10A41F006465206578657263696365203F005061EC
:10A42F007373657220656E206D6F6465207465733C
:10A43F0074203F00466F726D61746572204C6F67B8
:10A44F0043617264203F0045666661636572206DEB
:10A45F002A6D6F697265204C6F6743617264203F8C
:10A46F0000442A66696E6972202A746174207A2A00
:10A47F00726F203F00522A696E69742E20746F75B7
:10A48F0073202A74617473203F00522A696E6974B5
:10A49F002E206475722A652065786572636963651D
:10A4AF00203F0050722474202320642A66696E694D
:10A4BF007220636F65662E202A74616C6F6E2E207A
:10A4CF002100442A66696E697220636F65662E20CB
:10A4DF002A74616C6F6E2E203F00507224742023FB
:10A4EF0020642A66696E6972204944206170706128
:10A4FF007265696C202100442A66696E6972204971
:10A50F004420617070617265696C203F0020442A9D
:10A51F0066696E6972202A746174207A2A726F20BC
:10A52F000057617474006D6F792E007C004A0074BF
:10A53F006F74616C006B4A007D002F316B6D006D85
:10A54F0000436C61732E006D61782E00706163653E
:10A55F0000742F6D007E0020496E697469616C690B
:10A56F0073657220636170746575727320002020AB
:10A57F00200025346400253364002E253164002526
:10A58F00326400253034640020526573742000203B
:06A59F00526563616C6C63
:10A5A50020005075697373616E636500496E74654B
:10A5B50072762E206D61782E5E5E3A2025752057C5
:10A5C50000456E657267696500496E746572762E21
:10A5D500206D61782E5E5E3A20252E3166206B4A0D
:10A5E500005669746573736500496E746572762EDD
:10A5F500206D61782E5E5E3A202575206B6D2F6883
:10A605000044697374616E636500496E74657276A2
:10A615002E206D61782E5E5E3A202575206D0043F3
:10A625006164656E636500496E746572762E206D92
:10A6350061782E5E5E3A2025752072706D00464366
:10A6450000496E746572762E206D61782E5E5E3AD5
:10A655002025752062706D004D6F79656E6E655EA3
:10A665005E3A202575205700546F74616C5E5E3A22
:10A6750020252E3166206B4A004D6F79656E6E651B
:10A685005E5E3A202575206B6D2F6800546F7461EE
:10A695006C5E5E3A202575206D004D6F79656E6E96
:10A6A500655E5E3A2025752072706D004D6F796587
:10A6B5006E6E655E5E3A2025752062706D002849D4
:10A6C5006E746572762E202575206D696E2900459C
:10A6D5006E6572676965205B4A5D005669746573CE
:10A6E5007365205B6B6D2F685D00507569737361D1
:10A6F5006E6365205B575D00477261706865002574
:10A70500752020002020257520200020202575009B
:10A715003073005369676E616C0020302E357320ED
:10A7250000202031730020203173202000202032AA
:10A735007300466F726365206D61782E3A2025752A
:10A74500204E202020004A676368652020202020B5
:10A7550020202020302320203138302320202020A5
:10A76500204A64727465003930232020202020207F
:10A7750020202020202020202020202020202020D4
:10A78500202020202020202020203930230031388F
:10A795003023202030230025752525200020257510
:10A7A5002525002575270020257520002575206D98
:10A7B50020282564206D2900252E3066206D20284F
:10A7C5002564206D29002575206D00252E30662015
:10A7D5006D007000253032643A2530326400502A0D
:10A7E50064616C657200456E747261266E656D6597
:10A7F5006E74004D2A6D6F69726500436F6E6669F0
:10A805006775726572004C6F6743617264004465D9
:10A81500726E69657220456E747261266E656D652E
:10A825006E74005374616E64617264005265666192
:10A8350069726520456E747261266E656D656E740C
:10A8450000506572736F2E20284C6F6743617264E8
:10A855002900506572736F2E004E6F7576656C20FA
:10A86500456E747261266E656D656E7400312030BB
:10A875003030206D003320303030206D00342030F2
:10A885003030206D00313020303030206D003330D5
:10A89500206D696E75746573003630206D696E754F
:10A8A500746573005E456E747261266E2E5E5E522F
:10A8B5002A6375702E5E5E527974686D6500257524
:10A8C5002E5E253032643A253032643A25303264C2
:10A8D5005E5E253032643A253032645E5E25303264
:10A8E500643A2530326420282F316B6D2900257597
:10A8F5002E5E256C646D5E5E253032643A253032FD
:10A90500645E5E253032643A2530326420282F316A
:10A915006B6D2900532A616E6365003A2025750029
:10A925004475722A6500506C7573206427696E74CE
:10A93500657276616C004475722A652028683A6DE7
:10A945003A73295E5E5E3A0025303264203A20254E
:10A95500303264203A202530326420202000253012
:10A9650032643A253032643A253032642020202082
:10A975002020200044697374616E636520286D2969
:06A985005E5E5E3A002553
:10A98B0075202575202575202575202575202575A5
:10A99B000025752575257525752575257500447557
:10A9AB00722A6520722A632E20286D3A73295E5E07
:10A9BB005E3A0025303264203A2025303264202064
:10A9CB002000253032643A253032642020202020AC
:10A9DB00202000527974686D6520286D3A73295ECA
:10A9EB005E5E3A0025303264203A202530326420F6
:10A9FB002020282F316B6D2900253032643A253009
:10AA0B00326420282F316B6D292020202020004715
:10AA1B00726170686971756500546578746500447E
:10AA2B002A66696E697220496E74657276616C0074
:10AA3B0050726F7072692A742A730053757070723A
:10AA4B00696D657220746F75740053757070722E1A
:10AA5B00206465726E2E20732A616E6365005478D4
:10AA6B00202A6368616E74696C6C6F6E2E00417581
:10AA7B0063756E0000257520666F69730000436572
:10AA8B00696E7475726520414E5400506F6C617223
:10AA9B0000253575202825732900414E542B537002
:10AAAB006F7274005375756E746F00496E746572B6
:10AABB0076616C6C655E5E3A202575206D696E0063
:10AACB0056657273696F6E206D6963726F70726F0A
:10AADB00672E5E5E5E3A20252E316600494420616A
:10AAEB007070617265696C5E5E5E3A20256C640005
:10AAFB00494420636170746575725E5E5E3A202511
:10AB0B006C6400494420636170746575725E5E5EAF
:10AB1B003A206E6F6E20636F6E6E6563742A00420F
:10AB2B00617474657269655E5E5E3A2025730053CD
:10AB3B002A616E6365735E5E5E3A20252D3264007A
:10AB4B004D2A6D6F6972655E5E5E3A20252D642518
:10AB5B0025206672656500496E74657276616C6C52
:10AB6B00655E5E5E3A20252D64206D696E00466F32
:10AB7B007263655E5E5E3A2041203D20252D382EA6
:10AB8B003566003A2042203D20252D362E336600B7
:10AB9B003A2043203D20252D352E32660052617917
:10ABAB006F6E206D616E69762E5E5E5E3A20257546
:10ABBB00206D6D004865757265735E5E5E3A20258B
:10ABCB006C64004D656E75204C6F67436172640059
:10ABDB004D2A6D6F697265204C6F67436172645EBD
:10ABEB005E5E3A20252D342E316625252066726552
:10ABFB0065004D656E75207072696E636970616C6E
:10AC0B0000522A73756D2A004E6F6D207574696C36
:10AC1B00697361746575725E5E5E3A2025730052CE
:10AC2B00617070656C005574696C697461697265EB
:10AC3B0073004E6F6D207574696C69736174657503
:10AC4B00725E5E5E5E3A202573004D2A6D6F6972EF
:10AC5B0065204C6F67436172645E5E5E5E3A2025D1
:10AC6B002D342E316625252066726565004E6F6D7D
:10AC7B0062726520646520732A616E6365735E5E24
:10AC8B005E5E3A202575004D6F6469662E20646FF9
:10AC9B006E6E2A6573207574696C69732E00456638
:10ACAB006661636572206D2A6D6F697265204C6FEA
:10ACBB00674361726400546F757420666F726D61C7
:10ACCB00746572004E6F6D207574696C69732E5EBE
:10ACDB003A0025630025730020496E666F732000D0
:10ACEB0045534300454E5445520020532A6C65632F
:10ACFB00742E20732A616E63652072617070656CAF
:10AD0B00200020532A6C6563742E20732A616E63B6
:10AD1B0065202320726566616972652000532A6184
:10AD2B006E63655E5E3A202575202F2025750044E5
:10AD3B006174655E5E3A20253032642E25303264B4
:10AD4B002E3230253032640048657572655E5E3A8E
:10AD5B0020253032643A253032643A253032640093
:06AD6B004475722A655ECA
:10AD71005E3A20253031643A253032643A2530324A
:10AD8100643A2530326400496D706F7274616E747B
:10AD91003A5E5E4D2A6D6F6972652064652072614D
:10ADA1007070656C20706C65696E652021005E5E57
:10ADB1005365756C6520756E652070617274696587
:10ADC100206465206C6120732A616E6365206120B7
:10ADD1002A742A207361757665676172642A652E0B
:10ADE1000020522A6375702E20004D2A6D6F697202
:10ADF100652064652072617070656C20706C656996
:10AE01006E65202100417563756E20722A73756D20
:10AE11002A206465206C6120732A616E63650028B5
:10AE21004D2A6D6F6972652064652072617070656D
:10AE31006C20706C65696E652900253031643A2596
:10AE41003032643A30303A3030202D2025303164B0
:10AE51003A253032643A253032643A253032640082
:10AE6100507569732E206D6F792E5E5E3A202575BF
:10AE7100205700456E65726769655E5E3A20252E32
:10AE81003166206B4A0056697465737365206D6F76
:10AE9100792E5E5E3A20252E3166206B6D2F68007B
:10AEA10044697374616E63655E5E3A20252E306677
:10AEB100206D00436164656E63655E5E3A202575B1
:10AEC1002074722F6D6E004643206D6F792E5E5E89
:10AED1003A2025752062706D00522A73756D2A2003
:10AEE100732A616E6365202575004475722A655E5B
:10AEF1005E5E5E5E5E3A20253031643A2530326412
:10AF01003A253032643A2530326400507569732E27
:10AF1100206D6F792E5E5E5E5E5E5E3A2025752045
:10AF21005700507569732E206D61782E5E5E5E5EEE
:10AF31005E5E3A202575205700252547202F2025C4
:10AF410025445E5E5E5E5E5E3A202575202F2025DB
:10AF51007500436164656E63655E5E5E5E5E5E3A6A
:10AF61002025752074722F6D6E004361642E206D53
:10AF710061782E5E5E5E5E5E5E3A2025752074729B
:10AF81002F6D6E0044697374616E63655E5E5E5E13
:10AF91005E5E3A20252E3066206D00456E65726733
:10AFA10069655E5E5E5E5E5E3A20252E3166206BCF
:10AFB1004A005669742E206D6F792E5E5E5E5E5E6C
:10AFC1005E3A20252E3166206B6D2F6800464320A6
:10AFD1006D6F792E5E5E5E5E5E5E3A202575206243
:10AFE100706D002573253032643A253032643A257C
:10AFF1003032643B2000002573256C646D3B2000DA
:10B0010000566964650000257520257300002E2E09
:10B011000000253564002575002530356C64002558
:10B02100356C6400253031643A253032643A25307C
:10B03100326400417563756E6520732A616E6365C4
:10B0410020232072617070656C6572202100457249
:10B0510072657572202100532A616E6365207065E7
:10B0610072736F2E20566964650043617074657553
:10B071007220636F6E6E6563742A206572726F6EE3
:10B081002A0043617074657572206E6F6E20636F64
:10B091006E6E6563742A0046696E20646520732AAA
:10B0A100616E63652021004D2A6D6F69726520769E
:10B0B1006964652021004D2A6D6F697265204C6FAE
:10B0C1006743617264207669646520210052656C72
:10B0D10061782021004475722A6520646520722AF6
:10B0E1006375702E0050722474202320726566618E
:10B0F100697265206C6120732A616E63652021008D
:10B101005072247420617520642A70617274202148
:10B111000020532A616E63655E3A20257500204444
:10B1210075722A655E3A20253032643A25303264E0
:10B131003A25303264002044697374616E63655E40
:10B141003A20256C64206D00532A616E6365206589
:06B151006E747261266EAF
:10B157002E2025752F257500532A616E63652023E0
:10B167002072656661697265207465726D696E2A01
:10B177006520210046696E206465206C27656E7422
:10B187007261266E656D656E7420210025752073CA
:10B197002A616E636573002A76616C752A65730090
:10B1A700426174746572696520642A6368617267B5
:10B1B7002A65202100457874696E6374696F6E0093
:10B1C700417563756E6520616374697669742A20B9
:10B1D70021004175207265766F697200496D706F45
:10B1E700737369626C6520646520642A66696E6999
:10B1F70072206C272A746174007A2A726F20706536
:10B207006E64616E74206C6120732A616E636520C1
:10B217002100532A616E6365206E6F6E207361751E
:10B227007665676172642A6500537570707265731D
:10B23700732E206465726E2E20532A616E6365201B
:10B247007465726D696E2A65202100257520732A41
:10B25700616E6365732072657374616E74657300E4
:10B267005472616E736665727420646520732A6117
:10B277006E636500257520656E20636F7572732098
:10B2870021005472616E7366657274206465206470
:10B297006F6E6E2A657320616E6E756C2A202100B1
:10B2A700546F7573202A7461747320722A696E69EA
:10B2B7007469616C69732A732021004C6563747526
:10B2C7007265204C6F674361726420696D706F739C
:10B2D7007369626C652021004173737572657A2DFD
:10B2E700766F757320717565206C61204C4300651E
:10B2F700737420636F7272656374656D656E742015
:10B30700696E732A722A652E00496E697469616CC9
:10B3170069736174696F6E20636F7572736520213D
:10B327000050722A706172657A2D766F757320707E
:10B337006F7572206C6120636F75727365202100D1
:10B347003B3C00436F75727365207465726D696E5F
:10B357002A65202100436C617373656D656E7420E7
:10B3670066696E616C3A20257500436F7572736567
:10B3770020696E746572726F6D7075652021005259
:10B387006563686572636865206365696E74757265
:10B39700652873292046432E202100566575696C60
:10B3A7006C657A2070617469656E7465722E2E2ED5
:10B3B700004365696E7475726520464320696E7433
:10B3C700726F757661626C6520210040205F2025D1
:10B3D7007300466169626C6500456C65762A004DAD
:10B3E7006F79656E00253032643A2530326420204B
:10B3F7000003000000000000000000000200808041
:10B40700808080008000000400A0A00000000000F1
:10B41700000005006090906000000000000510200B
:10B42700006090F080600000070048B0501028349A
:10B437002800000440A00040404040400000054074
:10B447002000601070907000000400204080808011
:10B45700808040200400804020202020204080055C
:10B467001020006090F0806000000600000020209F
:10B47700F82020000002000000000000008080008B
:10B48700030000000000C0000000000200000000F0
:10B497000000008000000400202040404080800021
:10B4A700000500609090909090600000030040C0FD
:10B4B700404040404000000500609010202040F0D0
:10B4C700000005006090102010906000000600103A
:10B4D700305090F81010000005007040E090109078
:10B4E7006000000500609080E0909060000005001B
:10B4F700F0102020404040000005006090906090D0
:10B50700906000000500609090701090600000024D
:10B5170000000080000000800000020000008000A2
:10B5270000008080000400002040804020000000D0
:06B5370005000000F00019
:10B53D00F00000000004000080402040800000006A
:10B54D000600708808302000200000080000000070
:10B55D000000000000000800102828447C448200F0
:10B56D00000600F08888F08888F0000006007088DA
:10B57D00808080887000000600F08888888888F0B8
:10B58D0000000600F88080F88080F800000600F8C2
:10B59D008080F08080800000060070888098888808
:10B5AD007000000600888888F888888800000200EE
:10B5BD0080808080808080000005001010101010A9
:10B5CD009060000006008890A0C0A0908800000543
:10B5DD0000808080808080F00000080082C6C6AAAE
:10B5ED00AAAA920000060088C8C8A89898880000EA
:10B5FD0006007088888888887000000600F08888AA
:10B60D00F08080800000060070888888889078001F
:10B61D00000600F08888F090888800000600708889
:10B62D00807008887000000600F82020202020205F
:10B63D0000000600888888888888700000080082CD
:10B64D008244442828100000080082925454545417
:10B65D002800000600885050205050880000060039
:10B66D008850502020202000000700FC08102040AA
:10B67D0080FC00000300C080808080808080C0043A
:10B68D00008080404040202000000300C04040402A
:10B69D0040404040C0040040A0A000000000000059
:10B6AD0006000000000000000000F802008080008D
:10B6BD000000000000000500000060107090700098
:10B6CD000005008080E0909090E0000005000000F3
:10B6DD006090809060000005001010709090907048
:10B6ED000000050000006090F08060000004002064
:10B6FD0040E04040404000000500000070909090F8
:10B70D0070906005008080E09090909000000200A5
:10B71D008000808080808000000300400040404019
:10B72D00404040800500808090A0C0A090000002A5
:10B73D000080808080808080000008000000EC92F6
:10B74D00929292000005000000E090909090000011
:10B75D00050000006090909060000005000000E082
:10B76D00909090E080800500000070909090701097
:10B77D001005000000B0C0808080000005000000B2
:10B78D0070806010E0000004000040E04040402068
:10B79D0000000500000090909090700000060000E1
:10B7AD00008850505020000006000000A8A8A8A84E
:10B7BD0050000005000000906060609000000600E1
:10B7CD0000008850505020204004000000E0204030
:10B7DD0080E00000030000000000000000000002F7
:10B7ED0000808080808080808000180080404040F4
:10B7FD0020404040800000000E001C002A00380050
:10B80D00460061006F007D008B009900A700B50018
:10B81D00C300D100DF00ED00FB0109011701250177
:10B82D00330141014F015D016B01790187019501E3
:10B83D00A301B101BF01CD01E80203021E023902CD
:10B84D005402620270028B02A602B402C202DD0231
:10B85D00EB03060321033C03570372038D03A80377
:10B86D00B603D103EC040704220430043E044C0457
:10B87D005A046804760484049204A004AE04BC0443
:10B88D00CA04D804E604F405020510051E052C05AE
:10B89D003A055505630571057F058D059B05A905C0
:10B8AD00B705C505E005FB06090624063206400668
:10B8BD005B06830400000000000000000000000093
:10B8CD000004606060606060600060600000000700
:10B8DD006C6C6C00000000000000000000083018C7
:10B8ED00003C461E3666663E00000008386C003C83
:10B8FD0066667E60663C0000000A720052005200CF
:10B90D00540074000B800A800A801280138000009E
:06B91D00000000000670AE
:10B92300D8003030303030303000000004606060C8
:10B9330000000000000000000000051030206060DF
:10B9430060606060602030100480C04060606060B0
:10B9530060606040C080080C18003C66667E6066CC
:10B963003C0000000800000018187E1818000000B2
:10B9730000000400000000000000006060204000A0
:10B98300050000000000000070000000000004003B
:10B99300000000000000006060000000051010209F
:10B9A300202040404080800000000778CCCCCCCCE5
:10B9B300CCCCCCCC7800000007183878581818186D
:10B9C3001818180000000778CC0C0C18383060C029
:10B9D300FC0000000778CC0C0C380C0C0CCC780065
:10B9E30000000718183838585898FC181800000039
:10B9F300077C60C0F8CC0C0C0CCC78000000073836
:10BA03004CC0C0F8CCCCCCCC7800000007FC0C18A0
:10BA1300183030306060600000000778CCCCCC7800
:10BA2300CCCCCCCC780000000778CCCCCCCC7C0C34
:10BA33000CC870000000040000006060000000609B
:10BA430060000000040000006060000000606020EF
:10BA53004000080000041C70C0701C0400000000BB
:10BA63000800000000FE00FE0000000000000800C7
:10BA73000040701C061C704000000000087CC606D5
:10BA8300060C18300030300000001088009001A62A
:10BA930082C544A54895508D680048008E0109026F
:10BAA30009040908090B0E000E001B001B001B00F4
:10BAB300318031803F8060C060C000000000000022
:10BAC300097E006300630063007E0063006300631C
:10BAD3000063007E000000000000000A1F003180A8
:10BAE30060006000600060006000600031801F0043
:10BAF300000000000000097C00660063006300632F
:10BB03000063006300630066007C00000000000027
:10BB130000087E6060607E606060607E00000008F8
:10BB23007E606060607E606060600000000A1F00ED
:10BB330031806000600060006780618061803180D7
:10BB43001F0000000000000009630063006300633E
:10BB5300007F006300630063006300630000000074
:10BB6300000000046060606060606060606000000E
:10BB730000080606060606060666663C000000097F
:10BB8300630066006C006C007C0076006600660053
:10BB930063006300000000000000086060606060F4
:10BBA300606060607E0000000B71C071C07BC07B71
:10BBB300C06AC06AC06AC06EC06EC064C0000000C4
:10BBC300000000096300730073007B006B006F00CB
:10BBD30067006700630063000000000000000A1EA6
:10BBE30000330061806180618061806180618033A6
:10BBF300001E00000000000000097E0063006300D7
:10BC0300630063007E00600060006000600000006D
:10BC1300000000000A1E00330061806180618061C2
:10BC2300806180658033001F0000800000000009F0
:10BC33007E0063006300630063007E0066006300B0
:10BC430063006180000000000000093E00630060A3
:10BC53000070003C001E000700030063003E00006C
:10BC6300000000000008FF181818181818181818F2
:10BC73000000000963006300630063006300630066
:10BC83006300630063003E000000000000000A60E0
:10BC9300C060C03180318031801B001B001B000E4F
:10BCA300000E000000000000000F638C638C3398CB
:10BCB30036D836D836D836D81C701C701C700000A5
:10BCC30000000000096300630036001C001C001C18
:10BCD300001C003600630063000000000000000841
:10BCE300C3C3663C3C181818181800000008FE0669
:10BCF3000C1818303060C0FE0000000570606060F2
:06BD0300606060606060FA
:10BD090060607005808040404020202010100000B5
:10BD19000004E06060606060606060606060E0082E
:10BD29000030307848CC0000000000000007000017
:10BD390000384446463E1C00000000046060600074
:10BD4900000000000000000000080000003C461E42
:10BD59003666663E000000086060606C766666665E
:10BD6900766C000000080000003C66606060663C7C
:10BD790000000008060606366E6666666E36000026
:10BD890000080000003C66667E60663C0000000515
:10BD9900306060F060606060606000000008000072
:10BDA90000366E6666666E3606463C086060606CF4
:10BDB9007666666666660000000460600060606022
:10BDC9006060606000000004606000606060606046
:10BDD90060606060C008606060666C78786C6C66F2
:10BDE9000000000460606060606060606060000086
:10BDF900000C0000000000006EC07760666066609D
:10BE090066606660666000000000000008000000CF
:10BE19006C766666666666000000080000003C668F
:10BE2900666666663C000000080000006C7666667F
:10BE390066766C60606008000000366E6666666E45
:10BE490036060606060000007860606060606000E3
:10BE59000000080000003C66703C0E663C000000D3
:10BE690006001030783030303030180000000800FB
:10BE7900000066666666666E36000000090000000E
:10BE8900000000630063003600360036001C001C09
:10BE9900000000000000000C0000000000006230FB
:10BEA9006730376035603DE01DC018C000000000F4
:10BEB90000000800000066663C183C666600000049
:10BEC90009000000000000630063003600360036F8
:10BED900001C001C001C0018007800070000007CF2
:10BEE9000C183030607C00000006000000000000E3
:10BEF900000000000000000C31807BC0FFE0FFE083
:10BF0900FFE07FC03F800E00040000000000000039
:10BF19000000158001808002809762E0A49490C49B
:10BF29009490A4989094989000000000000000005C
:10BF3900000000000000000000000E20107020200A
:10BF49004020802100120004000BB0124822484210
:10BF59004802480000000000000000000000000046
:10BF690000000000000000000000000000000000C8
:10BF7900000043007000B300F60139017C01BF02E3
:10BF8900020245028802CB030E0351110000000092
:10BF99000000000000000000000000000000000098
:10BFA9000000000000000000000000000000000088
:10BFB9000000000000000000000000000000000078
:10BFC90000000000000000000000000000000B005D
:10BFD9000000000000000000000000000000000058
:10BFE9000000000000000000000000000000000048
:10BFF900000E001F001F001F000E001100000000AE
:10C009000000000000000000000000000000000027
:10C019000000000000000000000000000000000017
:10C029000000000000000000000000000000000007
:10C0390000000000000000000000000000001107DF
:10C04900E0000FF0001FF8003FFC003C3C003C3CC6
:10C0590000781E00781E00781E00781E00781E00E9
:10C06900781E00781E00781E00781E00781E003C9D
:10C079003C003C3C003FFC001FF8000FF00007E0CB
:10C08900001100F00000F00001F00003F00007F0DB
:10C09900001FF0003FF0003EF00038F00020F000F3
:10C0A90000F00000F00000F00000F00000F00000D7
:10C0B900F00000F00000F00000F00000F00000F0D7
:10C0C9000000F0001107E0001FF8003FFC003FFCF2
:10C0D900007C3E00781E00781E00001E00001E0035
:06C0E900003C00007C0099
:10C0EF0000F80001F00003E00007C0000F80001F00
:10C0FF0000001E00003FFE003FFE007FFE007FFE9F
:10C10F00001107C0001FF0003FF8003FF8007C7CD3
:10C11F0000783C00383C00003C0000780003F00041
:10C12F0003E00003F800003C00001E00001E007832
:10C13F001E00781E007C3E003FFC001FFC000FF02D
:10C14F000007E0001100780000780000F80001F807
:10C15F000003F80003F80007F8000F78000E7800CE
:10C16F001E78003C7800387800707800F07800FF77
:10C17F00FE00FFFE00FFFE00FFFE000078000078CB
:10C18F0000007800007800113FFC003FFC003FFCEE
:10C19F00007FFC007800007800007800007FE0004E
:10C1AF007FF000FFF800FFFC00F87E00701E00001B
:10C1BF001E00001E00F01E00F83E00FC7C007FFCFD
:10C1CF00003FF8001FF0000FC0001103E0000FF850
:10C1DF00001FFC001FFC003E3E003C1E00780000CC
:10C1EF007800007BE0007FF8007FFC007FFC007C84
:10C1FF003E00781E00781E00781E00381E003C3E60
:10C20F00003FFC001FFC000FF80003E000117FFE51
:10C21F00007FFE007FFE007FFE00003C00007800E4
:10C22F0000700000F00000E00001E00001C000031A
:10C23F00C00003C000038000078000078000078054
:10C24F00000F00000F00000F00000F00000F000094
:10C25F001107E0001FF8003FFC007C3E00781E0035
:10C26F00781E00781E00781E003C3C001FF8000F5F
:10C27F00F0001FF8003C3C00781E00781E00781E6E
:10C28F0000781E00781E003C3C003FFC001FF800A9
:10C29F0007E0001107C0001FF0003FF8003FFC004F
:10C2AF007C3C00781C00781E00781E00781E007CF5
:10C2BF003E003FFE003FFE001FFE0007DE00001E97
:10C2CF0000001E00783E007C7C003FFC003FF80021
:10C2DF001FF0000FC000090000000018003C003CD8
:10C2EF000018000000000000000000000000000027
:10C2FF00000000000018003C003C00180000000087
:10C30F00000000000000000000000000000000001E
:10C31F00000000000000000000000000000000000E
:10C32F008D00D400D5016201EF027C03090396044E
:10C33F002304B0053D05CA0657069E074E07FE1B90
:10C34F0000000000000000000000000000000000DE
:10C35F0000000000000000000000000000000000CE
:10C36F0000000000000000000000000000000000BE
:10C37F0000000000000000000000000000000000AE
:10C38F00000000000000000000000000000000009E
:10C39F00000000000000000000000000000000008E
:10C3AF00000000000000000000000000000000007E
:10C3BF00000000000000000000000000000000006E
:10C3CF000000000000000000000000000F0000004F
:10C3DF00000000000000000000000000000000004E
:10C3EF00000000000000000000000000000000003E
:10C3FF00000000000000000000000000000000002E
:10C40F000000000000038007C00FE00FE00FE007FF
:10C41F00C00380001B003F800000FFE00003FFF817
:10C42F000007FFFC0007FFFC000FFFFE000FF1FEEF
:10C43F00001FE0FF001FC07F001FC07F001F803F55
:10C44F00003F803F803F803F803F803F803F803F65
:10C45F00803F803F803F803F803F803F803F803FD5
:10C46F00803F803F803F803F803F803F803F803FC5
:10C47F00803F803F801F803F001FC07F001FC07F15
:10C48F00001FE0FF000FF1FE000FFFFE0007FFFC93
:10C49F000007FFFC0003FFF80000FFE000003F80F3
:10C4AF00001B0003F0000003F0000007F000000F76
:10C4BF00F000001FF000003FF000007FF00001FFD0
:06C4CF00F00007FFF00081
:10C4D5000FFFF0000FF7F0000FE7F0000FC7F000B7
:10C4E5000F07F0000C07F0000007F0000007F00050
:10C4F5000007F0000007F0000007F0000007F0005B
:10C505000007F0000007F0000007F0000007F0004A
:10C515000007F0000007F0000007F0000007F0003A
:10C525000007F0000007F0000007F0000007F0002A
:10C535000007F0000007F0001B003FC00000FFF8F7
:10C545000001FFFC0003FFFE0007FFFF000FFFFFD8
:10C55500000FF0FF800FE07F801FC03F801FC03FAE
:10C56500800FC03F8000003F8000003F8000007FBB
:10C575000000007F000000FE000001FE000003FC3B
:10C58500000007F800000FF000001FE000003FC0AA
:10C5950000007F800000FF000001FE000003FC009A
:10C5A5000003F8000007F000000FFFFF800FFFFFFA
:10C5B500801FFFFF801FFFFF803FFFFF803FFFFFC2
:10C5C500803FFFFF801B003F800000FFE00003FF6E
:10C5D500F00007FFF80007FFFC000FFFFC000FF15C
:10C5E500FE001FE0FE001FC0FE0003C0FE000000AD
:10C5F500FE000001FC000003FC00000FF800001F16
:10C60500E000001FC000001FF800001FFC00000034
:10C61500FE0000007F0000007F0000003F8000005A
:10C625003F8000003F800F803F803F803F803FC0BC
:10C635007F801FC07F001FF1FF001FFFFE000FFF5F
:10C64500FE0007FFFC0003FFF80001FFE000003FCC
:10C6550080001B0000FC000001FC000003FC000042
:10C6650003FC000007FC00000FFC00000FFC0000AD
:10C675001FFC00003FFC00007FFC00007FFC000069
:10C68500FDFC0001F9FC0001F9FC0003F1FC0007C9
:10C69500E1FC0007E1FC000FC1FC001F81FC001F4D
:10C6A50081FC003F01FC007E01FC007FFFFF807FD5
:10C6B500FFFF807FFFFF807FFFFF807FFFFF807F81
:10C6C500FFFF800001FC000001FC000001FC0000F0
:10C6D50001FC000001FC000001FC000001FC001B46
:10C6E50001FFFF0001FFFF0001FFFF0003FFFF0047
:10C6F50003FFFF0003FFFF0003FFFF0003F8000037
:10C7050007F0000007F0000007F0000007F0000048
:10C7150007E7C0000FFFF0000FFFFC000FFFFE0052
:10C725000FFFFE000FFFFF001FF0FF001FC07F80FF
:10C7350003803F8000003F8000003F8000003F8075
:10C745000F803F803F803F803FC07F801FC07F00BC
:10C755001FF0FF001FFFFE000FFFFE0007FFFC009C
:10C7650003FFF80001FFE000003F80001B001FC031
:10C7750000007FF00001FFF80003FFFC0007FFFC4D
:10C785000007FFFE000FF1FE000FE0FF001FC07F56
:10C79500001F807C001F8000003F8000003F80005C
:10C7A500003F8FC0003FBFF0003F7FF8003FFFFC18
:10C7B500003FFFFE003FFFFF003FE0FF003FC07F5F
:10C7C500803F803F803F803F803F803F801F803F8C
:10C7D500801F803F801FC03F801FC07F800FF0FFFC
:10C7E500000FFFFF0007FFFE0003FFFC0001FFF83D
:10C7F5000000FFF000003FC0001B3FFFFF803FFF30
:10C80500FF803FFFFF803FFFFF803FFFFF803FFF2F
:10C81500FF803FFFFF0000007E000000FC000001DC
:10C82500F8000003F8000003F0000007E00000072F
:10C83500E000000FC000001FC000001F8000003F87
:10C845008000003F0000003F0000007F0000007EE8
:10C85500000000FE000000FE000000FE000001FCDC
:10C86500000001FC000001FC000001FC000001F8D3
:10C87500000003F8000003F8000003F8000003F8C7
:10C88500000003F800001B003F800001FFF00003DB
:10C89500FFF80007FFFC000FFFFE000FF1FE001F71
:10C8A500E0FF001FC07F001FC07F001FC07F001F6B
:06C8B500C07F001FC07FE0
:10C8BB00000FE0FE000FF1FE0007FFFC0001FFF090
:10C8CB000000FFE00003FFF80007FFFC000FE0FE95
:10C8DB00001FC07F001FC07F003F803F803F803F15
:10C8EB00803F803F803F803F803F803F803FC07FC5
:10C8FB00801FC07F001FF0FF000FFFFE0007FFFE31
:10C90B000003FFF80001FFF000003FC0001B007F99
:10C91B00800001FFE00003FFF00007FFF8000FFFAE
:10C92B00FC001FFFFE001FE1FE003FC07F003F80A9
:10C93B007F003F803F003F803F003F803F803F8034
:10C94B003F803F803F803FC07F801FE0FF801FFF05
:10C95B00FF800FFFFF8007FFFF8003FFDF8001FFDA
:10C96B00BF80007E3F8000003F8000003F800000C2
:10C97B003F0007C03F001FC07F001FE07E000FF18C
:10C98B00FE000FFFFE000FFFFC0007FFF80003FF88
:10C99B00F00001FFC000007F00000F00000000004E
:10C9AB000000000000038007C00FE00FE00FE0075E
:10C9BB00C003800000000000000000000000000029
:10C9CB00000000000000000000038007C00FE00F14
:10C9DB00E00FE007C0038000000000000000000033
:10C9EB00002700003F00000007FFF800001FFFFEBC
:10C9FB0000007FFFFF8000FFFFFFC001FFFFFFE094
:10CA0B0003FFFFFFE007FFFFFFF007FF007FF00FC3
:10CA1B00FC001FE00FF80010001FF80000001FF0D3
:10CA2B000000001FF00000001FF00000003FF00F9F
:10CA3B00FFF83FF00FFFF83FF00FFFF83FF00FFF4D
:10CA4B00F81FF00FFFF81FF00FFFF81FF00FFFF8A4
:10CA5B001FF0001FF81FF8001FF80FF8001FF80F4A
:10CA6B00FC001FF807FF007FF807FFFFFFF803FF2D
:10CA7B00FFFFF801FFFFFFF000FFFFFFC0007FFF8C
:10CA8B00FF00003FFFFC000007FFF00000003E002E
:10CA9B00002700007C00000007FFC000003FFFF8EC
:10CAAB0000007FFFFC0000FFFFFF0001FFFFFF0006
:10CABB0003FFFFFF8007FFFFFFC007FE00FFE00F34
:10CACB00FC007FE00FF8003FE01FF8003FF01FF085
:10CADB00001FF01FF0001FF01FF0001FF01FF000F1
:10CAEB001FF83FF0001FF83FF0001FF83FF0001F4A
:10CAFB00F81FF0001FF01FF0001FF01FF0001FF0D9
:10CB0B001FF0001FF01FF8003FF00FF8003FE00F81
:10CB1B00FC007FE007FE00FFE007FFFFFFC003FF05
:10CB2B00FFFF8001FFFFFF8000FFFFFF00007FFF83
:10CB3B00FC00003FFFF8000007FFE00000007C0056
:10CB4B0000010204081020408080402010080402DD
:10CB5B00017FBFDFEFF7FBFDFE1E466982ADB75CC1
:10CB6B00707A02BC02BC02D402E302ED02F402F8BA
:10CB7B0002FB02FE030203090400000004002B0762
:10CB8B000002030405060704010203040505000166
:10CB9B0002030401020408102006000000190032F1
:03CBAB000064041F
:10CBAE00411DF700012880012900012A00417BEB7D
:10CBBE0000411A420041699300411A6B104169C14C
:10CBCE0000416C6B004169AF004213A9000042683E
:10CBDE00190000441A3D000000004269AA000A42F2
:10CBEE006601006542660F00C8411A6700620415AF
:10CBFE00D80100007A44000000000000000100800F
:10CC0E003B45000000000000000100007A450000D6
:10CC1E0000000000000100401C4600000000000063
:10CC2E00000200000000001E0000000000020000D4
:10CC3E0000000100000000000001000000000000E4
:10CC4E0000000000000000000000000000000000D6
:10CC5E0000000000000000000000000000000000C6
:10CC6E0000000000000000000000000000000000B6
:10CC7E0000000000000000000000000000000000A6
:10CC8E000000000000000000000000000000000096
:10CC9E000000000000000000000000000000000086
:10CCAE000000000000000000000000000000000076
:10CCBE000000000000000000000000000000000066
:10CCCE000000000000000000000000000000000056
:10CCDE000000000000000000000000000000000046
:10CCEE000000000000000000000000000000000036
:10CCFE000000000000000000000000000000000026
:10CD0E000000000000000000000000000000000015
:10CD1E000000000000000000000000000000000005
:10CD2E0000000000000000000000000000000000F5
:10CD3E0000000000000000000000000000000000E5
:10CD4E0000000000000000000000000000000000D5
:10CD5E0000000000000000000000000000000000C5
:10CD6E0000000000000000000000000000000000B5
:10CD7E0000000000000000000000000000000000A5
:10CD8E000000000000000000000000000000000095
:10CD9E000000000000000000000000000000000085
:10CDAE000000000000000000000000000000000075
:10CDBE000000000000000000000000000000000065
:10CDCE000000000000000000000000000000000055
:10CDDE000000000000000000000000000000000045
:10CDEE000000000000000000000000000000000035
:05CDFE00000000000030
:10004600759850438780758DFEE589540F4420F5D9
:1000560089D28EC2ABD2ACC20CC20FE4901A41F068
:090066009017E2F0C298C2992241
:10006F00D20F9002D57406F09002D4E0FF24809056
:10007F006994F0901A417401F0C2998F99C20D22C0
:10008F00D20F9002D57406F09002D4E0FF24809036
:10009F006994F0901A417401F0C2998F99C20D22A0
:030023000200AF29
:1000AF00C0E0C0F0C083C082C0D075D00830993294
:1000BF00C299300F2D901A41E0C394C85003E00449
:1000CF00F0906994E0FF901A41E0FED39F4006E460
:1000DF00F0C20F800D74D32EF582E43402F583E065
:1000EF00F599309847C298900000E599F09017E283
:1000FF00E0C394C85003E004F0900000E0FF9017B5
:10010F00E2E0FE240FF582E43415F583EFF0EFF40F
:10011F00701AEEFF7E0078087C027D027B027A1552
:10012F00790F12EAA5D20CE49017E2F0D0D0D0826A
:07013F00D083D0F0D0E032C4
:06000600200FFDD20D22C7
:1001460090BFFFE05403B403F790BFFF7481F090B3
:10015600BFFFE05403B403F790BFFF7498F090BF5D
:10016600FFE05403B403F790BFFEE4F090BFFFE056
:100176005403B403F790BFFEE4F090BFFFE05403CE
:10018600B403F790BFFF7442F090BFFFE05403B48E
:1001960003F790BFFE741EF090BFFFE05403B40354
:1001A600F790BFFEE4F090BFFFE05403B403F7906E
:1001B600BFFF7443F090BFFFE05403B403F790BF52
:1001C600FEE4F090BFFFE05403B403F790BFFE7463
:1001D6000FF090BFFFE05403B403F790BFFF7440E5
:1001E600F090BFFFE05403B403F790BFFE7428F00D
:1001F60090BFFFE05403B403F790BFFEE4F090BF56
:10020600FFE05403B403F790BFFF7441F090BFFFC3
:10021600E05403B403F790BFFEE4F090BFFFE05450
:1002260003B403F790BFFEE4F090BFFFE05403B4BD
:0902360003F790BFFF7424F022CD
:10023F00EF1460201460541470030202D124036081
:10024F000302033E7E0F7F007D007B027A6C79E311
:10025F0012EE9D227564047565CE756329E563C33F
:10026F009470400302033E7E007F107D0074E325EF
:10027F0065F9746C3564FA7B0212EE9D741E256568
:10028F00F565E43564F564056380D27564037565BF
:10029F004975631CE563C39480400302033E7E00EF
:1002AF007F0E7D0074E32565F9746C3564FA7B026B
:1002BF0012EE9D741E2565F565E43564F5640563DE
:1002CF0080D275640B7565D6756365E563C39472EB
:1002DF0050247E007F1A7D0074E32565F9746C3518
:1002EF0064FA7B0212EE9D741E2565F565E4356494
:1002FF00F564056380D5741E2565F565E43564F5F1
:10030F0064756373E563C3948050247E007F1A7D08
:10031F000074E32565F9746C3564FA7B0212EE9D67
:10032F00741E2565F565E43564F564056380D52293
:10033F0075600275616C7562E375A61E75A6E1E4C2
:10034F00FFEFC3940F4003020478E4FE90BFFFE079
:10035F005403B403F790BFFEEEF090BFFFE05403D9
:10036F00B403F790BFFEEFF090BFFFE05403B40368
:10037F00F790BFFF7424F0902D82E0605590BFFF7F
:10038F00E05403B403F790BFFEEEF090BFFFE054CC
:10039F0003B403F790BFFEEFF090BFFFE05403B438
:1003AF0003F790BFFF7424F090BFFFE05403B40332
:1003BF00F7AB60AA61A96212EAD790BFFEF090BFB7
:1003CF00FFE05403B403F790BFFF74C4F0E4902D23
:1003DF0082F090BFFFE05403B403F7AB60AA61A9AA
:1003EF006212EAD790BFFEF090BFFFE05403B40350
:1003FF00F790BFFF74C4F0902D82E0605590BFFF5F
:10040F00E05403B403F790BFFEEEF090BFFFE0544B
:10041F0003B403F790BFFEEFF090BFFFE05403B4B7
:10042F0003F790BFFF7424F090BFFFE05403B403B1
:10043F00F7AB60AA61A96212EAD790BFFEF090BF36
:10044F00FFE05403B403F790BFFF74C4F0E4902DA2
:10045F0082F074012562F562E43561F561EEF460B6
:0A046F00040E02035B0F020350228B
:10047900EFC394F0503BEDC394805035EF13131341
:10048900541FFE75F01EEDA42EF582E435F0F583B8
:10049900E58224E3F582E583346CF583C083C08269
:1004A900E0FEEF540790CB5493FFEE4FD082D083F8
:0204B900F0222F
:10000C00AC07ECD39B5008AF041204790C80F3229C
:10002E00AC07EDD39B5008AF041204790D80F32278
:0A04BB007B027A0179C81204C52201
:1004C5008F638D648B658A668967E4900001F0AB64
:1004D50065AA66A96712EAD7FF606FB45E1290003D
:1004E50001E090CB6493F563900001E004F0804D4A
:1004F500EF24E0FFE434FFFE7C007D0B12EB358E2C
:10050500688F6974F92FF974B33EFA7B05AD63857D
:10051500646F74F82FF582EE34B3F583E493F570C8
:1005250075710A1207FF74F82569F582E56834B319
:10053500F583E4932563F563C394F0500D740125A9
:0B05450067F567E43566F566808522E7
:10055000E4FE8B688A69896AAB68AA69A96A12EAAB
:10056000D7FD601F75F00BA42498F582E5F034B236
:10057000F583E4932EFE7401256AF56AE43569F586
:100580006980D5EF24FE6009047010C3E5679EFF03
:0E05900022EEC313FFC3E5679FFF227F002208
:0A059E007B027A0179C81205A82239
:1005A8008F638D648B658A668967E4900002F0AB7F
:1005B80065AA66A96712EAD7FF70030206AA644013
:1005C8007049E56475F01EA4AEF024C5F56AEE34F2
:1005D800FFF569E4F568E568C3940F400302069CDB
:1005E8007E007F1C901DF7E075F0FFA4FD74E325E5
:1005F8006AF9746C3569FA7B0212EE9D741E256ADD
:10060800F56AE43569F569056880CBAB65AA66A922
:100618006712EAD7FFB45E12900002E090CB6A93AB
:10062800F563900002E004F0806AEFB4C712E4B406
:10063800FF0E90B84493FC7401938C69F56A801698
:10064800EF25E024C2F582E434B7F583E493FE7421
:1006580001938E69F56A74C1256AF974B83569FA27
:100668007B05AD6385646F74C0256AF582E56934DE
:10067800B8F583E493F57075710D1207FF74C02502
:100688006AF582E56934B8F583E4932563F563C3B5
:1006980094F0500E74012567F567E43566F5660237
:0306A80005B72271
:1006AB00E4FE8B658A668967AB65AA66A96712EA61
:1006BB00D7FD602B25E024C2F582E434B7F583E443
:1006CB0093FC74019324C0F582EC34B8F583E49366
:1006DB002EFE74012567F567E43566F56680C9EF74
:1006EB0024FE6009047010C3E5649EFF22EEC31361
:0A06FB00FFC3E5649FFF227F002289
:0A0705007B027A0179C812070F2267
:10070F008F578D588B598A5A895BAB59AA5AA95B57
:10071F0012EAD7FF605C25E0241EF582E434BFF5B2
:10072F0083E493FE7401938E5CF55D2495F974BF99
:10073F003EFA7B05AD5785586F7494255DF582EEB3
:10074F0034BFF583E493F5707571161207FF749437
:10075F00255DF582E55C34BFF583E4932557F557A6
:10076F00C394F0500D7401255BF55BE4355AF55ACF
:03077F008098223D
:0A0782007B027A0179C812078C226D
:10078C008F608D618B628A638964AB62AA63A96492
:10079C0012EAD7FF605C25E024D2F582E434C2F57E
:1007AC0083E493FE7401938E65F566244FF974C34C
:1007BC003EFA7B05AD6085616F744E2566F582EE61
:1007CC0034C3F583E493F5707571231207FF744EEF
:1007DC002566F582E56534C3F583E4932560F56001
:1007EC00C394F0500D74012564F564E43563F5632E
:0307FC00809822C0
:1007FF008B6B8A6C896D8D6EED2570F577E433F513
:10080F0076D3E57794F0E57694004006757600751B
:10081F0077F0E5702407FF131313541FF57012932D
:10082F0056856F74E4F572E572C395714003020942
:10083F0044856E75E4F573E573C395704003020943
:10084F003DAB6BAA6CA96D12EAD7FDE574C394801A
:10085F004003020927E57554077039E575C394E81D
:10086F005032E575131313541FFB7A00E57475F0BE
:10087F001EA42BFFEA35F0FE901DF7E06005EDF4A6
:10088F00FC8002AC0574E32FF582EE346CF583EC3B
:10089F00F00209277980AC75E5752408FFECC39F3A
:1008AF004003020927ECC395775066EC13131354DA
:1008BF001FFB7A00E57475F01EA42BFFEA35F0FEDE
:1008CF00901DF7E06005EDF4FB8002AB05EB59607E
:1008DF002174E32FF582EE346CF583C083C082E080
:1008EF00FBEC540790CB5493FAEB4AD082D083F0B1
:1008FF00801F74E32FF582EE346CF583C083C082C2
:10090F00E0FFEC540790CB5C93FEEF5ED082D08378
:10091F00F0E9C313F90C808074082575F57574011F
:10092F00256DF56DE4356CF56C057302084605749D
:06093F00057202083622D9
:100945008F63AA05A903E56304FFE914FB12000CF4
:10095500E56304FFAD66AB0112000CAF63EA04FD6D
:10096500E56614FB12002EAF01EA04FDE56614FBF3
:1009750012002EE914FFE56614FD120479E904FF5F
:10098500EA2402FDAB6612002EE5632402FFE5664C
:0809950004FDAB0112000C226D
:10099D007F4A7D6C7B6D7566791209457F5C7D752F
:1009AD001204797F5B1D7B5D12000C7F5A1D0B12AB
:1009BD00000C7F591D0B12000C7F581D0B12000CE3
:1009CD007F571D0B12000C7F8B7D6C7BAE7566798E
:1009DD001209457F9D7D701204797F9C0D7B9E12BF
:1009ED00000C7F9B0D0B12000C7F9A0D0B12000C4F
:0F09FD007F990D0B12000C7F980D0B12000C222E
:100A0C00D297D296C297E4FFEFC394105004000F14
:050A1C0080F6C29622E5
:100A2100C297D296E4FFEFC394105004000F80F6F2
:030A3100D2972237
:100A34003097047F0180027F00D296E4FEEEC394D7
:0A0A4400105004000E80F6C2962246
:06001C00D297120A342203
:100A4E00AD07E4FBEBC39408500EED339297120AF8
:090A5E0034ED25E0FD0B80EC22D3
:100A6700E4FDFCECC39408500EED25E0FD120A34BA
:0A0A7700EF60010D0C80ECAF0522CA
:100A81008E5B8F5C8B5D8A5E895FE4F563F564C381
:100A9100E5649561E56395605067908002E0F52A11
:100AA10020E3037F0122120C2AEF7002FF22120AB7
:100AB1000C7FA0120A4E12001CE55BFF120A4E12B7
:100AC100001CAF5CE55C120A4E12001C120A0C7F7E
:100AD100A1120A4E12001C120A67AB5DAA5EA95F41
:100AE100EF12EB217401255FF55FE4355EF55E05DC
:100AF1005CE55C7002055B0564E56470020563807A
:100B01008EAB5DAA5EA95FE412EB21D297120A3483
:060B1100120A217F0122FF
:100B17008E4A8F4B8B4C8A4D894EE4900003F090A0
:100B27008002E0F52A20E3037F0122120C2AEF70EE
:100B370002FF22120A0C7FA0120A4E12001CE54A7D
:100B4700FF120A4E12001CAF4BE54B120A4E120061
:100B57001CAB4CAA4DA94E12EAD7FE7009900003B0
:100B6700E0C3954F5030908002E0F52A20E3037FE1
:100B77000022EE6011FF120A4E7401254EF54EE475
:100B8700354DF54D8005E4FF120A4E12001C90000A
:0C0B970003E004F080BB120A217F012261
:100BA3008E578F588B598A5A895BE4900004F090D2
:100BB3008002E0F52A20E3037F0122900004E0C3D2
:100BC300955C5060120C2AEF7002FF22908002E0C5
:100BD300F52A20E3037F0022120A0C7FA0120A4E9B
:100BE30012001CE557FF120A4E12001CAF58E558BD
:100BF300120A4E12001CAB59AA5AA95B12EAD7FF7C
:100C0300120A4E7401255BF55BE4355AF55A12005E
:100C13001C900004E004F00558E5587002055712D3
:070C23000A2180977F0122E6
:100C2A00E4F566120A0C7FA0120A4E12001C8F65A8
:100C3A00129356E566B4FA037F00220566E56570ED
:070C4A00E2120A217F0122E2
:100C5100438E02123980129356906C6BE0D394321A
:100C6100400A7F1B124009E4906C6BF0D390681A24
:100C7100E0942C906819E094014019902D8BE0705C
:100C81000C12033F7F02E4FD7B01128EDAE49068CF
:100C910019F0A3F09069C2E06003020D317B027A82
:100CA10000790612DE3EEF644270677F417EF0FDFF
:100CB100FC12EE25900006E0FCE412E64312E5EAA0
:100CC100406E7F437E707D007C0012EE2590000611
:100CD100E0FCE412E64312E5EA600250539000069C
:100CE100E0FB901DFAF07F457EBB7D807C0012EE1B
:100CF10025AC03E412E64312E53B12E6779069D294
:100D0100EEF0A3EFF0E49069A8F0A3F0D208D20BC3
:100D1100801EC39069A9E094BC9069A8E094024048
:100D21000FE4901DFAF09069A8F0A3F0D208D20B5D
:090D31007F71124009020C5722E7
:0300430002002692
:0100260032A7
:03000300020D3AB1
:100D3A00C0E0C0F0C083C082C0D075D018129356EC
:100D4A00E490681EF0200803020E2CC208D3906CAF
:100D5A00E0E09401906CDFE094005003020E2C7FD7
:100D6A00417EF07D007C0012EE25901DFAE0FCE445
:100D7A0012E64312E5EA5003020E2C7F437E707D91
:100D8A00007C0012EE25901DFAE0FCE412E6431204
:100D9A00E5EA60054003020E2C9069D2E0FAA3E06E
:100DAA00FB901DF3E02BF0901DF2E03AF0901DDE6F
:100DBA0012EDBC12EE25AF1BAE1AE4FCFD12EC02DA
:100DCA00901DDE12EDD8901DF1E004F0901DDA12AC
:100DDA00EDBC12EE257F017E007D007C0012EC0244
:100DEA00901DDA12EDD8901DDA12EDBCE412E63B42
:100DFA0012EE257F427EC87D007C0012E4C312EE0B
:100E0A0025901DDE12EDBCE412E63B12EE257F4270
:100E1A007E707D007C0012E53B12E53B901DA2121C
:100E2A00EDD8200E03021242C20EE4906C75F0A3B4
:100E3A00F0906CDFE0FEA3E0FFD39401EE94005043
:100E4A00030210D2EF64024E700C90681D04F0E4A5
:100E5A009013A9F0A3F0125672901DC212EDBC12A3
:100E6A00E6777C007D0A12EB49901DF6E0FD75F0ED
:100E7A0002A424B3F582E5F03413F583EEF0A3EF70
:100E8A00F075F002EDA424B3F582E5F03413F5838E
:100E9A00E0FEA3E0FFC390668DE09F90668CE09E23
:100EAA005005EEF0A3EFF075F002EDA424B3F5823D
:100EBA00E5F03413F583C083C082E0FEA3E0FF7C33
:100ECA00007D4412EB35D082D083EEF0A3EFF09090
:100EDA001DBE12EDBC12E6777C007D0A12EB49902A
:100EEA001DF6E0FD75F002A42427F582E5F034141E
:100EFA00F583EEF0A3EFF075F002EDA42427F58256
:100F0A00E5F03414F583E0FEA3E0FFC390668FE0BA
:100F1A009F90668EE09E5005EEF0A3EFF075F0020A
:100F2A00EDA42427F582E5F03414F583C083C0824A
:100F3A00E0FEA3E0FF7C007D4412EB35D082D08333
:100F4A00EEF0A3EFF0901DC612EDBC12E6777C001E
:100F5A007D0A12EB35901DF6E0FD75F002A4249B84
:100F6A00F582E5F03414F583EEF0A3EFF075F002A4
:100F7A00EDA4249BF582E5F03414F583E0FEA3E0AA
:100F8A00FFC3906691E09F906690E09E5005EEF058
:100F9A00A3EFF075F002EDA4249BF582E5F034147A
:100FAA00F583C083C082E0FEA3E0FF7C007D44128B
:100FBA00EB35D082D083EEF0A3EFF0901DF6E0047B
:100FCA00F0E0FFC3943A400E9065E7E004F0700643
:100FDA009065E6E004F0EF75F03A84901DF6E5F0CE
:100FEA00F0901DFBE070030212421200069002D438
:100FFA0074BAF09002D6744CF0754004E4F53FE5FB
:10100A003FC3940B40030210CCE53F75F003A424C0
:10101A0045F582E4341AF583E0FBA3E0FAA3E0F98C
:10102A0012ED7E8F278E268D258C24E524547FFF92
:10103A00AE40054074D32EF582E43402F583EFF016
:10104A00E525547FFFAE40054074D32EF582E43483
:10105A0002F583EFF0E526547FFFAE40054074D3D6
:10106A002EF582E43402F583EFF0E527547FFFAED4
:10107A0040054074D32EF582E43402F583EFF0E59F
:10108A0025A2E713A2E7135420FFE524A2E713548D
:05109A00404FFFE526B8
:10109F007803A2E713D8FB54104FFFE5277804A27B
:1010AF00E713D8FB54084FFFAE40054074D32EF51D
:1010BF0082E43402F583EFF0053F02100912006F4E
:1010CF00021242906CDFE07004A3E064016003023F
:1010DF001242901A43E02486601024FE601A240402
:1010EF007022901A437479F0801A901A43747BF02F
:1010FF009013A67401F0800C901A43747DF0901336
:10110F00A67401F07E007F667D007B027A1D798ECA
:10111F0012EE9D7E007F637D007B027A6C797712E1
:10112F00EE9D9003A1E0C3942840297427F0E0FFBF
:10113F007E007C007D6312EB35741B2FF9741E3E0D
:10114F00FA7B02C01B78C67C69AD1BD01B7E007F6B
:10115F000612EAA578907C6C7D027B027A6979C6CB
:10116F007E007F0612EAA578967C6C7D027B027A60
:10117F006979C67E007F0612EAA5906C7C12EDE4B9
:10118F0000000000906C9E12EDE400000000906CD7
:10119F00867403F09069C6E0D394034003021230C3
:1011AF009069B9E07003FF80079069B9E02402FFEE
:1011BF00906CA2EFF09069B9E025E024A5F582E4E8
:1011CF0034CBF583E493740193906CB1F09013AE2C
:1011DF00E0906CA3F090660312EDBC906CA412ED3E
:1011EF00D890660712EDBC906CA812EDD890660BE4
:1011FF0012EDBC906CAC12EDD89002D1E0906CB0B7
:10120F00F09013AF12EDBC906C8712EDD8906695ED
:10121F0012EDBC906C8B12EDD89013A7E0906C8FF1
:10122F00F0902D8B7401F090681DF0901DF4F090EC
:10123F00667CF0432980908001E529F090681E7448
:0D124F0001F0D0D0D082D083D0F0D0E032BA
:03002B0002125C62
:10125C00C0E0C0F0C083C082C0D075D010C2CF90A7
:10126C006C76E004F07006906C75E004F090667C8F
:10127C00E0601DC3906CE0E09401906CDFE09400A2
:10128C00400E901DE8E004F07006901DE7E004F0BD
:10129C00901A6BE0700312961D9065E8E0D39400F1
:1012AC004005E014F08003432880908000E528F08E
:1012BC009069A9E004F070069069A8E004F09068C9
:1012CC001AE004F07006906819E004F0906C6BE082
:1012DC0004F09013AAE004F070069013A9E004F057
:1012EC00C39013AAE0942C9013A9E0940140199098
:1012FC00681D7401F0E49013A9F0A3F0FF12939809
:10130C009066A7EEF0A3EFF090667CE0600312937A
:10131C00C5907BE8E070030218ED906820E0600354
:10132C000218ED90667CE0601A901DB612EDBC12AE
:10133C00EE257F3F7E807D007C0012E3B8901DB6C9
:10134C0012EDD89069B9E0D3940050030213E490E5
:10135C00669BE0FF9069C1E0C39F50030213E4E475
:10136C00F090669AE0FF9069BFE02FFF9069BEE0B5
:10137C003400FE90669BE0FD7C0012EB9E9017E023
:10138C00EEF0A3EFF0E49069BEF0A3F09065EAE014
:10139C00902D83F0E49065EAF09069B0E09069904C
:1013AC00F0E49069B0F0906C67E09001C7F0E490C5
:1013BC006C67F09069C0E09065FCF0E49069C0F057
:1013CC0090667CE06012C3906CE0E09401906CDF5E
:1013DC00E09400400312438F9069C1E004F09068E0
:1013EC0021E07003021545906601E0FEA3E0FF24A6
:1013FC0064901E01F0E43E901E00F0901A67E0FD30
:10140C00B402047C0180027C00907BEAECF0EDB429
:10141C0002047C0180027C00906C74ECF0EDB40151
:10142C00047D0180027D00906CDAEDF0E4901A6787
:10143C00F09069AAE0FCA3E02FFFEE3CFE90660F53
:10144C00E0FCA3E0FDC3EF9DEC6480F8EE648098B3
:10145C00400A9069AA74FFF0A374F6F09069AAE0B0
:10146C00FEA3E0FF906602E02FFF906601E03EFED7
:10147C009013ADE0FCA3E0FDD3EF9DEC6480F8EE9F
:10148C00648098400302152F901A3D12EDBC12EEA9
:10149C00257F017E007D007C0012EC02901A3D122B
:1014AC00EDD8901A3D12EDBC12EE257F027E007D28
:1014BC00007C0012F67212EE4CEC4D4E4F60047F25
:1014CC000180027F02901A67EFF09069AAE4F0A302
:1014DC00740AF0EF6402704B906610E02405F090F3
:1014EC00660FE03400F0E0FEA3E0FF7C027D5812B2
:1014FC00EB9E90660FECF0A3EDF09013ADE0FEA325
:10150C00E0FFD3ED9FEE6480F8EC6480985014906B
:10151C0013AEE024C8906610F09013ADE034009048
:10152C00660FF09069AAE0FEA3E0FF906602E02F40
:10153C00F0906601E03EF080447F01129398901E7B
:10154C0000EEF0A3EFF07F01129398901E00EEF0E6
:10155C00A3EFF030C0047F0180027F00907BEAEFA4
:10156C00F03092047F0180027F00906C74EFF030B9
:10157C0094047F0180027F00906CDAEFF09069C2D6
:10158C00E064026003021647901DF5E004F09069D8
:10159C00C0E004F0901DF5E0FF700D907BE904F0C5
:1015AC00E4901DFAF002163F907BEAE070030216FD
:1015BC003F906C6CE0600302163F907BE9EFF0FB10
:1015CC00E4901DF5F0906C6704F0E49069C0F07F36
:1015DC00417EF0FDFC12EE25AC13E412E64312E55D
:1015EC00EA40197F437E707D007C0012EE25907BD3
:1015FC00E9E0FCE412E64312E5EA4007E4901DFA48
:10160C00F08030907BE9E0FB7A007EEA7F60FDACF5
:04161C001212EB4972
:10162000EF2405FFE43EFE7C007D0A12EB49901D8D
:10163000FAEFF09069D2EAF0A3EBF0D208D20B9067
:101640007BEAE0906C6CF0901DFBE07006200D03CF
:10165000121917901E00E0FEA3E0FF9069BFE02F73
:10166000F09069BEE03EF09013ADE0FCA3E0FDD346
:10167000EF9DEC6480F8EE648098500F9013ADE01D
:10168000FFA3E0901E00CFF0A3EFF0906CDAE0FF34
:101690006019906C68E07013901A687402F0906999
:1016A000B014F0901A6CE09013ACF0906C68EFF00E
:1016B000906C74E0FB70030217AE906C65E0600301
:1016C0000217AE901A68E0640260030217AE04F0DD
:1016D0009065EAF0902F2DE0FFA3E090681BCFF01B
:1016E000A3EFF0E4902F2DF0A3F09069BA12EDBCB7
:1016F000902D8612EDD89069BA12EDE4000000003A
:10170000906CE0E004F07006906CDFE004F0902F45
:1017100032E0902F31F0B401047F0080027F01900D
:101720002F32EFF0901A6CE09013A5F09013ACE01C
:10173000907BE7F09066A0E0902D81F090698C128C
:10174000EDBC9065ED12EDD890039CE0FFA3E09016
:101750006692CFF0A3EFF0907BE7E025E0FFE43363
:10176000FE748A2FF582EE342DF583E0FFA3E0901E
:101770006822CFF0A3EFF0E4901A6CF09013ACF075
:1017800090698C12EDE400000000E49066A0F090F7
:10179000039CF0A3F09065E9E0600BE4906992F09F
:1017A0009065E9F080069069927401F0D20E906C19
:1017B00065EBF09013ADE0FEA3E07802C333CE33C7
:1017C000CED8F924A2F582EE3403F58312EDBC12D3
:1017D000EE25901E00E0FEA3E07802C333CE33CEA8
:1017E000D8F924A2F582EE3403F58312EDBC12EC95
:1017F0001590000912EDD89069BA12EDBC12EE25D1
:1018000090000912EDBC12EC029069BA12EDD8906A
:10181000000912EDBC780C12ED57900008EFF09023
:101820001A6CE0C394C740030218BC900008E0F9AA
:10183000FF7E009017E3E0FCA3E0FD12EB35AC1651
:10184000AD17901A6CE025E0FFE433FE902F32E0F4
:10185000FB75F090A4246EF582E5F0341AF583EB65
:101860002583F583E5822FF582EE3583F583ECF051
:10187000A3EDF09066A0E0C399500EE9F090000946
:1018800012EDBC90698C12EDD8E9FF90039DE02F1A
:10189000F090039CE03400F0E0FCA3E0FD901A6CB3
:1018A000E025E0FFE433FE748C2FF582EE342DF555
:1018B00083ECF0A3EDF0901A6CE004F0C3902F2EAF
:1018C000E094B8902F2DE0940B40069013A6E060B2
:1018D00010902F2EE004F07006902F2DE004F08081
:1018E0000C902D8BE06006902D8A7401F090681E9C
:1018F000E06009200E0330080353297F908001E542
:1019000029F0902D827401F0902D84F0D0D0D082F7
:07191000D083D0F0D0E032DB
:101917001200069002D47488F09002D67435F090C5
:101927001E00E0FCA3E0FDAE147803CEA2E713CEC1
:1019370013D8F8547F9002D7F0901DFAE0FFC31335
:10194700547F9002D8F0E4A3F0ED30E004E04401C6
:10195700F0906C74E0600D906C65E070079002D9B0
:10196700E04402F0E49002DAF0901E00E0FEA3E00B
:10197700FF30E1079002DAE04401F0906CDAE060B2
:101987000D906C68E070079002DAE04402F0E49092
:1019970002DBF0EF30E204E04401F0901DFAE030A2
:0D19A700E0079002DBE04402F012008F2206
:1019B4008D5AAB07AA06E4900010F0A3F0A3F0A39D
:1019C400F0A312EDE40000000090001812EDE40012
:1019D40000000090001C12EDE400000000900020C4
:1019E40012EDE40000000090002412EDE400000079
:1019F40000906CE2E06026AE02AF037C007D0A1228
:101A0400EB35906C78E02428FD906C77E03400CDC1
:101A14002F90000FF0ED3E90000EF08012906C9528
:101A2400E02B90000FF0906C94E03A90000EF012CE
:101A3400935690668812EDE400007042E490000D25
:101A4400F090000DE0FF9065FFE0FCA3E0FDC3EF24
:101A54009DE49C4003021CC5906CE2E07003021BF1
:101A640016906C79E0FEA3E0FF24F6FDEE34FFFC53
:101A740090000EE0FAA3E0FB6D7002EC6A706190D6
:101A84006C7BE0705B906C78E02428FD906C77E0D0
:101A94003400FCC3EF9DFFEE9CFE7C007D0A12EB3C
:101AA40049EF24FFFFEE34FFFEE4FCFD12EE257F38
:101AB400707E177D007C0012EC2912EE25906C7C60
:101AC40012EDBC12EC15E412E63B12EE257F427EC9
:101AD400C87D007C0012E53B90668812EDD8801822
:101AE400906C79E0FEA3E0FFC390000FE09F9000AC
:101AF4000EE09E4003021CC590000EE0FEA3E0FF32
:101B04007B027A66797E75600075610A120A810229
:101B14001BC8906C9AE0FEA3E0FF24FFFDEE34FFA7
:101B2400FC90000EE0FAA3E0FB6D7002EC6A7052C8
:101B3400906C9CE0704C906C94E0FCA3E0FDC3EFCF
:101B44009DFFEE9CCF24FFCF34FFFEE4FCFD12EE9C
:101B5400257F707E177D007C0012EC2912EE259003
:101B64006C7C12EDBC12EC15E412E63B12EE257F00
:101B7400427EC87D007C0012E53B90668812EDD859
:101B84008018906C9AE0FEA3E0FFC390000FE09FE2
:101B940090000EE09E4003021CC590000EE0FEA3E0
:101BA400E0FF7C007D0A12EB3574332FF9742F3E6D
:101BB400FA7B02C003787E7C66AD03D0037E007F8F
:101BC4000A12EAA590001412EDBC12EE2590667E6E
:101BD400E0FCA3E0FDE412E63F12EE257F447E7AAA
:101BE4007D007C0012E53B12E3B890001412EDD89E
:101BF40090001812EDBC12EE25906685E0FCA3E07F
:101C0400FDE412E63F12E3B890001812EDD8E55A4D
:101C140020E00920E10620E20330E34A900020128C
:101C2400EDBC12EE25906680E0FCA3E0FDE412E634
:101C34003F12E3B890002012EDD890002412EDBCBE
:101C440012EE25906682E0FCA3E0FDE412E63F126A
:101C5400EE257F417E207D007C0012E53B12E3B837
:101C640090002412EDD8E55A30E412906684E0FF27
:101C7400900011E02FF0900010E03400F0E55A30AD
:101C8400E512906687E0FF900013E02FF0900012B9
:101C9400E03400F0906CE2E0601090000FE0240A61
:101CA400F090000EE03400F0800E90000FE004F09D
:101CB400700690000EE004F090000DE004F0021AAB
:101CC400457E007F187D007B027A6979D412EE9DEF
:0C1CD40090668812EDBC12EE2590000D09
:101CE000E014FCE412E64312EE257F427E707D0094
:101CF0007C0012E4C312E3B890668812EDD890001D
:101D00000DE07003021E437F007E007D007C001208
:101D1000EE2590001412EDBC12E5EA601C401A900A
:101D2000002012EDBC12EE2590001412EDBC12E55D
:101D30003B9069D412EDD8800A9069D412EDE4008A
:101D40000000007F007E007D007C0012EE2590697F
:101D5000D412EDBC12E5EA602A402890002412ED6E
:101D6000BC12EE2590001412EDBC12E53B12EE25DC
:101D70007F407E667D667C6612E4C39069DC12ED6E
:101D8000D8800A9069DC12EDE40000000090002089
:101D900012EDBC9069D812EDD890002412EDBC90E1
:101DA00069E012EDD8900010E0FCA3E0FDE412E63B
:101DB0003F12EE2590001412EDBC12EE257F427EFC
:101DC000707D007C0012E53B12E53B9069E412ED6A
:101DD000D8900012E0FCA3E0FDE412E63F12EE25ED
:101DE0007F427EC87D007C0012E4C312EE25900085
:101DF0001812EDBC12EE257F427E707D007C001231
:101E0000E53B12E53B9069E812EDD87F417EF07D1D
:101E1000007C0012EE259069E812EDBC12E5EA4064
:101E2000187F437E707D007C0012EE259069E812D9
:101E3000EDBC12E5EA600C400A9069E812EDE4009E
:091E400000000090000DE0FF22FB
:101E4900E4906C75F0A3F0906991E070087F65FDEE
:101E5900FB1296052290020BE075F00AA4FF90028E
:101E69000AE075F064A42FFF90020CE02F9000287F
:101E7900F012EE771EED101EDC171F49181F5819B6
:101E89001EE21A1EE21B1EFF1C1F271D1F0B1F1F10
:101E99001F201EF3211F3B221ED6301F6C311F8BC2
:101EA900371EC0491F964D1FA84E20895020C75183
:101EB90020C752000020F07F01124AE7901A4374AC
:101EC90002F0E4FF1249EF129DE10220F01244559D
:101ED9000220F01220FD0220F0900028E0FF129568
:101EE9005B0220F01295DC0220F07F217D03E4FBE8
:101EF9001296050220F07F1C7D18E4FB129605025C
:101F090020F0901A43E064B660030220F074B9F03F
:101F190012351F0220F07F01129CA00220F0901AB6
:101F290043E064B560030220F074B8F012351F0273
:101F390020F07F067B027A6579F812A0BE0220F0B4
:101F490012437BEF60030220FC124DCD0220F012F8
:101F5900437BEF60030220FC90020DE0FF124F9ECD
:101F69000220F012437BEF60030220FC7F0112493B
:101F790029E4FF12023F901A437402F012351F023E
:101F890020F07F37E4FDFB1296050220F0901A43FA
:101F990074BEF07F187DFFE4FB1296BB0220F07F30
:101FA9004EE4FDFB12960590020DE0FF7E007C00D9
:101FB9007D6412EB3512935D7F077B027A66791196
:101FC90012A0BE90661112EDBC9069B312EDD890C3
:101FD90013AB7406F0901A4374BFF0E490669CF05A
:101FE900A3F0A37406F0E4A3F0902D8004F09066AA
:101FF9007CF09065ECF0E4902F20F0902D7A12EDB2
:10200900E4000000009069CE12EDE40000000090A9
:1020190013ABE0D39400403C1293569065ECE0601A
:10202900149013ABE014F07F18E0FDE4FB1296BBAB
:10203900E49065ECF07F52129DB9EF60D2C20C902A
:102049001A437402F0901A6B7410F07F1AE4FDFBC6
:102059001296BB22E4906C71F07F067D0112841DFB
:10206900906CDFE4F0A304F0D20E53297F90800135
:10207900E529F0907BE87401F090669404F080679C
:10208900901DFBE0606190020DE0902F20F07F062B
:102099007B027A66791112A0BE90661112EDBC908E
:1020A9002D7A12EDD87F0B7B027A66791112A0BEC8
:1020B90090661112EDBC9069CE12EDD88029901D61
:0720C900FBE06023901A43C5
:1020D00074C0F0901A6B7410F0900028E0B45104B2
:1020E0007F1980027F1A90020DE0FDE4FB1296BB7F
:0D20F0007F7E900028E0FDE4FB12960522A3
:1020FD001200069002D474A4F09002D6744BF07FB7
:10210D00049013ADE0FCA3E0FD129FCF7F08900279
:10211D00D1E0FD7C00129FCF90660312EDBC8F4F76
:10212D008E4E8D4D8C4C7F0A129FFD90660712EDE1
:10213D00BC8F4F8E4E8D4D8C4C7F0F129FFD906638
:10214D000B12EDBC8F4F8E4E8D4D8C4C7F14129F0C
:10215D00FD9013AF12EDBC8F4F8E4E8D4D8C4C7F7D
:10216D0019129FFD90669512EDBC8F4F8E4E8D4DC1
:10217D008C4C7F1E129FFD7F239013A7E0FD7C00EA
:07218D00129FCF12006F2228
:10219400E4F548EF24E070030224FB24E07003021A
:1021A400291D24C07003022D24249070030234BD21
:1021B40024E0600302351C901A43E012EE772331C9
:1021C40002233103233104233105233106233A0743
:1021D400233A08233A09233A0A233A0B23430C23CC
:1021E400430D23430E23430F234310234311234C56
:1021F40012234C13234C14234C15234C16234C1735
:1022040023551823601923601A23601B23601C23A1
:10221400601D23601E23691F2369202369212386EF
:102224002223862323862423E42623E42723E42865
:1022340023ED2D23ED2E23ED2F248332248C332400
:10224400CB3424C23523F63923F63A23FF3C23FF4B
:102254003D23FF3E23FF3F23FF4023FF412408503B
:10226400240851241A55241A56241A57242C5A2463
:102274002C5B242C5C24235F24D46024356124DD6E
:1022840062241170241171241172230778230779B1
:10229400231B7A231B7B231B7C231B7D239A7E23F6
:1022A400A37F23AC8023B58123B582233183237498
:1022B4008C23748D23748E23748F237490237491D0
:1022C400237492237DA0237DA1237DA2237DA323B8
:1022D4007DA4237DA5237DA6237DA7237DA8237D1F
:1022E400A9249EB424A7B524B0B624B9B724E6B86B
:1022F40024F2B92495BB2307BE2307BF2307C000DC
:1023040000351C7F01124AE7EF600302351C901A66
:10231400437402F002351C7F01124AE7EF600302A6
:10232400351C906694E0901A43F002351C901A43D1
:102334007402F002351C901A437403F002351C90A9
:102344001A437408F002351C901A43740AF00235DB
:102354001C906694E0901A43F002351C901A437462
:102364000BF002351C906694E0901A43F002351C81
:09237400901A43741FF002351C9D
:10237D00901A437420F002351C906CE2E060047FEB
:10238D005680027F04901A43EFF002351C901A43D9
:10239D007409F002351C901A437422F002351C901A
:1023AD001A437423F002351C9003A0E06013E4F08F
:1023BD00906820F090667CF0901A437402F002351C
:1023CD001C901A43E0B48106747FF002351C901AFC
:1023DD00437480F002351C901A437405F002351CCD
:1023ED00901A437426F002351C901A437427F0029C
:1023FD00351C901A437439F002351C901A43742819
:10240D00F002351C901A437402F002351C901A43E9
:10241D007406F002351C901A437455F002351C9069
:10242D001A437457F002351C906999E0FF647B6084
:10243D0003EF700F7E007F0A7D007B027A69799928
:10244D0012EE9D901A69E0FFC3940A501074992FF3
:10245D00F582E43469F583E0B47B02E4F0E4FF7EB9
:10246D00017B027A697999755C0B120BA3901A4363
:10247D00745AF002351C901A43742DF002351C90DD
:10248D001A43742EF002351C901A437426F002354F
:10249D001C901A437450F002351C901A437451F07D
:1024AD0002351C901A437405F002351C901A4374C2
:1024BD0028F002351C901A43742FF002351C901A27
:1024CD00437424F002351C901A43745CF002351CE1
:1024DD00901A43745BF002351C901A437451F0123C
:1024ED00930F02351C901A437405F002351C901A97
:1024FD0043E012EE7726420226420326420426428C
:10250D0005264206265D07265D08265D09265D0A1D
:10251D00265D0B266C0C266C0D266C0E266C0F267C
:10252D006C10266C11267B12267B13267B14267BC2
:10253D0015267B16267B17268A19268A1A268A1BAC
:10254D00268A1C268A1D268A1E26991F2699202634
:10255D009921275D22275D23275D24276C26276C73
:10256D0027276C28277B2D277B2E277B2F286C3444
:10257D00278A39278A3A27993C27993D27993E275B
:10258D00993F27994027994127AD5027AD5127D025
:10259D005527D05627D05727DF5A27DF5B27DF5C1B
:1025AD0027EE6127C17027C171260E78260E792678
:0125BD0028F5
:1025BE007A26287B26287C26287D28327E28327F84
:1025CE0028328028BA8128C78226BE8C26CF8D2637
:1025DE00E08E26F18F27029027139127249227351C
:1025EE00A02735A12735A22735A32735A42735A542
:1025FE0026F1A62702A72713A82724A90000351C19
:10260E00E4FFFDFBF54D123E11E490681DF07F07CF
:10261E007D017B01128EDA02351CE4FFFDFBF54DC8
:10262E00123E11E490681DF07F077D017B01128E32
:10263E00DA02351C7F047D017B02906C4BE0B408FE
:10264E00047E0680027E058E4D123E1102351C7FE1
:10265E00047D017B07754D0B123E1102351C7F0464
:10266E007D017B0C754D11123E1102351C7F047DD0
:10267E00017B12754D17123E1102351C7F047D0130
:10268E007B19754D1E123E1102351C7F047D017B98
:10269E001F901A6AE024F975F00684E5F0D39400D1
:1026AE0040047E2180027E208E4D123E1102351C8A
:1026BE00906C5AE004F0E075F00A84E5F0F0023513
:1026CE001C906C5BE004F0E075F03C84E5F0F002E9
:1026DE00351C906C5CE004F0E075F03C84E5F0F0A5
:1026EE0002351C906C5DE004F0E075F03C84E5F082
:1026FE00F002351C906C5EE004F0E075F03C84E571
:10270E00F0F002351C906C5FE004F0E075F03C8454
:10271E00E5F0F002351C906C60E004F0E075F03CE2
:10272E0084E5F0F002351C901A43E024B4F582E4FF
:10273E00346BF583E004F0901A43E024B4F582E4A0
:10274E00346BF583E075F00A84E5F0F002351C7FFA
:10275E00047D017B22754D24123E1102351C7F042F
:10276E007D017B26754D28123E1102351C7F047D9E
:10277E00017B2D754D2F123E1102351C7F047D01FC
:10278E007B39754D3A123E1102351C7F047D017B5B
:10279E003C902F30E0243BF54D123E1102351C7F4C
:1027AE00047D017B50754D51123E11E49069C5F0C8
:1027BE0002351C7F047D017B70754D71123E110236
:1027CE00351C7F047D017B55754D57123E11023528
:1027DE001C7F047D017B5A754D5C123E1102351C27
:1027EE00901A69E0FFC3940A400302351C74992FB6
:1027FE00F582E43469F583E0FE70057441F0800CD7
:10280E00EE24C075F03B84E5F02441F074992FF569
:10281E0082E43469F583E0645B600302351C746105
:10282E00F002351C902F2FE004F0906CE2E0601760
:10283E00902F2FE0FF906C45E0FEEF8EF084902FEE
:10284E002FE5F0F002351C902F2FE0FF9003A1E052
:10285E00FEEF8EF084902F2FE5F0F002351C90667F
:10286E0000E004F070069065FFE004F09065FFE074
:10287E007004A3E0643D70079065FFF0A304F09030
:10288E0065FFE0FFA3E0906611CFF0A3EFF07F04A9
:10289E007E00906611E0FD12E0B07F057E0090662E
:1028AE0012E0FD12E0B012E0C202351C7F03E4FD1F
:1028BE00FBF54D123E1102351C9065FFE0FEA3E0C4
:1028CE00FF9066AEE0FCA3E0FDD39FEC9E403D90F2
:1028DE0065FFE0FEA3E0FFC3ED9FFFEC9EFEC390FD
:0228EE006CDE9E
:1028F000E09F906CDDE09E50179065FFE0FEA3E046
:10290000FF906CDEE02FF0906CDDE03EF002351CB5
:10291000E4906CDDF0A3F002351C7F0022901A4396
:10292000E012EE772A66022A66032A66042A660502
:102930002A66062A81072A81082A81092A810A2A09
:10294000810B2A900C2A900D2A900E2A900F2A9023
:10295000102A90112A9F122A9F132A9F142A9F152A
:102960002A9F162A9F172AAE192AAE1A2AAE1B2AA8
:10297000AE1C2AAE1D2AAE1E2ABD1F2ABD202ABDAE
:10298000212B89222B89232B89242B98262B9827CE
:102990002B98282BA72D2BA72E2BA72F2C9B342B26
:1029A000B6392BB63A2BC53C2BC53D2BC53E2BC5A6
:1029B0003F2BC5402BC5412BD9502BD9512BFC5552
:1029C0002BFC562BFC572C0B5A2C0B5B2C0B5C2C2A
:1029D0001A612BED702BED712A30782A30792A4B51
:1029E0007A2A4B7B2A4B7C2A4B7D2C5E7E2C5E7F89
:1029F0002C5E802CE5812CF3822AE28C2AF48D2B2C
:102A0000068E2B188F2B2A902B3C912B4E922B60ED
:102A1000A02B60A12B60A22B60A32B60A42B60A530
:102A20002B18A62B2AA72B3CA82B4EA90000351C3F
:102A3000E4FF7D01FBF54D123E11E490681DF07F2F
:102A4000077D017B01128EDA02351CE4FF7D01FB5C
:102A5000F54D123E11E490681DF07F077D017B016A
:102A6000128EDA02351C7F04E4FD7B02906C4BE091
:102A7000B408047E0680027E058E4D123E1102359A
:102A80001C7F04E4FD7B07754D0B123E1102351CC3
:102A90007F04E4FD7B0C754D11123E1102351C7F45
:102AA00004E4FD7B12754D17123E1102351C7F04A4
:102AB000E4FD7B19754D1E123E1102351C7F04E4A6
:102AC000FD7B1F901A6AE024F975F00684E5F0D3C7
:102AD000940040047E2180027E208E4D123E110221
:102AE000351C906C5AE02409F0E075F00A84E5F09A
:102AF000F002351C906C5BE0243BF0E075F03C8408
:102B0000E5F0F002351C906C5CE0243BF0E075F0E1
:102B10003C84E5F0F002351C906C5DE0243BF0E075
:102B200075F03C84E5F0F002351C906C5EE0243BCF
:102B3000F0E075F03C84E5F0F002351C906C5FE04D
:102B4000243BF0E075F03C84E5F0F002351C906C1D
:102B500060E0243BF0E075F03C84E5F0F002351CC9
:032B6000901A4385
:102B6300E024B4F582E4346BF583E02409F0901A91
:102B730043E024B4F582E4346BF583E075F00A8412
:102B8300E5F0F002351C7F04E4FD7B22754D241231
:102B93003E1102351C7F04E4FD7B26754D28123E51
:102BA3001102351C7F04E4FD7B2D754D2F123E1160
:102BB30002351C7F04E4FD7B39754D3A123E110248
:102BC300351C7F04E4FD7B3C902F30E0243BF54D26
:102BD300123E1102351C7F04E4FD7B50754D5112EA
:102BE3003E11E49069C5F002351C7F04E4FD7B705F
:102BF300754D71123E1102351C7F04E4FD7B557542
:102C03004D57123E1102351C7F04E4FD7B5A754D6E
:102C13005C123E1102351C901A69E0FFC3940A400E
:102C23000302351C74992FF582E43469F583E0FEC1
:102C33007005747AF0800CEE24F975F03B84E5F0AE
:102C43002441F074992FF582E43469F583E06460DC
:102C5300600302351C745AF002351C906CE2E0608C
:102C630017906C45E0FF14FE902F2FE02EF0E08FBD
:102C7300F084E5F0F002351C9003A1E014FF902FDF
:102C83002FE02FF0E0FF9003A1E0FEEF8EF08490A1
:102C93002F2FE5F0F002351C906600E024FFF09042
:102CA30065FFE034FFF0E07002A3E070089065FF79
:102CB300F0A3743CF09065FFE0FFA3E0906611CFB2
:102CC300F0A3EFF07F047E00906611E0FD12E0B008
:102CD3007F057E00906612E0FD12E0B012E0C202B2
:102CE300351C7F037D01E4FBF54D123E1102351CBB
:102CF3009065FFE0FEA3E0FF906CDDE0FCA3E0FD48
:102D0300C39FEC9E40189065FFE0FEA3E0FFC3ED78
:102D13009F906CDEF0EC9E906CDDF002351C7F0022
:102D230022901A43E012EE772F06022F3D032F461F
:102D3300042F4F0531C8062EAD072F5808308D09D3
:102D43002F610A2F6A0B2F730C2F730D2F730E2F06
:102D5300730F2F73102F73112F8A122F8A132F8A39
:102D6300142F8A152F8A162F8A172FA9182FB619F1
:102D73002FB61A2FB61B2FB61C2FB61D2FB61E2F1C
:102D8300DB1F2FE4202FED21308D22308D2330F2F5
:102D93002430FB2631042731B62833962D33AD2E4C
:102DA30033DE2F339F3233D033348F3433673531AF
:102DB3001A39310D3A31333C31333D31333E3133FE
:102DC3003F31334031334131D15531DA5631E35755
:102DD30031EC5A31FA5B32035C320C6032C261333C
:102DE300386231BF7031C87131BF722E55782E559C
:062DF300792E557A2E55E1
:102DF9007B2E557C2E557D34297E34397F344D8088
:102E0900346181346182300A8C300A8D300A8E3007
:102E19000A8F300A90300A913036923045A03045F9
:102E2900A13045A23045A33045A43045A53045A67B
:102E39003045A73045A8307EA9335FB43383B73412
:102E490098B834A4B934B2BB0000351C9066ABE025
:102E590090CB8A93640560179066ABE090CB8A9318
:102E69006406600B9066ABE090CB8A93B4070D7F44
:102E790001E4FDFBF54D123E1102351C901DFBE0EE
:102E8900600302351C7F05FDFBF54D123E117F01E4
:102E9900124582E490681DF07F077D017B01128E47
:102EA900DA02351C901A43E0906694F0906C4BE07E
:102EB900B408167430FF7E017B047A007949756085
:102EC90000756101120A818006906C69E0F54990EC
:102ED900CB89E493FFE5498FF08485F049E549C33F
:102EE9009406500AAF49E4FD12841D02351C901A5C
:102EF9006AE549F0901A437418F002351C9068216C
:102F0900E07006901A44E0601B7FFFE4FD12849A8A
:102F1900901A437478F07F01124582907BE874011E
:102F2900F002351C7F04E4FDFB1296BBE4907BE8BC
:102F3900F002351C901A437407F002351C901A43AD
:102F49007422F002351C901A437426F002351C9045
:102F59001A43740CF002351C901A437412F00235AE
:102F69001C901A437419F002351C901A43E09066BC
:102F790094F0901A43E024F4FFE4FD12841D023515
:102F89001C901A43E0906694F0901A43E075F0069D
:102F9900A4249B901A6AF0901A437418F002351C05
:102FA900901A6AE0FFE4FD12841D02351C901A4351
:102FB900E0906694F0901A43E075F006A4247190AD
:102FC9001A6AF0F0E4FFFD1280B4901A43EFF002A0
:102FD900351C901A43748CF002351C901A4374A066
:102FE900F002351C901A6AE075F00CA424D8F58219
:102FF900E5F03415F583E4F0901A43740BF00235CB
:103009001C901A43E0B48E11906C5AE0700BA3E047
:103019007007A3E0700302351C7F04E4FD7B8C7507
:103029004D92123E11E49069C5F002351C7F027D74
:10303900011280B4901A43EFF002351C901A43E054
:1030490064A5701D906C54E07017A3E07013A3E0A1
:10305900700FA3E0700BA3E07007A3E070030235C3
:103069001C7F04E4FD7BA0754DA9123E11E4906913
:10307900C5F002351C7F017D011280B4901A43EF1F
:10308900F002351C906CE2E060147480FF7E017BD5
:05309900027A6C79458C
:10309E00756000756101120A81906CE2E0FF6006B6
:1030AE00906C45E06009EF70119003A1E0700B7F0A
:1030BE0001E4FDFB1296BB02351C901A43E0B422CC
:1030CE0005747FF08016901A43E0B423057480F0E7
:1030DE00800A901A43E0B40903747EF0E4902F2F17
:1030EE00F002351C901A437434F002351C901A43CA
:1030FE00742DF002351C901A437439F002351C9071
:10310E0069C27402F0901A43F002351C12A144EF0A
:10311E00B40109901A43743CF002351C901A4374A2
:10312E0039F002351C901A43E025E024DFF582E4E5
:10313E00347BF583E0FFA3E09065E3CFF0A3EFF0DF
:10314E00901A43E0244FF582E4347CF583E0701E40
:10315E00907CB37478F0907CB27401F0907CB4746F
:10316E0039F0907C7F741FF0A37486F0801C907CE5
:10317E00B37404F0907CB27402F0907CB47441F09D
:10318E00907C7F7419F0A3749AF012D372E4FF90BE
:10319E0065E3E0FCA3E0FD12DE68E49069C2F09006
:1031AE001A437402F002351C901A437450F0023523
:1031BE001C901A437402F002351C901A437455F099
:1031CE0002351C901A43745FF002351C901A43743A
:1031DE0022F002351C901A43745AF002351CE4900A
:1031EE001A69F0901A437461F002351C901A4374F8
:1031FE0062F002351C901A437460F002351C7E009A
:10320E007F0B7D007B027A69799912EE9D7B057AA0
:10321E00A179BF129D4E7F417D327BAF75664612FE
:10322E0009457F557D6A7B057AA179D61204C512B0
:10323E00033FE4F546E546C394045066E4F547E5DE
:10324E0047C394805058129356908002E0F52A544A
:10325E00087002FF22E54775F080A4FDE546C433F1
:10326E003354C0FEE42DFFEE35F0FE7B057AA179D6
:10327E00F4754F80120B17E547543F701D1293568D
:10328E00AF480548EF75F00CA4244BFF7D377B0546
:10329E007AA179F51205A812033F054780A10546CC
:1032AE008093E4906C45F0901A69F0901A43746123
:1032BE00F002351C901A69E0FFC3940A50437499CA
:1032CE002FF582E43469F583E0FF647B6003EF70D1
:1032DE0030901A69E0FFFDC3740A9DFDE49400FC72
:1032EE00C004C0057E0074992FF9E43469FA7B029C
:1032FE00AD06D007D00612EE9D901A69740AF080C2
:10330E0006901A69E004F0901A69E0640A600302FC
:10331E00351CFF7E017B027A697999755C0B120B65
:10332E00A3901A43745AF002351CE4906C45F07465
:10333E0080FF7E017B027A6C7945755C01120BA3CE
:10334E007F07E4FDFB1296BB901A43745BF00235C7
:10335E001C7F011249EF02351C906821E06004E4E5
:10336E00F080069068217401F0901A43742FF012C9
:10337E00445502351C901A437428F09065F412EDF2
:10338E00E40000000002351C901A437432F002353E
:01339E001C12
:10339F007F01124929901A43742DF002351C9003B6
:1033AF00A1E0D394004009901A437433F002351C06
:1033BF007F06E4FDFB1296BB901A43742EF0023584
:1033CF001C7F01124970901A43742EF002351C7F36
:1033DF0002E4FDFBF54D123E119069B9E0D3940064
:1033EF004029E025E024A5F582E434CBF583E4936E
:1033FF00FC740193FD7E007F6412EB9E90669BEF41
:10340F00F0E0FFC31390669AF08009E490669BF09A
:10341F0090669AF012033F02351C9066947409F07F
:10342F007F067D0212841D02351C901A437481F0B1
:10343F00E4906CDDF0A3F0906CDBF002351C901A79
:10344F00437482F0E4906CDDF0A3F0906CDBF0023B
:10345F00351C906CDBE064017012901A43E0B4826B
:10346F00057481F08006901A437482F0906CDBE053
:10347F0060047F0080027F01906CDBEFF002351C4F
:10348F00901A437424F002351C901A437451F012B1
:10349F0053E502351C901A437405F0E4FF129CA00B
:1034AF0002351C901A437426F0124455805F901A0F
:1034BF0043E024FB605124DD604524F9602924DFBB
:1034CF00602D146032242B7044906821E0700690B8
:1034DF001A44E06008901A4374BBF080307F04E414
:1034EF00FDFB1296BB8026901A437435F0801E9018
:1034FF001A4374B4F08016901A4374B5F0800E908E
:10350F001A4374B7F08006901A4374B6F07F012205
:10351F00901A43E012EE77364D02364D03364D04C6
:10352F00364D05364D063662073662083662093665
:10353F00620A36620B36780C36780D36780E36788E
:10354F000F367810367811368E12368E13368E145B
:10355F00368E15368E16368E1736B31836D3193675
:10356F00D31A36D31B36D31C36D31D36D31E36F89B
:10357F001F36F82036F82137492237492337492497
:10358F00376D26376D27376D2837832D37832E37C5
:10359F00832F38D23238E033387C3438EE353799D0
:1035AF003937993A37AF3C37AF3D37AF3E37AF3F3B
:1035BF0037AF4037AF4137C55037D9513819553824
:1035CF00195638195738405A38405B38405C382FF5
:1035DF005F39096038566139166237ED7037ED7112
:1035EF0038037238677E38747F387480388D81382D
:1035FF00AB82371D8C371D8D371D8E371D8F371DB5
:10360F0090371D91371D923733A03733A13733A22F
:10361F003733A33733A43733A53733A63733A73719
:10362F0033A83733A93930B4394AB53964B6393D7F
:10363F00B73957B83971B93923BB0000397CE4FF6A
:10364F007B057AA179F7901A43E014F551126DFAC0
:10365F0002397C7F017B057AA27908901A43E02416
:10366F00FAF551126DFA02397C7F027B057AA27945
:10367F0017901A43E024F5F551126DFA02397C7F49
:10368F0003906C4BE0B408087B057AA2792F800673
:10369F007B057AA27949901A43E024EFF551126D18
:1036AF00FA02397C7F04906C4BE0B408087B057AF2
:1036BF00A2792F80067B057AA279497551FF126D89
:1036CF00FA02397C7F05906C4BE0B408087B057AD1
:1036DF00A2796080067B057AA2797C901A43E02458
:0636EF00E8F551126DFA2E
:1036F50002397C7F0A906C4BE0B408087B057AA2FE
:10370500799580067B057AA279AE901A43E024E28A
:10371500F551126DFA02397C7F107B057AA279C4C6
:10372500901A43E02475F551126DFA02397C7F1128
:103735007B057AA279E1901A43E02461F551126D77
:10374500FA02397C7F3C906CE2E060087B057AA345
:10375500790280067B057AA37913901A43E024DF6A
:10376500F551126DFA02397C7F067B057AA3791D26
:10377500901A43E024DBF551126DFA02397C7F0B78
:103785007B057AA3792A901A43E024D4F551126D6A
:10379500FA02397C7F0C7B057AA3793C901A43E0C9
:1037A50024C8F551126DFA02397C7F0D7B057AA389
:1037B5007949901A43E024C5F551126DFA02397C16
:1037C5007F147B057AA37958E4F551126DFA120935
:1037D5009D02397C7F157B057AA37965E4F5511245
:1037E5006DFA12099D02397C7F287B057AA37974CD
:1037F500901A43E02491F551126DFA02397C7F2924
:103805007B057AA37980901A43E0248FF551126DD8
:10381500FA02397C7F2A7B057AA3798C901A43E0DA
:1038250024ACF551126DFA02397C7F2D7B057AA304
:103835007996E4F551126DFA02397C7F2B7B057A76
:10384500A379A7901A43E024A7F551126DFA02391E
:103855007C7F2C7B057AA379BDE4F551126DFA02C4
:10386500397CE4906C47F07F04127A8302397C7FBF
:1038750002127A8302397C7F3D7B057AA379D6E4EF
:10388500F551126DFA02397C7F08E4FD7B01125B6C
:1038950070906820E0700302397C7F04E4FD7B01B1
:1038A500128EDA02397C906CDDE0FEA3E0FF7DFF2D
:1038B5001219B47F18127A83906820E070030239D8
:1038C5007C7F04E4FD7B01128EDA02397C7B057A6C
:1038D500A379EA7D0112789602397C7B057AA37972
:1038E500FC7D0112789602397C906821E060087BA6
:1038F500057AA4791380067B057AA4792D7D0112BA
:10390500789680737B057AA479437D011278968039
:0C391500667B057AA479567D0112789635
:1039210080597B057AA479707D01127896804C7B51
:10393100057AA479847D01127896803F7B057AA46B
:1039410079997D0112789680327B057AA479B2E467
:10395100FD12789680257B057AA479D17D011278B4
:103961009680187B057AA479E9E4FD127896800B9C
:0F3971007B057AA579067D0112789612033F2215
:10398000D2C1C2AFC2A875F60375B71075B830754D
:10399000F702E4F5F843A707129356908003748961
:1039A000F0908000E528F0A3E529F0A3E52AF05384
:1039B00029DF908001E529F07F0A7E0012935D43A4
:1039C0002920908001E529F0120146E4FF12023F10
:1039D00012033F75F63FE4F5F275F320D2E9C2CD4C
:1039E000C2CCC2C9C2C8C2CBF5C975CB70F5CA7505
:1039F000CD70F5CCD2CAD2ADC2B3C2C2901A42F0D9
:103A000012CE2612004612D372432980908001E51F
:103A100029F0D288123B80E4901A44F012930FEF01
:103A200060067E007F0080047E007F0012935DD2DE
:103A3000AFD2A89069C2E070179065E3E07002A36E
:103A4000E0600DE4FF9065E3E0FCA3E0FD12DE68BA
:103A50001295DC901A43E0906694F07F04124009BE
:103A6000906991E06401703D906694E0901A43F093
:103A7000E02487600824FB50112406701A901A4332
:103A80007402F0901A6B7480F022901A437403F061
:103A9000901A6B7480F022901A437402F0E4901A2A
:063AA0006BF012351F223D
:103AA6007E007F667D007B027A1D798E12EE9D1266
:103AB6004A6EE4907BE8F0901A68F0906C75F0A37B
:103AC600F09065EBF09065EAF09069B0F0902D8B80
:103AD600F090667CF0906C6CF09003A0F03092044D
:103AE6007F0180027F00906C74EFF0906C65F0307F
:103AF60094047F0180027F00906CDAEFF0906C688E
:103B0600F0C208D20BC20EE4906992F09065E9F01B
:103B16009069C0F09065ED12EDE400000000906938
:103B26008C12EDE400000000E4902D81F09066A078
:103B3600F0902F32F0902F3104F0E4901DFAF090BF
:103B46007BE9F0901DF5F0902D7EF0906CDFF0A3F0
:103B5600F0902F2DF0A3F09069BEF0A3F09066923E
:103B6600F0A3F0906822F0A3F090039CF0A3F090ED
:0A3B760069BA12EDE400000000221D
:103B8000E49066B0F0906C72F090681E04F07E00D5
:103B90007F407D007B027A0179C812EE9DE490653A
:103BA000E8F0906C4BF090699104F0E49017E3F02A
:103BB000A3F09069C5F09066ACF0902D8004F0E41D
:103BC0009065ECF0901DF4F0902D8AF0901DFBF0C4
:103BD000906C47F090039EF0C20D9013A6F0906891
:103BE00020F0901A44F0902F2FF0906CDDF0A3F0AD
:103BF0009069B2741EF0E4906993F0901A6B74FFB0
:103C0000F0E4906819F0A3F0123AA67E107F007DD0
:103C1000007B027A0379A212EE9D90669512EDE484
:103C2000000000007E007F0C7D007B027A66790335
:103C300012EE9DE49002D1F0906C6D12EDE4000064
:103C400000009069A412EDE4000000009003A1E0E0
:103C5000D39400405DE0FF7E007C007D6312EB3575
:103C600074BE2FF9741D3EFA7B02C00378C67C69CE
:103C7000AD03D0037E007F0612EAA59069C9E00477
:103C8000F070069069C8E004F0D39069C9E094FF31
:103C90009069C8E0943F4029E4F0A3F09069C7E040
:103CA00004F0E0D3941F4019E4F09069C6E004F0FA
:103CB000800F7E007F067D007B027A6979C612EE56
:103CC0009D9069C6E0D3940340047F0180027F0089
:103CD000906615EFF0C39069CBE094789069CAE0E4
:103CE000940540047F0180027F00906C73EFF09098
:103CF000CBADE493FF9069B9E0C39F4003EF14F0AC
:103D00009069B9E0D394004029E025E024A5F5822C
:103D1000E434CBF583E493FC740193FD7E007F646F
:103D200012EB9E90669BEFF0E0FFC31390669AF053
:103D30008009E490669BF090669AF090CB91E493B2
:103D4000FF9066ABE0C39F4002E4F090CB98E49311
:103D5000FF906C71E0C39F40037402F090CB9DE430
:103D600093FF901A6DE0C39F4002E4F090CBA4E46F
:103D700093FF9065FEE0C39F4002E4F09069C2E0CB
:103D8000D394024002E4F0901A457402F0A3741D2B
:103D9000F0A374B6F0A37402F0A3741DF0A3749A98
:103DA000F0A37402F0A3741DF0A374C2F0A3740214
:103DB000F0A3741DF0A3748EF0A37402F0A3741D1D
:103DC000F0A374C6F0A37402F0A3741DF0A374965C
:103DD000F0A37402F0A3741DF0A374BAF0A37402EC
:103DE000F0A3741DF0A3749EF0A37402F0A3741DDD
:103DF000F0A374BEF0A37402F0A3741DF0A3749238
:103E0000F0A37402F0A3741DF0A374FAF0129DE104
:013E1000228F
:103E11008D4B8B4CEF147003023F1D147003023F56
:103E210060147003023FA3147003023FD7147003A0
:103E3100023EA124056003024005901DFBE0600CD9
:103E410090CB92E49314900029F0800A90CB91E4F6
:103E51009314900029F0E54B14601C04702F90001E
:103E610029E0FF9066ABE0C39F5005E004F0801DA0
:103E7100E49066ABF080169066ABE0D39400400509
:103E8100E014F08008900029E09066ABF09065E9BD
:103E91007401F0E4906992F07F01124582024005BD
:103EA100E54B14601E04703390CB98E49314FF909B
:103EB1006C71E0C39F5005E004F0801FE4906C71C9
:103EC100F08018906C71E0D394004005E014F0800C
:103ED1000A90CB98E49314906C71F0906C47E06079
:103EE10003024005901A43E0647B600EE0647D604C
:103EF10009E0647A6004E0B47C129013A3E0C394F7
:103F01000640099069AEE06003024005906C71E0E3
:103F1100608EE0640160030240058084E54B14601B
:103F21001E04703390CB9DE49314FF901A6DE0C38F
:103F31009F5005E004F0801FE4901A6DF080189006
:103F41001A6DE0D394004005E014F0800A90CB9DF7
:103F5100E49314901A6DF07F01124582024005E549
:103F61004B14602304600302400590CBADE493142D
:103F7100FF9069B9E0C39F5006E004F0024005E4F8
:103F81009069B9F00240059069B9E0D39400400608
:103F9100E014F002400590CBADE493149069B9F0C0
:103FA1008062E54B14600B0470159065FEE004F02F
:103FB100800D90CBA4E49314FF9065FEE02FF09068
:103FC10065FEE0FF90CBA4E493FEEF8EF084906554
:103FD100FEE5F0F0802EE54B146014047020901A79
:103FE10043E004F0E0D3954D4014E54CF0800F9090
:103FF1001A43E014F0E0C3954C5003E54DF090698D
:08400100C57401F01293562270
:104009008F45E490002CF090002EF0E54520E30365
:104019000240E99066B0E0600890002C7417F080C7
:1040290047D3906C76E094C0906C75E0945D40083D
:1040390090002C740EF0803090CB6DE493FE7401E7
:1040490093FFC39066A8E09F9066A7E09E501490E6
:104059006993E004F0E0C39432400D90002C740D94
:10406900F08005E4906993F090002CE060727F0184
:10407900124AE790002CE0FFE4FDFB1296BBE4FF37
:1040890012023F12033F9065F412EDBC90661112C3
:10409900EDD87F087E00906611E0FD12E0B07F093F
:1040A9007E00906612E0FD12E0B07F0A7E00906605
:1040B90013E0FD12E0B07F0B7E00906614E0FD1264
:1040C900E0B012E0C27FD07E0712935DC2C17F6467
:1040D9007E0012935DD2C17F647E0012935D80ECF5
:1040E900E54530E457906991E064016007E4901A6E
:1040F9006BF08048901A6BE0FF6041E4906C75F0BA
:10410900A3F090002DEFF0E4901A6BF09065E8743D
:1041190002F053287F908000E528F0122194EF6483
:10412900017019901A43E0FF90002EE06F600D9026
:104139001A43E090002EF012351F80E7E54530E084
:1041490058901A43E0B4BF037F01229065ECE06008
:10415900489065F412EDBC12EE257F017E007D00CA
:104169007C0012EC029065F412EDD878957C697D9B
:10417900027B027A66799C7E007F0312EAA57F049E
:10418900E4FD7B01128EDA906820E06007E4906C10
:1041990075F0A3F0E49065ECF0E54520E10620E236
:1041A900030242DF908002E0F52A540890002BF0C8
:1041B9007019906991E0701304F0E4906C4BF090E1
:1041C9001A437402F012351F0242DF90002BE0FF00
:1041D900906C4BE0FE6F70030242DFEE6003024217
:1041E900C37F01124AE7E4FF7E017B027A6979996C
:1041F900F56075610B120A81EF7015906991F09065
:104209001A437402F07F16E4FDFB1296BB7F00226D
:10421900E49069A3F090002AF090002AE0FFC3948B
:104229000B502174992FF582E43469F583E0FFC3BB
:1042390094414006EFC3947B4002E4F090002AE0E9
:1042490004F080D57480FF7E017B027A6C79457514
:104259006000756101120A81906C45E0FFD39400FA
:104269004039EF1475F040A42400FFE5F03414FE42
:104279007B027A6C7977756000756127120A81D3A0
:10428900906C7AE094F5906C79E094FF40047F019A
:1042990080027F009013A2EFF08005E49013A2F052
:1042A900906999E0700C901A69F0901A437461F062
:1042B900800E901A437470F08006901A437472F05D
:1042C90090002BE0906C4BF09069917401F0E545FA
:1042D90030E10312351FE54530E608300C05121EA2
:1042E90049C20CE54520E503024378901DF4E060DE
:1042F90007E4FF124AE78027902D8AE060217F05B5
:10430900E4FDFB1296BB7F01124AE7EF700E901A8B
:10431900437402F0901A6B7480F0800312351F9079
:1043290065EBE06011E4F090667CE060047F018059
:09433900027F00125A149066ACD8
:10434200E064017031F0906820E0600F9013A3E008
:1043520004F0E0FFE4FD12849A801B7F01124AE719
:10436200906C47E0600690039E7401F09013A3E006
:09437200FF7D0112849A7F0122F3
:10437B00902D8BE0600B7F64E4FDFB1296057F01B3
:04438B00227F00226B
:10438F00E490002FF0906615E0600302443F901711
:10439F00E0E0FEA3E07802CEA2E713CE13D8F8FF39
:1043AF001294E69017E0E0FEA3E07806C333CE3315
:1043BF00CED8F954C0FF90002FE02FF0902D83E05E
:1043CF00600790002FE04420F0906990E060079024
:1043DF00002FE04410F0901DFAE0900030F0300B09
:1043EF0047902D7EE0FF700F90002FE0240FF0908C
:1043FF002D7E7401F08031EFB40119900030E0FF91
:10440F00C4540F540FFF90002FE02FF0902D7E74A7
:10441F0002F08014900030E0540FFF90002FE02F37
:10442F00F0E4902D7EF0C20B90002FE0FF1294E687
:10443F00906615E0600F901DB612EDBC12E67790F6
:06444F006C9E12EDD82264
:10445500E4900031F090003512EDE400000000908A
:104465002D8BE060167F23E4FDFB1296057F0FE49C
:10447500FDFB1296BB7F0112458222901A43E0FF95
:10448500900033E4F0A3EFF0E4901A43F07B057A53
:10449500A5791C129D4E7F417D327BAF7566461214
:1044A500094512033FC2ADE4900032F0900032E0BE
:1044B500C394C8505812935690003512EDBC12EEB5
:1044C500257F01129398E4FCFD12EC029000351251
:1044D500EDD87F057E0012935D900032E075F019EE
:1044E50084E5F07020129356900031E0FF04F0EF60
:1044F50075F00CA4244BFF7D377B057AA179F51265
:1045050005A812033F900032E004F0809F9000352B
:1045150012EDBC12EE257FC87E007D007C0012F6F0
:104525007212EE449013ADEEF0A3EFF0906821E027
:1045350060099013ADE4F0A37464F01220FD7F01CF
:104545007D0212905F900034E0901A43F0E4FF1270
:10455500023F901A43E064786018E064796013E0E4
:10456500647A600EE0647C6009E0647B6004E0B41A
:0D4575007D057F0112458212351FD2AD2257
:104582008F4EE4FF12023F90681D7401F09066ABFB
:10459200E090CB8A9324FA600E1470149017E3E42F
:1045A200F0A3742DF080099017E3E4F0A37442F0B5
:1045B2009066ABE090CB8A9324FE604E14700302A7
:1045C200464314607C24FC400302468724086003AF
:1045D2000247327FDB7D3B7B057AA579301204C529
:1045E2007F697D4F7B057AA579351204C57F697D88
:1045F200597B057AA579301204C57FDB7D587B058E
:104602007AA5793A1205A80247327FDB7D3B7B050A
:104612007AA5793C1204C57F697D4F7B057AA5791D
:104622003E1204C57F697D597B057AA5794412043F
:10463200C57FDB7D587B057AA5793A1205A802472A
:10464200329066ABE090CB8A93B4030F7FDB7D3C64
:104652007B057AA579471205A8800D7FDB7D3B7B20
:10466200057AA579491204C57F697D597B057AA52A
:10467200794E1204C57FDB7D587B057AA5793A1203
:1046820005A8024732901A6DE090CB9993146036D8
:1046920014605C146059240360030247257FDB7DAC
:1046A2003B7B057AA579301204C57FDB7D4F7B0504
:1046B2007AA579351204C57FDB7D597B057AA57908
:1046C200301204C5805D7FDB7D3B7B057AA5793C9A
:1046D2001204C57FDB7D4F7B057AA5793E1204C5A6
:1046E2007FDB7D597B057AA579441204C58034901D
:1046F2001A6DE090CB9993B4020F7FDB7D3C7B0572
:104702007AA579471205A8800D7FDB7D3B7B057A70
:10471200A579491204C57FDB7D597B057AA5794EBF
:104722001204C57FDB7D767B057AA5793A1205A84E
:104732009066ABE090CB8A93D394044003024898EE
:10474200906C71E090CB939324FE70030247D714D0
:10475200700302480E1470030248441470030248A6
:1047620044240460030248989000397404F09000D5
:1047720039E0C394CB5013E0FF7D722408FB120092
:104782000C900039E02410F080E4906C6674BEF066
:104792007FD07D647B7F12002E901DFBE0600F7F37
:1047A200D67D677B057AA579501204C580097FD032
:1047B2007D727BEF12000C906C66E0FCE412E64323
:1047C20012EE25906C4C12EDBC12E53B907BE3128D
:1047D200EDD80248987F697D6D7B057AA5795612DE
:1047E20004C57F697D777B057AA579301204C57F80
:1047F200DB7D6D7B057AA5795B1204C57FDB7D7756
:104802007B057AA579491204C50248987F697D6DB6
:104812007B057AA579561204C57F697D777B057A77
:10482200A579301204C57FDB7D6D7B057AA57956AB
:104832001204C57FDB7D777B057AA579601204C5FA
:1048420080547F697D6D7B057AA579351204C57F19
:10485200697D777B057AA579471205A8906C71E08E
:1048620090CB9393640570187FDB7D747BE5120017
:104872000C7FDB7D767B057AA5793A1205A8801636
:104882007FDB7D717BE712000C7FDB7D737B057A1A
:10489200A579641205A87FDB7D0A7B057AA5796478
:1048A2001205A8E4FF7D1A7BEF12000CE4FF0D1243
:1048B200000C9066ABE090CB8A931460540424FB06
:1048C200500624FD502C80497F7FE4FD7B1A1200A4
:1048D2002E7F7F7D497B6412002EE4FF7D477BEFB4
:1048E20012000CE4FF0D12000CE4FF7D6412000CB8
:1048F200801F7F7FE4FD7B7F12002E7F7F7D477BC1
:10490200EF12000C7F7F0D12000C7F7F7D6412007E
:104912000CE490681DF07F077D017B01128EDAE5C1
:074922004E600312033F2267
:104929008F4AC2AFE49003A1F0FE7F06FD7B027AB5
:104939006979C612EE9DE4906615F0906C73F07E6D
:104949000F7F78FD7B027A1E790212EE9DD2AFE5C8
:104959004A60087F06E4FDFB1296BB124DCD7F31FC
:07496900E4FDFB129605229C
:104970008F4A9003A1E0D394004057E014F0E0FF89
:104980007E007C007D6312EB35741B2FF9741E3E94
:10499000FA7B02C00378C67C69AD03D0037E007F3A
:1049A0000612EAA59069C6E0D3940340047F018013
:1049B000027F00906615EFF0C39069CBE094789089
:1049C00069CAE0940540047F0180027F00906C7307
:1049D000EFF0E54AB4010C7F129003A1E0FDE4FB87
:0F49E0001296BB124DCD7F3FE4FDFB12960522D0
:1049EF008F4AE4906821F090CBAD93149069B9F0A1
:1049FF00E025E024A5F582E434CBF583E493FC7441
:104A0F000193FD7E007F6412EB9E90669BEFF0E0BA
:104A1F00FFC31390669AF0E49066ABF0906C7174DC
:104A2F0002F0E49069AEF0901A6DF0906C6904F0AA
:104A3F009065F3F0FE7FB07D007B027A16792C1221
:104A4F00EE9D7F01E4FD125486E54A60117F15E467
:0F4A5F00FDFB1296BB901A437450F012351F22C4
:104A6E00C2AF1293567E037F207D007B027A1A79A5
:104A7E006E12EE9DE4901A6CF09013A5F09013ACAC
:104A8E00F0907BE7F090698C12EDE400000000904E
:104A9E0065ED12EDE400000000E49066A0F0902DAC
:104AAE0081F090039CF0A3F0906692F0A3F0901D1D
:104ABE00F6F07E017F5CFD7B027A1379B312EE9DD8
:104ACE007E007F067D007B027A66798C12EE9DE475
:094ADE009065E6F0A3F0D2AF22CE
:104AE7009002D27401F0EF147003024B7F0460034D
:104AF700024DC7E4FF12E1E278807C6C7D027B0205
:104B07007A6679A17E007F0612EAA5906C4BE06475
:104B1700087056906C45E0FFD39400403BEF147546
:104B2700F040A42400FFE5F03414FE7B027A0079FC
:104B37003C756000756104120A8190003EE0FEA397
:104B4700E0FF906C77EEF0A3EFF02428906C7AF0FA
:104B5700E43E906C79F08011906C777440F0A3E498
:104B6700F0A37440F0A37428F0E4901DF4F07F39AB
:104B7700FDFB129605024DC7E4907BE8F0902D8B64
:104B8700E07003024DC2E4901DFBF0906C47F0907B
:104B97002D8AF090667CF09065ECF0902D8BF0906C
:104BA70013A6F0901DB612EDBC12E677906C7C123E
:104BB700EDD87F007E007D007C0012EE25906C9E74
:104BC70012EDBC12ED32700F901DB612EDBC12E65D
:104BD70077906C9E12EDD8D3906CE0E09401906CC6
:104BE700DFE094005003024CECD3901DE8E0940002
:104BF700901DE7E0940050069065EBE06009E490B3
:104C070065EBF0FF125A14906C9AE0FEA3E0FF9058
:104C17006C94E06E7003A3E06F7003024CDD906C40
:104C270090E0FFD39403503C9069C6E0FED3940311
:104C37004014906C967403F0A3741FF0A3743FF0B4
:104C4700A374FFF0803A906C96EEF09069C7E090FD
:104C57006C97F09069C8E0FDA3E0906C98CDF0A345
:104C6700EDF0801C906C96EFF0906C91E0906C9753
:104C7700F0906C92E0FFA3E0906C98CFF0A3EFF078
:104C87009003A1E0FF7E007C007D6312EB35740288
:104C97002FF9741E3EA801FC7D027B027A6C79779E
:104CA7007E007F6312EAA59003A1E0FF7E007C00EF
:104CB7007D6312EB35743D2FF9741E3EA801FC7D10
:104CC700027B027A1D798E7E007F2812EAA5900367
:104CD700A1E004F080557F10E4FDFB1296BBE49041
:104CE70002D2F0804678C67C697D027B027A6C79B5
:104CF700967E007F0612EAA59069C6E0D39403402A
:104D0700047F0180027F00906615EFF0C39069CBA6
:104D1700E094789069CAE0940540047F0180027F9F
:104D270000906C73EFF0E49002D2F0906C4BE0646B
:104D370008705A906C77E0FEA3E0FF2428FDE43E5C
:104D4700FCA3E0FAA3E0FB6D7002EC6A603F7B0214
:104D57007A1D798E755C28120BA3906C45E075F06F
:104D670040A42400FFE5F03414FE7B027A6C7977C7
:104D7700755C27120BA3906C45E004F07480FF7EEE
:104D8700017B027A6C7945755C01120BA39002D204
:104D9700E0602D7F3AE4FDFB1296059003A07401B5
:104DA700F0A3E014902F2FF0901A437482F0E49050
:104DB7006CDDF0A3F0906CDBF08005E49002D2F09C
:064DC7009002D2E0FF2281
:104DCD00E49000A0F09003A1E0D394005003024FB3
:104DDD0089E490009FF09003A1E0FF90009FE0C355
:104DED009F4003024F8974F4FF7E0112935D900082
:104DFD009FE0FF7E007C007D6312EB3574022FF97E
:104E0D00741E3EFA7B02C00378777C6CAD03D00331
:104E1D007E007F6312EAA51200067F007E007D00F2
:104E2D007C0012EE25906C9E12EDBC12ED326002EC
:104E3D005003024F80906C91E0FFE4FCFDFE12EEFA
:104E4D00257F007E407D007C0012EC2912EE25901E
:104E5D006C90E0FFE4FCFDFE12EE257F007E007DF0
:104E6D00087C0012EC2912EC0212EE25906C92E0F7
:104E7D00FEA3E0FFE4FCFD12EC0212EE25906C9710
:104E8D00E0FFE4FCFDFE12EE257F007E407D007C00
:104E9D000012EC2912EE25906C96E0FFE4FCFDFE6D
:104EAD0012EE257F007E007D087C0012EC2912ECAD
:104EBD000212EE25906C98E0FEA3E0FFE4FCFD12DB
:104ECD00EC0212EC159000A112EDD812935690023F
:104EDD00D474A5F09002D67418F090009FE004549D
:104EED007F9002D7F0E4A3F078D97C027D027B029B
:104EFD007A6C7980FE7F0612EAA5906CB1E0900283
:104F0D00DFF0906C86E09002E0F0906CA2E09002F1
:104F1D00E1F09000A112EDBC8F4F8E4E8D4D8C4C5B
:104F2D007F0F129FFD906C9E12EDBC8F4F8E4E8D9C
:104F3D004D8C4C7F14129FFD906C8712EDBC8F4FE2
:104F4D008E4E8D4D8C4C7F19129FFD906C8B12EDFA
:104F5D00BC8F4F8E4E8D4D8C4C7F1E129FFD7F232F
:104F6D00906C8FE0FD7C00129FCF12006F9000A01F
:104F7D00E004F090009FE004F0024DE39000A0E00B
:104F8D0070077F18FDFB1296057F967E0012935DCC
:014F9D0022F1
:104F9E008F46901A43E0906694F07F13E54604FD29
:104FAE00E4FB1296BBAF467E007C007D6312EB35B0
:104FBE0074022FF9741E3EFA7B02C00378777C6C64
:104FCE00AD03D0037E007F6312EAA51200069002A5
:104FDE00D474A4F09002D6744BF07F04906CA3E0CE
:104FEE00FD7C00129FCF7F08906CB0E0FD7C00121C
:104FFE009FCFE49000A5F09000A5E0C3940350313C
:10500E00E0FE75F005A4240AFFC007EE25E025E0BA
:10501E0024A4F582E4346CF58312EDBC8F4F8E4ED2
:10502E008D4D8C4CD007129FFD9000A5E004F080B2
:10503E00C6906C8712EDBC8F4F8E4E8D4D8C4C7F73
:10504E0019129FFD906C8B12EDBC8F4F8E4E8D4DB5
:10505E008C4C7F1E129FFD7F23906C8FE0FD7C0099
:10506E00129FCF12006F7F32AD46E4FB129605AF52
:10507E00467E007C007D6312EB3574022FF9741EA0
:10508E003EFA7B02C00378777C6CAD03D0037E00C2
:10509E007F6312EAA5906C91E0FBFFE4FCFDFE122B
:1050AE00EE257F007E407D007C0012EC2912EE255D
:1050BE00906C90E0FFE4FCFDFE12EE257F007E007A
:1050CE007D087C0012EC2912EC0212EE25906C92F7
:1050DE00E0FEA3E0FFE4FCFD12EC02901DFC12EDDD
:1050EE00D8906C97E0FFE4FCFDFE12EE257F007E6B
:1050FE00407D007C0012EC2912EE25906C96E0FFAC
:10510E00E4FCFDFE12EE257F007E007D087C001281
:10511E00EC2912EC0212EE25906C98E0FEA3E0FF53
:10512E00E4FCFD12EC02902F1C12EDD89000AC1294
:10513E00EDD8906C90E090039FF09013A4EBF0905C
:10514E006C92E0FFA3E09069CCCFF0A3EFF0902D2E
:10515E00857452F09002D474E1F09002D67433F05C
:10516E00901DFC12EDBC12EE25902F1C12EDBC1200
:10517E00EC1512EE257F52E4FCFDFE12EC8B12EEC6
:10518E004C9000ABEFF02401FFE433FE3395E0FDCD
:10519E00FC12EE25902F1C12EDBC12EC15902F1C5C
:1051AE0012EDD812521EEF60667F017E007D007CEC
:1051BE000012EE25902F1C12EDBC12EC02901DFC7D
:1051CE0012EDD89000AC12EDBC902F1C12EDD890C1
:1051DE0000ABE0902D85F0E0FF75F0078475F008C8
:1051EE00A4FEEF75F00784EE25F024849002D4F02F
:1051FE0012521EEF60197F34AD46E4FB12960590F5
:10520E006694E0901A43F0E4FF12023F12351F221B
:10521E00120006901DFC12EDBC9000B812EDD89055
:10522E002F1C12EDBC12EE259000B812EDBC12ED43
:10523E003240030253E2129356120006E49000B07D
:10524E00F09000B2F09000B57403F0A37407F090E4
:10525E002D85E0FF9000B0E0FEC39F400302538314
:10526E00C3EF9E9000B4F0C39407500FE09000B6C9
:10527E00F004FF9000B5E02FF080079000B5E02419
:10528E0008F09000B5E024D3F582E43402F583E40F
:10529E00F09000B704F0E49000B1F09000B6E0FF9B
:1052AE009000B1E0C39F400302537A90039FE0FF4A
:1052BE001392C3EFD394014003D38001C392C4531E
:1052CE0029E09013A4E04229908001E529F090692D
:1052DE00CCE044C0FEA3E0F5828E83E09000B4F0F3
:1052EE009069CDE004F070069069CCE004F0D390A4
:1052FE0069CDE094FF9069CCE0943F4018E4F0A3B0
:10530E00F09013A4E004F0E0D3941F4008E4F09072
:10531E00039FE004F09000B4E0FF547FFE9000B2D3
:10532E00E024D7F582E43402F583EEF0EF30E71F88
:10533E009000B5E024D3F582E43402F583C083C037
:10534E0082E0FF9000B7E0FEEF4ED082D083F09067
:10535E0000B7E0FF25E0F09000B0E004F09000B25E
:10536E00E004F09000B1E004F00252A99000B2E027
:10537E0004F002525D12006FE4906C75F0A3F07FA2
:10538E0037129DB9EF7006901A6BE06029C20CE4DB
:10539E00901A6BF07F37FDFB1296057F14E4FDFB30
:1053AE001296BB906694E0901A43F0E4FF12023F0F
:1053BE0012351F7F00229000B812EDBC12EE259020
:1053CE002D85E0FFE4FCFDFE12EC029000B812ED1C
:0753DE00D802522D7F0122CD
:1053E5009065F812EDBC90669512EDD87F077B02AB
:1053F5007A66790312A0BE7F0C7B027A6679071262
:10540500A0BE7F117B027A66790B12A0BE7F187B46
:10541500027A0079BC12A0BE9000BC12EDBC12E667
:10542500779002D1EFF0E0FCE412E64312EE257F1F
:10543500407EC97D0F7CDB12E4C312EE257F447EDE
:105445007A7D007C0012E53B906C6D12EDD8906C76
:105455006D12EDBC12EE2590CB8512EDC8EC12E66F
:105465003B12E53B9069A412EDD87F017D011290B6
:105475005FE4FF7D011254867F1DE4FDFB12960556
:015485002204
:105486008D4B9000C1744BF0907BE8E09000C0F02B
:10549600E4907BE8F0EF1470030255BC046003024D
:1054A6005669E54B602A901A43E0FF9000C4E4F089
:1054B600A3EFF0E4901A43F07B057AA57966129D76
:1054C6004E7F417D327BAF75664612094512033F1A
:1054D600E49000C2F0A3F09000C2E0FCA3E0FDC39C
:1054E60094FFEC940340030255A2E412E63F12EE49
:1054F6002590660B12EDBC12E4C312EE25906607EA
:1055060012EDBC12E3B812EE259000C2E0FCA3E057
:10551600FDE412E63F12E4C312EE2590660312ED97
:10552600BC12E3B812EE2590CB8512EDC8EC12E65C
:105536003B12E4C312E67712EE259000C2E0FEA30A
:10554600E07802C333CE33CED8F924A2F582EE3406
:1055560003F58312EE4412EDD8129356E54B602BF9
:105566009000C2E0FEA3E0FF547F701FEF7807CEE5
:10557600C313CE13D8F975F00CA4244BFF7D377BEB
:10558600057AA179F51205A812033F9000C3E0043D
:10559600F070069000C2E004F00254DDE54B7003A3
:1055A6000256699000C5E0901A43F0E4FF12023FEC
:1055B60012351F0256691293569000C612EDE4DBAF
:1055C6000FC93FE49000C2F0A3F0C39000C3E0947B
:1055D600689000C2E0940140030256699000C6122A
:1055E600EDBC12F54A12EE257F427EC87D007C0096
:1055F60012E4C312E6779000C2E0FCA3E024B1F502
:1056060082EC3466F583EFF01293569000C2E0FE0A
:10561600A3E0FF24B1F582EE3466F583E0FBEF24C8
:105626005AFFE43EFE7C017D6812EB4974242DF599
:1056360082EC3468F583EBF09000C612EDBC12EEF6
:10564600257F3C7E8E7DFA7C3512E3B89000C6122B
:10565600EDD89000C3E004F070069000C2E004F0BC
:0C5666000255D09000C0E0907BE8F022DC
:105672001293567F457EBB7D807C0012EE2590689A
:105682001BE0FCA3E0FDE412E63F12E53B901DBAED
:1056920012EDD890681BE0FCA3E0FDE412E63F1295
:1056A200EE257F427EC87D007C0012E53B901DD630
:1056B20012EDD8901DE312EDBC12EE25901DD6120C
:1056C200EDBC12E3B8901DE312EDD8901DD212ED9D
:1056D200BC12EE25901DD612EDBC12E3B8901DD27D
:1056E20012EDD81293567F417EA07D007C0012EE0F
:1056F20025901DBA12EDBC12E5EA5003025A107F42
:10570200437EC87D007C0012EE25901DBA12EDBCCE
:1057120012E5EA60054003025A10901DE2E004F02F
:10572200901DB212EDBC12EE257F017E007D007C41
:105732000012EC02901DB212EDD8902D82E060FAB8
:10574200E4902D82F0901DBA12EDBC12EE25901D50
:10575200AA12EDBC12E5EA500C901DBA12EDBC90F3
:105762001DAA12EDD8901DB212EDBCE412E63B1256
:10577200EE25901DD212EDBC12EE257F427E707D89
:10578200007C0012E53B12E53B901D9E12EDD8D342
:10579200906693E09400906692E09400403C90689A
:1057A20022E0FCA3E0FDE412E63F12EE25906692B1
:1057B200E0FCA3E0FDE412E63F12E53B901DCE12B1
:1057C200EDD8901DAE12EDBC12EE25901DCE12ED5D
:1057D200BC12E3B8901DAE12EDD8902D82E060FAB3
:1057E200E4902D82F0902D8612EDBCEC12E63B1275
:1057F200EE2590681BE0FCA3E0FDE412E63F12E513
:105802003B12EE259069A412EDBC12E4C3901DBEBA
:1058120012EDD87F007E007D007C0012EE25901DE7
:10582200BE12EDBC12E5EA500A901DBE12EDE40074
:10583200000000901DE912EDBC12EE25901DBE1273
:10584200EDBC12E3B8901DE912EDD8901D9212ED55
:10585200BC12EE25901DBE12EDBC12E3B8901D9253
:1058620012EDD8129356901DBE12EDBC12EE259089
:105872001DD612EDBC12E53B901DC212EDD8901D53
:105882009212EDBC12EE25901DD212EDBC12E53B38
:09589200901D8E12EDD8901DC28C
:10589B0012EDBC12EE25901DA612EDBC12E5EA50DE
:1058AB000C901DC212EDBC901DA612EDD8902D824E
:1058BB00E060FAE4902D82F0FFFEFDFC12EE2590E5
:1058CB001DC212EDBC12E5EA60324030901DC212CF
:1058DB00EDBC12F40712EE257F3E7EBD7D2F7C1BA7
:1058EB0012E4C312F36B12EE257F407EA77D347C4E
:1058FB00D712E4C3901DC612EDD8800A901DC612B4
:10590B00EDE400000000901DD612EDBC12EE2590C8
:10591B001DC612EDBC12E4C312EE257F407E667DE0
:10592B00667C6612E53B901DCA12EDD8902D82E085
:10593B0060FAE4902D82F0901A43E0647D706590DC
:10594B006C4C12EDBC12EE25901DCA12EDBC12EE82
:10595B0025901D9A12EDBC12E3B812E5EA40459072
:10596B001DED12EDBC12EE25901D9A12EDBC12EE40
:10597B0025906C4C12EDBC12E3B412E3B8901DED04
:10598B0012EDD8906C4C12EDBC901D9A12EDD89084
:10599B001DFBE06007E4907BE8F080389066AC7408
:1059AB0001F08030901DED12EDBC12EE25901DCA5A
:1059BB0012EDBC12E3B8901DED12EDD8901D9A12AA
:1059CB00EDBC12EE25901DCA12EDBC12E3B8901D72
:1059DB009A12EDD8902D82E060FAE4902D82F0902F
:1059EB001D9A12EDBC12EE25901DD212EDBC12E5E4
:1059FB003B12EE257F407E667D667C6612E4C3908B
:095A0B001D9612EDD812935622EB
:105A14008F4A901DE2E07003025B6F786A7C667DBA
:105A2400027B027A1D79E27E007F1212EAA57E00D3
:105A34007F0A7D007B027A66797E12EE9D7F447E2A
:105A44007A7D007C0012EE2590666B12EDBC12E4A8
:105A5400C312E67790667EEEF0A3EFF090667AE0EC
:105A6400FFA3E0906685CFF0A3EFF07F3F7E007D3B
:105A7400007C0012EE2590667112EDBC12E3B812A0
:105A8400E677906680EEF0A3EFF07F417E207D0004
:105A94007C0012EE2590667512EDBC12E4C312E68A
:105AA40077906682EEF0A3EFF090666AE0906684E9
:105AB400F0906679E0906687F09013A2E0703E90D3
:105AC4006C4BE064087036906C79E0FEA3E0FFD381
:105AD40094F5EE94FF501C7B027A66797E755C0A1D
:105AE400120BA3906C7AE0240AF0906C79E03400F5
:105AF400F0800A9013A27401F0906C7BF0906C73A8
:105B0400E070599069CAE0FEA3E0FFC39478EE9474
:105B140005503F7C007D0A12EB3574332FF9742F46
:105B24003EA801FC7D027B027A66797E7E007F0AB4
:105B340012EAA59069CBE004F070069069CAE0040B
:105B4400F09069CAE0FFA3E0906C9ACFF0A3EFF065
:105B5400800A906C737401F0906C9CF07E007F124C
:0C5B64007D007B027A1D79E212EE9D228A
:105B70008F548D558B56129356E55424FB24FD50BB
:105B8000087003025DBE02610D901A6DE090CB9922
:105B900093147003025C29147003025CCC1470032C
:105BA000025CCC2403600302610D7F3F7E007D0018
:105BB0007C0012EE2590664A12EDBC12E3B812E6A4
:105BC000779000DAEEF0A3EFF0C394E8EE94034090
:105BD000277F837D207B057AA5797D12078C7B0545
:105BE0007AA579819000DAE0FCA3E0FD129EBF7FE8
:105BF000907D2D12070580187B057AA57985900088
:105C0000DAE0FCA3E0FD129EBF7F837D20120782B5
:105C10007B057AA5798190661612EDBC129EF77FFE
:105C2000907D4B12070502610D7F3F7E007D007C59
:105C30000012EE2590664612EDBC12E3B812E6772C
:105C40009000DAEEF0A3EFF0C394E8EE940340275F
:105C50007F837D207B057AA5797D12078C7B057A71
:105C6000A579819000DAE0FCA3E0FD129EBF7F9051
:105C70007D2D12070580187B057AA579859000DABD
:105C8000E0FCA3E0FD129EBF7F837D20120782907F
:105C9000661A12EDBC12EE257F447E7A7D007C00F0
:105CA00012E53B9000E312EDD8902D84E06004E40F
:105CB000F080DC7B057AA579819000E312EDBC12BF
:105CC0009EF77F907D4B12070502610D901A6DE0E3
:105CD00090CB99936402704B7F417E20FDFC12EEC5
:105CE0002590664E12EDBC12E4C312E6777C007D6F
:105CF0000A12EB497B057AA57989129EBF7FB87D90
:105D00002D12070590664E12EDBC12E677AC06AD7B
:105D1000077B057AA5798E129EBF7F837D201207AF
:105D200082800CE4FF129F3F7F877D2D1207057F45
:105D3000107E277D007C0012EE25906C6112EDBC78
:105D400012ED324051906C6112EDBC12EE257F10C5
:105D50007E277D007C0012EC8B12EE44AD07AC0672
:105D60007B057AA5798E129EBF7F817D4B12059EA1
:105D7000906C6112EDBC12EE257F107E277D007CB9
:105D80000012EC8B12EE4CAD07AC067B057AA579C0
:105D900092129EBF801E7F817D4B7B057AA5797D07
:105DA0001205A87B057AA57981906C63E0FCA3E0DD
:105DB000FD129EBF7F907D4B12070502610DE4FF2F
:105DC00012023F906820E060087B057AA5799780F1
:105DD000067B057AA5799E129D4E9000D37411F032
:105DE000E49000DAF0A3F09000F712EDE400000078
:105DF00000E49000CFF0906CE2E06019906C77E0E6
:105E0000FEA3E0FF7B027A1D798E75600075612824
:075E1000120A818013788E55
:105E17007C1D7D027B027A6C79B27E007F2812EAB4
:105E2700A59066AEE0FCA3E0FD9000DAE0FEA3E0FB
:105E3700FFC39DEE9C4003025F4E9065FEE090CB52
:105E47009E93FD1219B49065FEE090CB9E9324FEBD
:105E5700602224FE602C24FC603624F8604024F085
:105E6700604A241F70529069D412EDBC9000F3125F
:105E7700EDD880449069D812EDBC9000F312EDD8AC
:105E870080369069DC12EDBC9000F312EDD88028C3
:105E97009069E012EDBC9000F312EDD8801A90697A
:105EA700E412EDBC9000F312EDD8800C9069E81273
:105EB700EDBC9000F312EDD8906CDDE0FEA3E0FF9F
:105EC700C39000DBE09F9000DAE09E40439000CF54
:105ED700E0C39464503A7F3F7E007D007C0012EE61
:105EE700259000F312EDBC12E3B812E677AC06ADCD
:105EF700079000CFE025E0FFE433FE748C2FF58296
:105F0700EE342DF583ECF0A3EDF09000CFE004F034
:105F17009000F312EDBC12EE259000F712EDBC12C3
:105F2700E5EA500C9000F312EDBC9000F712EDD8A3
:105F37009065FFE0FEA3E0FF9000DBE02FF090000C
:105F4700DAE03EF0025E287F10127A839065FEE069
:105F570090CB9E9324FE603F24FE606724FC700371
:105F6700025FE824F8700302600624F07003026001
:105F770024241F60030260407F0C7D147B057AA5F3
:105F870079A71204C57B057AA579B19000F712EDC0
:105F9700BC129EF70260407F0C7D147B057AA579C1
:105FA700C61204C59000F712EDBC12EE257F447EA1
:105FB7007A7D007C0012E53B7B057AA579CE129E9F
:105FC700A180767F0C7D147B057AA579E61204C53E
:105FD7007B057AA579EE9000F712EDBC129EF7804B
:105FE700587F0C7D147B057AA679061204C57B05BC
:105FF7007AA6790F9000F712EDBC129EF7803A7FD0
:106007000C7D147B057AA679241204C57B057AA634
:10601700792C9000F712EDBC129EF7801C7F0C7D47
:10602700147B057AA679431204C57B057AA67946BF
:106037009000F712EDBC129EF77F0C7D211204BB76
:106047009065FEE090CB9E9324FE602524FE604081
:1060570024FC604D24F8605A24F06067241F707296
:106067007B057AA6795D9069D412EDBC129EF78004
:10607700619069D812EDBC12EE257F447E7A7D00CF
:106087007C0012E53B7B057AA6796D129EA18042C2
:106097007B057AA6797E9069DC12EDBC129EF780AB
:0760A700317B057AA6799117
:1060AE009069E012EDBC129EF780207B057AA679EE
:1060BE009F9069E412EDBC129EF7800F7B057AA6C5
:1060CE0079B19069E812EDBC129EF77F0C7D2E120D
:1060DE0004BB7B057AA679C39065FFE0FCA3E0FDC7
:1060EE00129EBF7F017B027A0179C8756782120505
:1060FE00507D141204BB7F0C7D1E7B8012000C128F
:10610E009356E55424FA7003026358147003026424
:10611E00FA1470030267F51470030268CE2404604B
:10612E0003026DF27F0112023F7F7FE4FD7B7F123F
:10613E00002E7F057D2A7B7212002EE55660677F4A
:10614E00057D707B7912000C7F3F7B7212002E7FD3
:10615E00797D7012002E901A6DE090CB999324FEEB
:10616E0060161460132402701E7F057D1F7B057A56
:10617E00A679D41204C580217F057D1F7B057AA6E2
:10618E0079E01204C58012E4901A6DF07F057D1F30
:10619E007B057AA679EF1204C57F5C7D1F7B057A9D
:1061AE00A679FD1204C59065E6E0FEA3E0FFD39448
:1061BE0000EE9400401AEF24FFFFEE34FFFE7C0049
:1061CE007D3A12EB35901DF6E02FFFEC3EFE80047B
:1061DE007E007F009000DAEEF0A3EFF0AC06FD7BC0
:1061EE00057AA77904129EBF7F057D741204BB7BCE
:1061FE00057AA779099000DBE0241DFD9000DAE016
:10620E003400FC129EBF7F027B027A0179C875674B
:10621E003F1205507D741204BB7B057AA77910904E
:10622E0000DBE0243AFD9000DAE03400FC129EBF61
:10623E007F017B027A0179C875677B1205507D74E8
:10624E001204BB901A6DE09000D5F0D39402400377
:10625E007402F09000D5E0FF7E007C007D7412EB9E
:10626E003574B32FF974133EFA9000DE7402F0A366
:10627E00EAF0A3E9F09000D5E025E0248CF582E465
:10628E003466F583E0FFA3E09000E1CFF0A3EFF0DA
:10629E00D3906CE0E09401906CDFE0940050030228
:1062AE006DF2D39000E2E094009000E1E094005093
:1062BE00030263529000D37406F0D39065E7E09426
:1062CE00009065E6E094004007901DF6E0FF800226
:1062DE007F009000D0EFF0E49000CEF09000CEE082
:1062EE00FFC3943A505E9000D0E0FEEF2E75F03A68
:1062FE0084E5F025E0FFE433FE9000DEE0FBA3E052
:10630E00FAA3E0F98F828E8312EBC8FFAEF09000F5
:10631E00E1E0FCA3E0FD12EB49C374709FFF900017
:10632E00D2F0FDA3E0FF04F07B6F12002E9000D39D
:10633E00E0FF04F09000D2E0FD12002E9000CEE0BF
:10634E0004F08098129356026DF27F0112023F7F85
:10635E007FE4FD7B7F12002E7F057D2A7B7212006B
:10636E002EE55660317F057D707B7712000C7F3EE7
:10637E007B7212002E7F777D7012002E7F057D744A
:10638E007B057AA779151204C57F627D1F7B057A7E
:10639E00A779181204C59013A5E0C3946C50047F1E
:1063AE000180027F029000D4EFF06401701C7F33F5
:1063BE007D747B057AA7791F1204C57F6B7D747B74
:1063CE00057AA779261204C5801A7F347D747B0561
:0F63DE007AA7792B1204C57F697D747B057AA796
:1063ED0079321204C5129356906992E07003026DD2
:1063FD00F99013A5E0D394005003026DF2902D8116
:10640D00E0D394005003026DF29000D37406F0E4D3
:10641D009000CEF09013A5E0FF9000CEE0FEC39F5C
:10642D0040030264B7EE25E0FFE433FE902F31E028
:10643D00FD75F090A4246EF582E5F0341AF583ED28
:10644D002583F583E5822FF582EE3583F583E0FE16
:10645D00A3E0FF902D81E0FD7C0012EB49C3746E2B
:10646D009FFF9000D2F0FDA3E0FF1204799000D3BE
:10647D00E004FF9000D2E0FD1204799000D3E0FF1C
:10648D009000D2E004FD1204799000D3E004FF9057
:10649D0000D2E004FD1204799000D3E004F0A3E0F3
:1064AD00FF9000CEE02FF00264211293569065ED1F
:1064BD0012EDBCEC12E63B12EE257F447E807D0092
:1064CD007C0012E53B12EE257F3F7E007D007C00B7
:1064DD0012E3B812E677AC06AD077B057AA77937DC
:1064ED00129EBF7F057D1F1204BB026DF27F02124B
:1064FD00023FE4FF7D1D7B057AA7794B1204C5E4AD
:10650D00FF7D4A7B057AA7796C1204C57F2A7D77BA
:10651D007B057AA779931204C57F7FE4FD7B7F12FB
:10652D00002E7F117D4D7B6B12000C7F3E7D207BFD
:10653D007A12002E906992E07003026DF99013A506
:10654D00E0C3941E50030267EFE0C394C7400302FB
:10655D0067EF7F437E347D007C0012EE25907BE754
:10656D00E0FCE412E64312E53B9000EF12EDD8900B
:10657D002D84E06010E4F09000E712EDBC9000E394
:10658D0012EDD880CDE49000CEF09013A5E014FF6D
:10659D009000CEE0C39F400302676A9000CEE0FFFB
:1065AD0070169000E312EDE4000000009000E71279
:1065BD00EDE4000000008075907BE7E06F704A7F8E
:1065CD00437E34FDFC12EE25907BE7E0FF9013A592
:1065DD00E0C39FFCE412E64312E53B9000EF12EDA1
:1065ED00D89000E312EDBC9000E712EDD87F437E0A
:1065FD00347D007C0012EE259000EF12EDBC12E30D
:10660D00B89000E312EDD880249000E312EDBC9019
:10661D0000E712EDD89000E312EDBC12EE259000CC
:10662D00EF12EDBC12E3B89000E312EDD8902D847B
:10663D00E06011E4F09000E712EDBC9000E312ED84
:10664D00D80265A89000CEE025E0FFE433FE902F40
:10665D0031E0FD75F090A42470F582E5F0341AF563
:10666D0083ED2583F583E5822FF582EE3583F58362
:10667D00E0FCA3E0FDE412E63F12EE25902D81E053
:10668D00FCE412E64312E53B12E6779000D6EEF0FD
:10669D00A3EFF0902D84E06004E4F080A79000E378
:1066AD0012EDBC12E6779000DAEEF0A3EFF0D39482
:1066BD0067EE94014007E49000DAF0A3F09000DA61
:1066CD00E0FAA3E0FB24B1F582EA3466F583E0FF3E
:0F66DD003395E0FE9000D6E0FCA3E0FD12EB3514
:1066EC007C007D6412EB9EEF243D9000D0F074246E
:1066FC002BF582EA3468F583E0FF3395E0FE9000D9
:10670C00D6E0FCA3E0FD12EB357C007D6412EB9E21
:10671C00C3744D9F9000D1F0902D84E06005E4F09F
:10672C000266AA9000D0E0FFA3E0FD12047990006D
:10673C00D0E004FFA3E01204799000D0E0FFA3E0C6
:10674C0004FD1204799000D0E004FFA3E004FD12D4
:10675C0004791293569000CEE004F00265977F42C4
:10676C007EC87D007C0012EE25901DCE12EDBC1271
:10677C00E4C312EE257F3F7E007D007C0012E3B85F
:10678C0012E6779000DCEEF0A3EFF0D39464EE9475
:10679C000050507B057AA7799C9000DCE0FCA3E0CC
:1067AC00FD129EBF7F087D767B027A0179C81205A7
:1067BC00A87B057AA779A29000DCE0FEA3E0FFC3DA
:1067CC0074649FFDE49EFC129EBF7F017B027A01E4
:1067DC0079C87564781206AB7D767B027A0179C82C
:1067EC001205A8129356026DF27F107D6E7B741207
:1067FC00000C7F107D3C7B7012002E7F427D6E1250
:10680C00002E7F747D6E12002EE49000CEF090006E
:10681C00CEE0FFC39403503E7B057AA779A8EF75B1
:10682C00F032A4FFAEF09065FFE0FCA3E0FD12EBAC
:10683C0035AC06AD07129EBF9000CEE075F030A4CB
:10684C00240DFF7D727B027A0179C81204C5900079
:10685C00CEE004F080B8E49000CEF09000CFE0FFE2
:10686C009000CEE0FEC39F4003026DF2EE25E0FFE8
:10687C00E433FE748C2FF582EE342DF583E0FEA309
:10688C00E0FFE4FCFD12EE257F307E007D007C00F5
:10689C0012EC29EC12E63B12EE259000F712EDBC3F
:1068AC0012E53B12E677C3746E9FFF9000D2F0FDA9
:1068BC00A3E0FF04F07B6D12002E9000CEE004F0FC
:1068CC0080997F0312023F901DFBE0601A902F20ED
:1068DC00E0FF60137B057AA779ACFD7C00129EBFAC
:1068EC007FD87D7212059E129356901A43E0647DF8
:1068FC006008E0647C6003026AF1901DFBE0FF70AD
:10690C0009906C47E07003026A2BEF60437F007EB6
:10691C00007D007C0012EE259069CE12EDBC12E5D4
:10692C00EA7007FFFC12EE258015902D7A12EDBC53
:10693C0012EE2590662212EDBC12E3B412EE2590F5
:10694C0069CE12EDBC12E3B89000FF12EDD8807046
:10695C0090666FE0FCA3E0FDE412E63F12EE257FAB
:10696C00427EC87D007C0012E53B12EE257F427E04
:10697C00707D007C0012E53B12EE259069C4E02589
:10698C00E0FF9069C3E033FE74E52FF582EE341717
:10699C00F583E0FCA3E0FDE412E63F12E4C39000B3
:1069AC00EB12EDD89017DC12EDBCE412E63B12EEC4
:1069BC00259000EB12EDBC12E3B89000FF12EDD85D
:1069CC00906C4C12EDBC12EE259000FF12EDBC1237
:0769DC00E5EA400E906C4C4F
:1069E30012EDBC9000FF12EDD880207F007E007D69
:1069F300007C0012EE259000FF12EDBC12E5EA5078
:106A03000A9000FF12EDE400000000907BE312ED1A
:106A1300BC12EE259000FF12EDBC12E4C312E67720
:106A23009000D3EFF0026AA89065F1E0FCA3E0FDCB
:106A3300E412E63F12EE25906C52E0FCA3E0FDE485
:106A430012E63F12E53B9000FF12EDD8906C52E046
:106A5300FEA3E0FFD39065F2E09F9065F1E09E40D6
:106A63000FEEF0A3EFF0906C66E09000D3F0801D82
:106A7300906C66E0FCE412E64312EE259000FF12F0
:106A8300EDBC12E4C312E6779000D3EFF09000FF61
:106A930012EDBC12EE25906C4C12EDBC12E4C390C7
:106AA30000FF12EDD890662212EDBC9000FB12EDB0
:106AB300D8906C4C12EDBC12EE259000FB12EDBC8D
:106AC30012E5EA400C906C4C12EDBC9000FB12ED09
:106AD300D8907BE312EDBC12EE259000FB12EDBCC7
:106AE30012E4C312E6779000D2EFF0026BED901A36
:106AF30043E0647B6008E0647A6003026BED9066B8
:106B03002212EDBC12EE25906C4C12EDBC12E5EA9C
:106B1300504A902F2BE0FF7E007C007D3C12EB352A
:106B2300A3E02FFDEC3EFCE412E63F12EE25906657
:106B33002212EDBC12EE257F447E7A7D007C00128A
:106B4300E53B12E4C312E677906C52EEF0A3EFF04C
:106B530090662212EDBC906C4C12EDD89066221216
:106B6300EDBC9000FB12EDD890662212EDBC12EE44
:106B730025906C4C12EDBC12E53B12EE25906C6631
:106B8300E0FCE412E64312E4C312E6779000D2EF8E
:106B9300F09065F1E0FCA3E0FDE412E63F12EE2580
:106BA300906C52E0FCA3E0FDE412E63F12E53B905B
:106BB30000FF12EDD8906C66E0FCE412E64312EE9F
:106BC300259000FF12EDBC12E4C312E6779000D3C8
:106BD300EFF09000FF12EDBC12EE25906C4C12ED1D
:106BE300BC12E4C39000FF12EDD8902D84E0600541
:106BF300E4F00268F61293567F3F7E007D007C002E
:106C030012EE259000FF12EDBC12E3B812E677C036
:106C130006C0077F3F7E007D007C0012EE259000BA
:016C2300FB75
:106C240012EDBC12E3B812E677AC06AD07D007D07C
:106C340006C3ED9F9000D9F0EC9E9000D8F0902D03
:106C440084E06004E4F080AF7F477E7F7DDC7C00DD
:106C540012EE259000FB12EDBC12E5EA503A75667F
:106C6400057567A77568B17F3F7E007D007C0012C3
:106C7400EE259000FB12EDBC12E3B812E6778E69A4
:106C84008F6A9000D8E0FEA3E08E6BF56C7B027AED
:106C94000179C812EF5B802B7566057567A7756867
:106CA400BD9000FB12EDBC8F6C8E6B8D6A8C69906D
:106CB40000D8E0FEA3E08E6DF56E7B027A0179C800
:106CC40012EF5B9000D2E0FED3946E40047F02800A
:106CD40004EE2412FF7D677B027A0179C81204C591
:106CE4009000D2E0FF7D66240EFB75666E120945A6
:106CF4007F477E7F7DDC7C0012EE259000FF12ED45
:106D0400BC12E5EA50117B057AA779CB9000FF12FB
:106D1400EDBC129EF7800F7B057AA779D09000FF17
:106D240012EDBC129EA19000D3E0FED3946E4004F9
:106D34007F028004EE2412FF7D767B027A0179C8FB
:106D44001204C59000D3E02406FF7D747B057AA766
:106D540079D71204C59000D3E0FF7D75240EFB752E
:106D6400667D120945901DFBE06003026DF27F0110
:106D7400129F3F7FD67D677B027A0179C81204C5D2
:106D8400906C47E060399069C4E025E0FF9069C3E6
:106D9400E033FE74EC2FF582EE3469F583E0FAA358
:106DA400E0FB7C007D3CFFAE0212EB49902F2BEF01
:106DB400F07C007D3CAF03AE0212EB49A3EDF0750D
:106DC40066057567A77568D9902F2BE0756900F57E
:106DD4006AA3E0756B00F56C7B027A0179C812EF47
:106DE4005B7FD67D757B027A0179C81204C5E555AF
:066DF400600312033F22C0
:106DFA008F4DE54DC394285007E4906CE2F080145F
:106E0A00E54DC39428400DE54DC3943C5006906C63
:106E1A00E27401F0129D4E90681FE551F0E54D12A3
:106E2A00EE776E75006EBA016F03026F48036F87C3
:106E3A00046F480573650670B60A73890B740D0CE6
:106E4A0074260D71271071271174C014758F157669
:106E5A00232876232976F42A77C32B77E72C771809
:106E6A002D73413C74A53D000078907F017B057A23
:106E7A00A779E3129AE87F027B057AA779EB129A3F
:106E8A00E87F037B057AA779F8129AE87F047B05E5
:106E9A007AA87900129AE8906C4BE06408600302C1
:106EAA0078907F057B057AA8790B129AE802789088
:106EBA007F017B057AA87913129AE87F027B057A0B
:106ECA00A87928129AE87F037B057AA87931129A61
:106EDA00E87F04906C4BE0B408087B057AA87946F1
:106EEA0080067B057AA87957129AE87F057B057A8E
:106EFA00A8795E129AE80278907F017B057AA879D0
:106F0A0072129AE87F027B057AA8797A129AE87F48
:106F1A00037B057AA87982129AE87F047B057AA80E
:106F2A00798A129AE87F057B057AA87993129AE8FA
:106F3A007F067B057AA8799E129AE80278907F07E5
:106F4A001282E17F01129AE87F0D1282E17F02121A
:106F5A009AE87F131282E17F03129AE87F1912825C
:106F6A00E17F04129AE87F1F1282E17F05129AE8F4
:106F7A007F251282E17F06129AE80278907F0C7DC3
:106F8A00187B057AA879A91204C57F147D237BE3AF
:106F9A0012000CE4900117F0900117E0C394064028
:106FAA0003027890129356900117E0FE75F00EA432
:106FBA002427A3F0E4FF901A6AE02EFD12800290C3
:106FCA002F21E014606714600302709475660575DA
:106FDA0067A87568C3900117E004756900F56A909F
:106FEA002F26E0756B00F56CA3E0756D00F56EA3B6
:106FFA00E0756F00F570A3E0757100F572A3E07596
:10700A007300F574A3E0757500F576A3E075770053
:0B701A00F5787B027A0179C812EF5B69
:107025007F0C900118E0FD7B027A0179C81204C536
:1070350080767566057567A87568F3900117E00495
:10704500756900F56A902F2212EDBC12E6778F6EF6
:107055008E6D8D6C8C6B902F29E0756F00F570A38C
:10706500E0757100F572A3E0757300F574A3E07522
:107075007500F5767B027A0179C812EF5B7F0C907B
:107085000118E0FD7B027A0179C81204C5801990C8
:107095000117E060030278957F02FDFB1296BB9015
:1070A5006694E0901A43F022900117E004F0026F15
:1070B500A27F077D647BE77566781209457F0F7DA2
:1070C500697B057AA979191205A87B057AA9792022
:1070D500901A6AE024F975F00684E5F004FD7C0059
:1070E500129EBF7F6C7D6912059E7F017B057AA983
:1070F5007925129AE87F027B057AA67906129AE825
:10710500901A6AE024F975F00684E5F0D3940050EE
:10711500030278907F037B057AA9792B129AE802FE
:107125007890E54D641060030271AC7F0C7D197B8E
:10713500057AA9793B1205A87401D39551500FE53D
:1071450051D3940350087B057AA9794D80067B05B8
:107155007AA979638B668A678968906C5AE0756944
:1071650000F56AA3E0756B00F56CA3E0756D00F59D
:107175006E7B027A0179C812EF5B7F8A7D19120551
:107185009EE551D394035016E55175F01AA4FE24DB
:107195006BFF7D14EE2481FB75662812094590016D
:1071A500197404F00272337F0C7D197B057AA97975
:1071B500791205A8E551D3940650087B057AA9797B
:1071C5008A80067B057AA9799C8B668A678968908F
:1071D5006C54E0756900F56AA3E0756B00F56CA366
:1071E500E0756D00F56EA3E0756F00F570A3E075B1
:1071F5007100F572A3E0757300F5747B027A01796D
:10720500C812EF5B7F8A7D1912059EE551D394065E
:107215005016E55175F00BA4FE247BFF7D14EE247A
:1072250088FB7566281209459001197407F07F0CD3
:107235007D377B057AA979A91205A8900119E0FF88
:10724500D395515011EF04FFE551D39F50087B05AD
:107255007AA979BE80067B057AA979CD8B668A677E
:087265008968906C5DE0756919
:10726D0000F56AA3E0756B00F56C7B027A0179C8B5
:10727D0012EF5B7F8A7D3712059E900119E0FFD3D7
:10728D0095515021EF04FEE551D39E5018C3E551A1
:10729D009F75F01AA4FE2485FF7D32EE249BFB75AD
:1072AD0066461209457F0C7D557B057AA979DE125C
:1072BD0005A8900119E0FF2402D395515012EF2437
:1072CD0004FFE551D39F50087B057AA979EF80061D
:1072DD007B057AAA79048B668A678968906C5FE072
:1072ED00756900F56AA3E0756B00F56C7B027A0198
:1072FD0079C812EF5B7F8A7D5512059E900119E0CA
:10730D00FF2402FED395514003027890EF2403FF32
:10731D00E551D39F4003027890C3E5519E75F01A55
:10732D00A4FE2485FF7D50EE249BFB756664120937
:10733D00450278907F017B057AAA791A129AE87F27
:10734D00027B057AAA7924129AE87F037B057AAA33
:10735D00792A129AE80278907F017B057AA779F84D
:10736D00129AE87F027B057AA67943129AE87F0389
:10737D007B057AAA793B129AE80278907F017B050A
:10738D007AAA7946129AE87F027B057AAA79551274
:10739D009AE87F037B057AAA7969129AE89069B910
:1073AD00E025E024A5F582E434CBF58374019370D8
:1073BD000193700D7B057AAA7979FDFC129EBF8031
:1073CD001F7B057AAA79809069B9E025E024A5F59F
:1073DD0082E434CBF583E493FC740193FD129EBFDC
:1073ED007F017B027A0179C87564EF1206ABEF2439
:1073FD00F6FF7D3B7B027A0179C81205A8027890D1
:10740D007F017B057AAA7989129AE87F027B057A3A
:10741D00AA7996129AE8027890E4900117F09001FB
:10742D0017E0FFC394065065EF25E02457F582E47D
:10743D00347CF583E0FEA3E0FF4E60517566057563
:10744D0067AA75689C900117E08E698F6A248BF589
:10745D0082E4347CF583E070087B057AAA79A580F7
:10746D00067B057AAA79AF8B6B8A6C896D7B027A64
:10747D0001790312EF5B900117E004FF7B027A01A3
:10748D007903129AE8900117E004F08091900117AA
:10749D00E0902F30F00278907B057AAA79B690654E
:1074AD00FFE0FCA3E0FD129EBF7F0C7D1912059E2F
:1074BD000278907B057AAA79CB7F407E197D997CE5
:0F74CD009A129EA17F0C7D131204BB7B057AAA35
:1074DC0079E79013AF12EDBC129ED97F0C7D1E1272
:1074EC0004BB901A44E0D3940040117B057AAA792E
:1074FC00FB90669512EDBC129ED9800C7B057AAB85
:10750C00790EE4FDFC129EBF7F0C7D291204BB1288
:10751C009B2F8B698A6A896B7566057567AB756875
:10752C002A7B027A0179C812EF5B7F0C7D3412043E
:10753C00BB7F0C7D407BE612000C7B057AAB793A65
:10754C009003A1E0FD7C00129EBF7F0C7D441204D1
:10755C00BB129BD2AC06AD077B057AAB794B129E66
:10756C00BF7F0C7D4F1204BB7B057AAB79629065B3
:10757C00FFE0FCA3E0FD129EBF7F0C7D5A1204BB02
:10758C000278907B057AAB797990660B12EDBC1280
:10759C009EA17F0C7D131204BB7B057AAB798E9078
:1075AC00660712EDBC129EA190CB66E493FF7D1E84
:1075BC001204BB7B057AAB799B90660312EDBC126F
:1075CC009EA190CB66E493FF7D291204BB7B057AC8
:1075DC00AB79A89002D1E0FD7C00129EBF7F0C7DA0
:1075EC00341204BB7F0C7D407BE612000C9065F4DA
:1075FC0012EDBC12EE257F107E0E7D007C0012F683
:10760C007212EE447B057AAB79BF129ED97F0C7D4A
:10761C00441204BB027890E54D6428706B7F027BAA
:10762C00057AAB79CE129AE8E4901DF7F0906C4590
:10763C00E07009FFFEFDFC12EE258031906C7AE0C3
:10764C002400FD906C79E034C0FCE412E63F12EEAD
:10765C00257F477E407D007C0012E53B12EE257FA6
:10766C00427EC87D007C0012E4C312EE257F427E70
:10767C00C87D007C0012E3B47B057AAB79DB129EEB
:10768C00A17F117D651204BB7F017B057AAB79FD6F
:10769C00129AE8E4901DF7F0906999E07003027873
:1076AC00907F077D437BE77566771209457F117DD7
:1076BC00497B057AAC790C1204C57F117D547BDDB6
:1076CC0012000C7566057567AC75681375690275E3
:1076DC006A69756B997B027A0179C812EF5B7F112D
:1076EC007D581204BB0278907F017B057AAC790C33
:1076FC00129AE87F027B057AAC792A129AE87F030A
:10770C007B057AAC7931129AE8027890756605752A
:05771C0067AC75683D3B
:10772100756902756A69756B997B027A0179C8126C
:10773100EF5B7F0C7D211204BB906C45E07009FF6B
:10774100FEFDFC12EE258031906C7AE02400FD9064
:107751006C79E034C0FCE412E63F12EE257F477EEF
:10776100407D007C0012E53B12EE257F427EC87D04
:10777100007C0012E4C312EE257F427EC87D007CAE
:107781000012E3B47B057AAC7955129EA17F0C7D82
:107791002E1204BB7480FF7E017B027A6C794575E1
:1077A1006000756101120A817B057AAC7978906C71
:1077B10045E0FD7C00129EBF7F0C7D3B1204BB02A5
:1077C10078907F017B057AAC7992129AE87F027BEF
:1077D100057AAC79A9129AE87F037B057AAC79C165
:1077E100129AE80278907F0C7D197B057AAC79CFEB
:1077F1001205A8901A69E0C3940A5071E490011728
:10780100F0900117E02499F582E43469F583E0FFF3
:1078110060047E0180027E00EE6038756605756742
:10782100AC7568DD8F697B027A0179C812EF5B7FE5
:10783100027B027A0179C8900117E075F00CA4244B
:1078410070F5641206AB7D1912059E900117E004D4
:10785100F080AE901A69E075F00CA4FE2468FF7DFB
:1078610014EE2477FB75662812094580227566059A
:107871007567AC7568E0756902756A69756B997BA6
:10788100027A0179C812EF5B7F6C7D1912059EE4C3
:05789100901DF7F0223C
:107896008B4D8A4E894F8D507B057AAC79E3129DCC
:1078A6004E7F02AB4DAA4EA94F7564771206AB7D8B
:1078B6002DAB4DAA4EA94F1205A87F187D557B63A7
:1078C60075666E1209457F2D7D5D7B057AAC79EB79
:1078D6001205A8E55060197F8B7D557BD675666EBF
:1078E6001209457F9C7D5D7B057AAC79EF1205A870
:0478F60012033F2218
:1078FA00906CE2E060727480FF7E017B027A6C79A0
:10790A0045756000756101120A81902F2FE075F0AC
:10791A0040A42400FFE5F03414FE7B027A6C7977E8
:10792A00756000756140120A81906C77E0FAA3E0F5
:10793A00FB2428FFE43AFEC3906C7AE09FFF906C28
:10794A0079E09EFE7C007D0A12EB499066AEEEF06D
:10795A00A3EFF0AF03AE027B027A1D798E75600049
:10796A00756128120A818057902F2FE0FF7E007CD4
:10797A00007D6312EB3574022FF9741E3EFA7B0206
:10798A00C00378777C6CAD03D0037E007F6312EA74
:10799A00A5906C94E0FEA3E0FFC3906C9BE09F90DF
:1079AA0066AFF0906C9AE09E9066AEF0788E7C1D81
:1079BA007D027B027A6C79B27E007F2812EAA5905A
:1079CA006C7C12EDBC12EE257F407E7E7D057C002C
:1079DA0012EC8B12EE44906C46EFF0906C7C12ED38
:1079EA00BC12EE257F407E7E7D057C0012EC8B1258
:1079FA00EE4C12EE257F707E177D007C0012EC8B18
:107A0A0012EE44906C44EFF0906C7C12EDBC12EED6
:107A1A00257F707E177D007C0012EC8B12EE4C12D3
:107A2A00EE257F647E007D007C0012EC8B12EE4412
:107A3A00906C48EFF0906C7C12EDBC12EE257F64DE
:107A4A007E007D007C0012EC8B12EE4C906C6AEF8B
:107A5A00F09065FFE0FEA3E08E58F5599065FF743B
:107A6A000BF0A374B8F0E4FFFE7DFF1219B4906521
:097A7A00FFE558F0A3E559F022E4
:107A83008F57E55720E10620E203027BB1E557302B
:107A9300E1087B057AAC79F580067B057AAD790D33
:107AA300129D4EC2AF1278FA7566057567AD75689B
:107AB30028902F2FE004756900F56A906CE2E0606E
:107AC30009906C45E0FF7E0080079003A1E0FF7EF4
:107AD300008E6B8F6C7B027A0179C812EF5B7F0C8F
:107AE3007D1912059E7566057567AD75683A906CCC
:107AF30083E0756900F56AA3E0756B00F56CA3E09C
:107B0300756D00F56E7B027A0179C812EF5B7F0C0D
:107B13007D3712059E7566057567AD756853906C64
:107B230082E0756900F56A906C81E0756B00F56C15
:107B3300906C80E0756D00F56E7B027A0179C81256
:107B4300EF5B7F0C7D4612059E7566057567AD7507
:107B5300686B906C46E0756900F56A906C44E0755B
:107B63006B00F56C906C48E0756D00F56E906C6A77
:107B7300E0756F00F5707B027A0179C812EF5B7FC5
:107B83000C7D5512059E906C9CE07006906C7BE01A
:107B9300601A7F0C7D667B057AAD79881204C57FF8
:107BA3000C7D707B057AAD79AF1204C5D2AFE55772
:107BB30030E5237B057AAD79E2129D4E7F357D2D2D
:107BC3007B057AAD79EB1205A87F177D3C7B057A9F
:107BD300AE79061205A8E55720E303027E399068C3
:107BE30020E060087B057AAD79E280067B057AA305
:107BF3007913129D4E906820E07019906C9CE07090
:107C030006906C7BE0600D7F327D017B057AAE7957
:107C1300201204C5C2AF906CDDE0FCA3E0FDE412CA
:107C2300E63F12EE257F427E707D007C0012E4C3A6
:107C330012EE2590668812EDBC12E3B812EE257F92
:107C4300427EC87D007C0012E4C312EE257F3F7E96
:107C5300007D007C0012E3B812E67790012212ED5A
:107C6300D890012212EDBC12EE257F407E7E7D0569
:107C73007C0012EC8B12EE4490011CEFF090012279
:107C830012EDBC12EE257F407E7E7D057C0012EC5A
:107C93008B12EE4C12EE257F707E177D007C001256
:057CA300EC8B12EE4421
:107CA80090011DEFF090012212EDBC12EE257F70BD
:107CB8007E177D007C0012EC8B12EE4C12EE257FB5
:107CC800647E007D007C0012EC8B12EE4490011E55
:107CD800EFF090012212EDBC12EE257F647E007D4C
:107CE800007C0012EC8B12EE4C90011FEFF07566D1
:107CF800057567AE75683B906CDDE0FAA3E0FB7C28
:107D0800007D3CFFAE0212EB498E698F6A7C007DD4
:107D18003CAF03AE0212EB498C6B8D6C90011CE0FA
:107D2800756D00F56EA3E0756F00F570A3E07571D1
:107D380000F572A3E0757300F5747B027A0179C8C7
:107D480012EF5B7F0C7D147B027A0179C81204C59F
:107D58007F0C7D1E7B8012000C7B057AA679C39070
:107D680065FFE0FCA3E0FD129EBF7F017B027A0164
:107D780079C87567821205507D1F1204BB7B057A8E
:107D8800AE79619069D412EDBC129EF77F0C7D2EFE
:107D98001204BB9069D812EDBC12EE257F447E7A9E
:107DA8007D007C0012E53B7B057AAE7974129EA1BA
:107DB8007F0C7D3B1204BB7B057AAE79879069DC2A
:107DC80012EDBC129EA17F0C7D481204BB7F007E81
:107DD800007D007C0012EE259069E012EDBC12E5F2
:107DE800EA500A9069E012EDE4000000007B057A91
:107DF800AE79A19069E012EDBC129EA17F0C7D5571
:107E08001204BB7B057AAE79B49069E412EDBC121A
:107E18009EF77F0C7D621204BB7B057AAE79C89011
:107E280069E812EDBC129EF77F0C7D6F1204BBD27D
:107E3800AFE55720E403028001C2AF1278FA7B0550
:107E48007AAE79DA902F2FE02401FDE433FC129EFC
:107E5800BF7F8A7D141204BB7F8A7D1E7BE51200DA
:107E68000C7F857D0F7BEA75667A12094575660574
:107E78007567AE7568EB906C46E0756900F56A90B9
:107E88006C44E0756B00F56C906C48E0756D00F51E
:107E98006E906C6AE0756F00F5707B027A0179C8A4
:107EA80012EF5B7F8A7D211204BB906CDBE06003DC
:107EB800027FAF7B057AAF790C9069D412EDBC12C2
:107EC8009EF77F8A7D2E1204BB7B057AAF792390BB
:0F7ED8001DA612EDBC129EF77F8A7D3B1204BBE4
:107EE7007F427EC87D007C0012EE25901DAE12ED0C
:107EF700BC12E4C312EE25901DB212EDBCE412E6EB
:107F07003B12E53B12EE257F3F7E007D007C001291
:107F1700E3B812E677900120EEF0A3EFF07566055F
:107F27007567AF75683A8E69F56AC374649FF56CB7
:107F3700E49EF56B7B027A0179C812EF5B7F8A7D3D
:107F4700481204BB7B057AAF79539069E412EDBC04
:107F5700129EF77F8A7D551204BB7B057AAF796B3A
:107F6700901DAA12EDBC129EF77F8A7D621204BB98
:107F77007F007E007D007C0012EE259069E012ED07
:107F8700BC12E5EA500A9069E012EDE40000000037
:107F97007B057AAF79859069E012EDBC129EA17FCF
:107FA7008A7D6F1204BB80509069D812EDBC12EE27
:107FB700257F447E7A7D007C0012E53B7B057AAF06
:107FC700799C129EA17F8A7D2E1204BB7B057AAF16
:107FD70079B39069DC12EDBC129EA17F8A7D3B12BA
:107FE70004BB7B057AAF79CE9069E812EDBC129E8F
:0B7FF700F77F8A7D481204BBD2AF2246
:108002008F538D54906C4BE064087058E554D394B0
:10801200064051E55424F9FD75F0068475F080A4FC
:108022002400FBE5F03404FAED75F00684E5F07502
:10803200F010A4AEF02BF556EE3AF555E553701359
:10804200AF56AE557B027A2F7921F56075610C121D
:108052000A8122AF56AE557B027A2F7921755C0CCC
:10806200120BA322E5537025AF54FEFC7D0C12EBDC
:108072003574D82FF974153EFA7B02C00378217C3F
:108082002FAD03D0037E007F0C12EAA522AF547EEF
:10809200007C007D0C12EB3574D82FF974153EA8C4
:1080A20001FC7D027B027A2F79217E007F0C12EA8D
:0280B200A52205
:1080B400ED7003028198902F21EFF0906C55E0FF52
:1080C400E4FCFDFE12EE257F107E277D007C00126D
:1080D400EC2912EE25906C54E0FFE4FCFDFE12EE58
:1080E400257FA07E867D017C0012EC2912EC021211
:1080F400EE25906C56E0FFE4FCFDFE12EE257FE8D1
:108104007E037D007C0012EC2912EC0212EE259015
:108114006C57E0FFE4FCFDFE12EE257F647E007DDB
:10812400007C0012EC2912EC0212EE25906C58E04F
:10813400FFE4FCFDFE12EE257F0A7E007D007C003C
:1081440012EC2912EC0212EE25906C59E0FFE4FCCB
:10815400FDFE12EC02EC12E63B902F2212EDD878D1
:10816400267C2F7D027B027A6C795A7E007F07126F
:10817400EAA57F01901A6AE0FD128002901A6AE073
:1081840024F975F00684E5F0B405037F0B22901AF8
:108194006AE004F0E4FF901A6AE0FD128002902F76
:1081A4002212EDBC12EE257F477EC37D507C001267
:1081B400E53B12E677906C54EFF0902F2212EDBC61
:1081C40012E67712EE257FA07E867D017C0012ECFC
:1081D4008B12EE4C8F4D8E4C8D4B8C4A12EE257FBC
:1081E400107E277D007C0012EC8B12EE44906C55BF
:1081F400EFF0AF4DAE4CAD4BAC4A12EE257F107E86
:10820400277D007C0012EC8B12EE4C8F4D8E4C8D32
:108214004B8C4A12EE257FE87E037D007C0012EC35
:108224008B12EE44906C56EFF0AF4DAE4CAD4BACB0
:108234004A12EE257FE87E037D007C0012EC8B124F
:10824400EE4C8F4D8E4C8D4B8C4A12EE257F647E06
:10825400007D007C0012EC8B12EE44906C57EFF022
:10826400AF4DAE4CAD4BAC4A12EE257F647E007D23
:10827400007C0012EC8B12EE4C8F4D8E4C8D4B8C8F
:108284004A12EE257F0A7E007D007C0012EC8B12E0
:10829400EE44906C58EFF0AF4DAE4CAD4BAC4A127F
:1082A400EE257F0A7E007D007C0012EC8B12EE4CE2
:1082B4008F4D8E4C8D4B8C4A906C59EFF0785A7CD4
:1082C4006C7D027B027A2F79267E007F0712EAA555
:0D82D400902F21E0B401037F20227F1F22A4
:1082E1008F527E007F407D007B027A01792712EE5A
:1082F1009DE4900126F0900126E0FEC39406400320
:108301000283B1E4FFE5522EFD128002902F21E09D
:1083110070030283B17B027A01792712F6D4C3EF8D
:108321009420EE6480948040030283A878677C01E6
:108331007D027B027A0179277E007F2012EAA590D7
:108341002F21E0640270347566057567AF7568E4C6
:10835100756902756A01756B67902F26E0756C006F
:10836100F56DA3E0756E00F56FA3E0757000F57112
:108371007B027A01792712EF5B802C7566057567A0
:10838100AF7568F8756902756A01756B67902F2280
:1083910012EDBC12E6778F6F8E6E8D6D8C6C7B0249
:1083A1007A01792712EF5B900126E004F00282F74F
:1083B100900126E070147566057567B07568027BDB
:1083C100027A01796712EF5B80247566057567B0E3
:1083D100756808900126E0756900F56A756B02758C
:1083E1006C01756D277B027A01796712EF5B7B0265
:1083F1007A01796712F6D4D3EF941EEE64809480EB
:10840100401378857C017D027B057AB0790F7E006F
:0C8411007F0412EAA57B027A0179672241
:10841D008F4AE4901DFBF09066ACF0906C47F090A5
:10842D00039EF0ED24FE6010047028901DFB740176
:10843D00F0E4906C71F0801B906C477401F0E49047
:10844D006C71F09069C3F0A3F09017DC12EDE400AD
:10845D00000000E54A6406602CAF4A9065F3EFF02A
:10846D009013A3EFF0906C4BE0B408137430FF7EC3
:10847D00017B047A00794A755C01120BA38006908A
:0D848D006C69E54AF0AF4AE4FD12849A22C2
:10849A008F4B8D4C906C6112EDE400000000E54BAF
:1084AA00F4704A123AA67E007F047D007B027A6944
:1084BA00799512EE9D7E007F047D007B027A6679B3
:1084CA009C12EE9D902D807401F09065ECF0E49082
:1084DA006820F0906C71E06008E064016003028A31
:1084EA00ED906C717402F0E49069AEF022E4FFAD95
:1084FA004B12800290039EE0703C906C47E0600350
:10850A0002858D901DFBE0600302858D9065F3E086
:10851A00600AE0FFC3E54B9F6406601A9065F3E0CA
:10852A00C39406500BE0FFE54BB5070AE54C70060D
:10853A00902F21E0704D123AA6E4906820F0907BCB
:10854A00E8F090667CF09003A004F07F0C9065F34D
:10855A00E0C3940650047D01800B9065F3E0FEC3EE
:10856A00E54B9EFEFDE4FB1296BBE4906C47F0904F
:10857A00039EF09002D2E07006901A437402F01241
:10858A00351F22E54BC394065011906C71E0C394D9
:10859A000250087402F0E49069AEF0906821E0702D
:1085AA0009901A44E07003028AE0E54C70030286DF
:1085BA0091E490667CF09065F1F0A3F0906995F0F3
:1085CA0090669CF0902F29E0FF906996F090669D46
:1085DA00F0902F2AE0FE906997F090669EF0E4A34F
:1085EA00F0902D80F090682004F0E490681DF090DF
:1085FA007BE804F0EF7007EE70047F0180027F00D1
:10860A009001A9EFF0E4FFE54B04FD1280029065AA
:10861A00F3E0600DE54B04FFE0FEC3EF9E640660E5
:10862A0006902F21E070257E007F047D007B027A70
:10863A0066799C12EE9D90667C7401F09002D2E0FD
:10864A006003028AED901A437402F0229001A9E0B5
:10865A00600790667C7401F0227F08E4FDFB1296A5
:10866A00BB9002D2E0700B901A437483F07F201201
:10867A007A8390667C7401F012351F7F04E4FD7BD7
:10868A0001128EDA028AE8902F21E0FF6402600864
:10869A00EF64016003028AE8E4906C71F09069AEBD
:1086AA0004F06F60030289AB901DFBE0600F9069D4
:1086BA00B312EDBC906C4C12EDD8028960906C47F5
:1086CA00E070030288E8906C4BE0B4082C906C7858
:1086DA00E02428FF906C77E03400FEC3906C7AE0C7
:1086EA009FFF906C79E09EFE7C007D0A12EB499018
:1086FA006C49EEF0A3EFF0801B906C94E0FEA3E0CF
:10870A00FFC3906C9BE09F906C4AF0906C9AE09E3D
:10871A00906C49F07E027F587D007B027A1779E5DA
:10872A0012EE9D7E027F587D007B027A6979EC12F7
:10873A00EE9DE49001A7F0A3F0906C49E0FCA3E061
:10874A00FD9001A7E0FEA3E0FFC39DEE9C4003025B
:10875A0088D0906C4BE0B4082B7C007D0A12EB3574
:10876A00906C78E02428FD906C77E03400CD2FFFE0
:10877A00ED3EFE7B027A66797E75600075610A12AB
:10878A000A8180369001A7E0FEA3E0FF906C95E095
:10879A002FFF906C94E03EFE7C007D0A12EB35744C
:0F87AA00332FF9742F3EFA7B02C003787E7C6672
:1087B900AD03D0037E007F0A12EAA5906C4AE0243B
:1087C900FFFF906C49E034FFFE9001A7E0FCA3E0B5
:1087D900FD6F7002EE6C70507F457EBB7D80FC1290
:1087E900EE2590667EE0FCA3E0FDE412E63F12E58B
:1087F9003B12EE25906682E0FCA3E0FDE412E63F21
:1088090012E4C312E677AC06AD079001A8E025E0B3
:10881900FF9001A7E033FE74E52FF582EE3417F5DA
:1088290083ECF0A3EDF0803D906682E0FCA3E0FDCF
:10883900E412E63F12EE257F417E207D007C001286
:10884900E53B12E677AC06AD079001A8E025E0FF0D
:108859009001A7E033FE74E52FF582EE3417F58316
:10886900ECF0A3EDF07F477E6A7D607C0012EE2577
:108879009001A8E025E0FF9001A7E033FE74E52F01
:10888900F582EE3417F583E0FCA3E0FDE412E63F40
:1088990012E53B12E677AC06AD079001A8E025E0AA
:1088A900FF9001A7E033FE74EC2FF582EE3469F5F1
:1088B90083ECF0A3EDF09001A8E004F070069001BC
:1088C900A7E004F00287439069E012EDBC906C4C7C
:1088D90012EDD8E4906C71F09069AE04F080789054
:1088E9002F2212EDBC906C4C12EDD8902F2BE0FF8B
:1088F9007E007C007D3C12EB35A3E02FFDEC3EFCB5
:10890900E412E63F12EE25906C4C12EDBC12EE25F6
:108919007F447E7A7D007C0012E53B12E4C312E6B7
:1089290077906C52EEF0A3EFF0FDAC06E412E63F4F
:1089390012EE257F007E007D007C0012E5EA700DB5
:10894900906C717402F0E49069AEF0800AE4906C66
:1089590071F09069AE04F0906C4C12EDBC12E677A0
:10896900906C6112EDD8E49065F1F0A3F0FE7F04FC
:10897900FD7B027A69799512EE9D7E007F047D0068
:108989007B027A66799C12EE9D902D807401F0909D
:1089990065ECF09066AB7403F0901A43747CF002B6
:1089A9008A92902F27E0FF7E007C007D3C12EB35F8
:1089B900AA06AB07902F26E0FF7E007C0E7D1012E1
:1089C900EB35EF2BFFEE3AFE902F28E07C002FFFCE
:1089D900EC3EFE906C50F0A3EFF0FDAC06E412E61D
:1089E9003F12EE25902F2BE0FF7E007C007D3C128C
:1089F900EB35A3E02FFDEC3EFCE412E63F12E53B2C
:108A090012EE257F447E7A7D007C0012E4C3906CCF
:108A19004C12EDD8906C50E0FCA3E0FDE412E63F67
:108A290012E677906C52EEF0A3EFF0E49065F1F066
:108A3900A3F0902F26E0906995F090669CF0902F16
:108A490027E0906996F090669DF0902F28E0906954
:108A590097F090669EF0E4A3F0902D80F09065EC7D
:108A690004F0901A43747AF0902F2BE07011A3E070
:108A7900700D906C717402F0E49069AEF0800AE4B4
:108A8900906C71F09069AE04F0123AA6901DFBE06B
:108A990070257F099065F3E0FEC3E54B9EFDE54B2C
:108AA900C3940650047B00800B9065F3E0FEC3E598
:108AB9004B9EFEFB1296BBE4906820F07F011245A5
:108AC90082907BE87401F0E490681DF07F057D01D8
:108AD9007B01128EDA80087F04E4FDFB1296BBE469
:058AE9009066ACF022D4
:108AEE008F528D5378167C667D027B027A1D798EAD
:108AFE007E007F6612EAA5901A43E0647D6005E071
:108B0E00647C704B90662212EDBC12EE25906C4C7C
:108B1E0012EDBC12E5EA500C906C6112EDE400000F
:108B2E000000804890662212EDBC12EE25906C4C2F
:108B3E0012EDBC12E3B412EE257F3F7E007D007C69
:108B4E000012E3B812E677906C6112EDD8801D7FAB
:108B5E003F7E007D007C0012EE2590662212EDBC59
:108B6E0012E3B812E677906C6112EDD8902D84E086
:108B7E006004E4F080817B057AA5798590664212C7
:108B8E00EDBC129EF77FA1E4FD1207059066ABE0E7
:108B9E0090CB8A9324FE6049147003028C421470A9
:108BAE0003028C4224FC4003028D2F240860030232
:108BBE008D3F7B057AA5798190664A12EDBC129E97
:108BCE00F77F337D201207827B057AA57981906627
:108BDE001612EDBC129EF77F1E7D4B120705028DFD
:108BEE003F7B057AA5798190664612EDBC129EF701
:108BFE007F337D2012078290661A12EDBC12EE258D
:108C0E007F447E7A7D007C0012E53B9001AC12ED34
:108C1E00D8902D84E06004E4F080DC7B057AB07996
:108C2E00139001AC12EDBC129EF77F0D7D4B120717
:108C3E0005028D3F9066ABE090CB8A936403704D36
:108C4E0090664E12EDBC12E677AC06AD077B057A48
:108C5E00A5798E129EBF7F447D201207827F417EB2
:108C6E00207D007C0012EE2590664E12EDBC12E4C3
:108C7E00C312E6777C007D0A12EB497B057AA57953
:108C8E0089129EBF7F797D20120782800CE4FF122D
:108C9E009F3F7F397D201207827FA07E867D017CDB
:108CAE000012EE25906C6112EDBC12ED32404D902B
:108CBE006C6112EDBC12EE257FA07E867D017C00DC
:108CCE0012EC8B12EE44AD07AC067B057AB0791729
:108CDE00129EBF7F057D4B12059E906C6112EDBCFE
:108CEE0012EE257FA07E867D017C0012EC8B12EEAB
:108CFE004C7B057AB0791A129ED9801C7F057D4B6C
:108D0E007B057AA5797D1205A87B057AB07920902E
:108D1E006C6112EDBC129ED97F0D7D4B1207058042
:108D2E00109066ABE090CB8A93FFAD52AB53125BC3
:108D3E00709066ABE090CB8A93D394044003028E7E
:108D4E00D9906C71E0D3940040097F7F7D657B7F65
:0A8D5E0012002E906C71E090CB9390
:108D68009324FE6023147003028E0F147003028E86
:108D78003C147003028E3C24046003028ED97F09E0
:108D8800E4FD7B01125B70227B057AA579819066F0
:108D98002E12EDBC129EF77F1E7D69120705906C9E
:108DA80047E060399069C4E025E0FF9069C3E0338B
:108DB800FE74EC2FF582EE3469F583E0FAA3E0FB4C
:108DC8007C007D3CFFAE0212EB49902F2BEFF07C2C
:108DD800007D3CAF03AE0212EB49A3EDF0756605CA
:108DE8007567A77568D9902F2BE0756900F56AA398
:108DF800E0756B00F56C7B027A0179C812EF5B7F36
:108E0800887D69120705227B057AA5798190662EEF
:108E180012EDBC129EF77F1E7D691207057B057A4D
:108E2800A5798590663212EDBC129EF77FA17D6907
:108E3800120705227F417E207D007C0012EE2590DE
:108E4800661E12EDBC12E4C312E6777C007D0A129E
:108E5800EB497B057AA57989129EBF7F467D691209
:108E6800070590661E12EDBC12E677AC06AD077BCF
:108E7800057AA5798E129EBF7F257D691207059018
:108E88006C71E090CB9393B404117B057AA5798536
:108E980090662612EDBC129EF7802F7F007E007D23
:108EA800007C0012EE2590662A12EDBC12E5EA60FD
:108EB8000A40087B057AA5798580067B057AA5791D
:108EC8007D90662A12EDBC129EF77FA17D6912077C
:028ED800052271
:108EDA008F4F8D508B51E49001B0F0901A43E064AB
:108EEA00796018E064786013E0647B600EE0647D6A
:108EFA006009E0647C6004E0B47A03D38001C39221
:108F0A0009901A43E064816009E064826004E0B475
:108F1A008303D38001C3920A200906200A03029020
:108F2A005EE54F30E25A7566057567B0756825903B
:108F3A006995E0756900F56AA3E0756B00F56CA3A5
:108F4A00E0756D00F56E7B027A0179C812EF5B90CD
:108F5A006820E060187F28E4FD7B027A0179C81254
:108F6A0005A87F017D0C7B6412000C800D7F0DE447
:108F7A00FD7B027A0179C812070F9001B07401F0E3
:108F8A00300948E54F30E143906820E0703D901D7C
:108F9A00FAE0FFD3940040087B057AA5798580061C
:108FAA007B057AA5797DEFFD7C00129EBF7FA1909B
:108FBA0066ABE090CB8A93D3940450047D4B800235
:108FCA007D691207059001B07401F0300912E54F6E
:108FDA0030E00DE4FFAD50128AEE9001B07401F05A
:108FEA009001B0E06007E551600312033F30096465
:108FFA00E54F6404705E906820E0705890681DE048
:10900A006052E4FFAD50128AEE901DFAE0FFD3944D
:10901A000040087B057AA5798580067B057AA579C3
:10902A007DEFFD7C00129EBF7FA19066ABE090CBE6
:10903A008A93D3940450047D4B80027D69120705FC
:10904A00D3906CE0E09402906CDFE094004005E479
:05905A0090681DF022EA
:10905F008F4A8D4BE4FF12CF29EF7002FF227F0161
:10906F007D0512D2349013A7EFF0640C60037F00DC
:10907F0022129356E54A1470030291DF0460030233
:10908F00930C7F017D2312D234EF7F00FEC006C008
:10909F00070F7D2412D234EFFDD0E02D9013AEF0E8
:1090AF00D0E034009013ADF0E49001B1F09001B135
:1090BF00E0C39404400302918C1293569001B1E0E7
:1090CF00FBC374039B75F008A4A3F090669512ED93
:1090DF00BC12EE257F01EB240AFD12D234E4FCFD15
:1090EF00FE9001B2E0FBF812ED6B12EC0290669568
:1090FF0012EDD890660312EDBC12EE257F019001A0
:10910F00B1E02414FD12D234E4FCFDFE9001B2E074
:10911F00FBF812ED6B12EC0290660312EDD890661D
:10912F000712EDBC12EE257F019001B1E02418FD6E
:10913F0012D234E4FCFDFE9001B2E0FBF812ED6BAD
:10914F0012EC0290660712EDD890660B12EDBC126E
:10915F00EE257F019001B1E0241CFD12D234E4FC16
:10916F00FDFE9001B2E0FBF812ED6B12EC0290667F
:10917F000B12EDD89001B1E004F00290BC7F017D9D
:10918F002D12D2349002D1EFF0E0FCE412E643123C
:10919F00EE257F407EC97D0F7CDB12E4C312EE25E6
:1091AF007F447E7A7D007C0012E53B906C6D12ED62
:1091BF00D8906C6D12EDBC12EE2590CB8512EDC8D8
:1091CF00EC12E63B12E53B9069A412EDD802930C2A
:1091DF00E54B640270309013ADE0FEA3E0FF7C011D
:1091EF007D0012EB9EAB077D237F0112D19F901361
:1091FF00ADE0FEA3E0FF7C017D0012EB9EAB057D91
:10920F00247F0112D19FE54B6401600302930C9000
:10921F0001B1F09001B1E0C39404400302930C122A
:10922F0093569001B1E0FEC374039E75F008A4FF3E
:10923F00A3F0FBEE240AFDC00590669512EDBCA8C5
:10924F000312ED5712EE257FFF7E007D007C00128A
:10925F00ECD5AB077F01D00512D19F9001B1E0246F
:10926F0014FDC00590660312EDBC9001B2E0FBF84F
:10927F0012ED5712EE257FFF7E007D007C0012EC71
:10928F00D5AB077F01D00512D19F9001B1E0241813
:10929F00FDC00590660712EDBC9001B2E0FBF8121D
:1092AF00ED5712EE257FFF7E007D007C0012ECD57E
:1092BF00AB077F01D00512D19F9001B1E0241CFDB7
:1092CF00C00590660B12EDBC9001B2E0FBF812EDF9
:1092DF005712EE257FFF7E007D007C0012ECD5AB90
:1092EF00077F01D00512D19F7F017D2D9002D1E024
:1092FF00FB12D19F9001B1E004F00292227F012274
:10930F00E49001B4F0FF12CF299001B3EFF0C2AF98
:10931F007F017D0512D2349001B4EFF01293569075
:10932F0001B4E0FF901A44E06F6014E4FFFD129067
:10933F005FE4FFFD1254869001B4E0901A44F0D21E
:07934F00AF9001B3E0FF2223
:0793560075A61E75A6E122B9
:10935D00E49001B5F0A3F0C39001B6E09F9001B584
:10936D00E09E5026E49001B7F09001B7E0C3941948
:10937D005008129356E004F080EF9001B6E004F02F
:0B938D0070069001B5E004F080CD22D6
:1093980053F3F8EF42F343F348E5F330E4FB53F3B8
:1093A800EFAFF5EF75F004A4FFE5F454037C002F4C
:0D93B800FFEC35F0FE9069ACF0A3EFF02261
:1093C500901A43E0647B6006906820E06018906620
:1093D5009CE07012A3E0700EA3E0700A90667CF02A
:1093E5009066AC04F02290669FE004F0C39464504C
:1093F50003029469E4F09065EC04F09065F2E004F2
:10940500F070069065F1E004F0902D80E064017045
:109415002990669EE004F0C3943C4048E4F09066D1
:109425009DE004F0C3943C403BE4F090669CE0046E
:10943500F0C3940A402EE4F0802A90669EE014F072
:10944500F47021743BF090669DE014F0F47015748F
:109455003BF090669CE014F0F47009F0A3F0A3F0E3
:1094650090667CF0C3901DE8E09470901DE7E09451
:1094750017406D902D8BE06067E4901DE7F0A3F039
:109485009065EB04F0906C47E06055906C4AE024E1
:10949500FFFF906C49E034FFFE9069C3E0FAA3E05A
:1094A500FBD39FEA9E50399017DC12EDBC12EE25D6
:1094B500EB25E0FFEA33FE74E52FF582EE3417F570
:1094C50083E0FEA3E0FFE4FCFD12EC029017DC1242
:1094D500EDD89069C4E004F070069069C3E004F02B
:0194E5002264
:1094E6009069C6E0FED3940340079066157401F0B8
:1094F60022EE1392C3EED394014003D38001C392AC
:10950600C45329E09069C7E04229908001E529F01B
:109516009069C8E044C0FCA3E0F5828C83EFF0902C
:1095260069C9E004F070069069C8E004F0D3906958
:10953600C9E094FF9069C8E0943F4018E4F0A3F0B6
:109546009069C7E004F0E0D3941F4008E4F0906906
:05955600C6E004F02254
:10955B00EF24E5603F047078120006E4FF12E1E2AD
:10956B007F1E7E0012935DE4FF12E1E27F1E7E0000
:10957B0012935D9002D47489F09002D6741AF0782D
:10958B00D77C027D027B027A6679A17F0612EAA55F
:10959B0012006F2290020DE09066A4F090020EE094
:1095AB009066A5F090020FE09066A6F0900210E096
:1095BB009066A3F0900211E09066A2F0900212E088
:1095CB009066A1F07F0112E1E27F1E7E0012935D97
:0195DB00226D
:1095DC007F1C7D18E4FB1296057FC87E0012935DFC
:1095EC007F1A12955B7FC87E0012935D7F01129CDF
:0995FC00A07FC87E0012935D22DD
:109605001200069002D47485F09002D6EFF0A3ED17
:08961500F0A3EBF012006F223C
:10961D00908002E09001B8F020E20E906C72E06054
:10962D000E9066B07401F08006906C727401F0902B
:10963D008002E0440FF454F0907BEBF07009901A27
:10964D0042E070030296BA907BEBE0F9B4F014900F
:10965D0066A9E0700E901A6B74F0F09066A9740113
:10966D00F0803A9066A9E07034901A42E0FF69707C
:10967D0024E954F060179069B2E0FE9065E5E0D3FF
:10968D009E400A901A6BE9F0E49065E5F09065E56F
:10969D00E004F08008E97005901A6BEFF0E97008AE
:0E96AD009066A9F09065E5F0901A42E9F0226F
:1096BB008F528D538B5475552775561075570575ED
:1096CB0058A17559F4755A05755BA1755CF4755DF8
:1096DB0005755EA1755FF47B057AAC79E3129D4E3F
:1096EB00E55214B41C004003029A929096FDF828A0
:1096FB00287302975102975D029772029787029720
:10970B009C0297A80297B40297C00297D502988D36
:10971B0002988D0298C00298FE02991902993A029A
:10972B00994F029A920299640299870299AF029912
:10973B00BB0299CD02992E0299F1029A3D029A65CC
:10974B00029A70029A897557057558B0755934028B
:10975B009A927557057558B075594F755D05755EBD
:10976B00B0755F58029A927557057558B075594F79
:10977B00755D05755EB0755F6B029A9275570575D1
:10978B0058B075594F755D05755EB0755F83029A5C
:10979B00927557057558B0755998029A9275570579
:1097AB007558B07559A8029A927557057558B075CA
:1097BB0059B7029A927557057558B07559CE755DA4
:1097CB0005755EB0755FD6029A92906C47E0FF60AC
:1097DB00087B057AB079E680067B057AB179018B37
:1097EB00578A5889597B057AB17912EF60067C004C
:1097FB007D018009E55404FF7E00AC06FD129EBF7F
:10980B007F0F7D537B027A0179C81205A87F077DF4
:10981B004B7BE7756678120945902F21E064027047
:07982B002B7566057567B19E
:1098320075681F90669CE0756900F56AA3E0756B18
:1098420000F56CA3E0756D00F56E7B027A0179C8B4
:1098520012EF5B80207F3F7E007D007C0012EE25B0
:10986200906C4C12EDBC12E3B812E6777B057AB12C
:109872007937129ED97F0F7D667B027A0179C812F1
:1098820005A875554E755620029A9275570575585A
:10989200B17559017566057567B1756849756900D5
:1098A20085536A756B0085546C7B027A0179C81204
:1098B200EF5B755D02755E01755FC8029A92906CEE
:1098C20047E0600C755A05755BB1755C5F029A9250
:1098D2007557057558B175597B7B057AB17993E552
:1098E20053FD7C00129EBF755A02755B01755CC800
:1098F200755D05755EB1755F9E029A927557057525
:1099020058B17559A7755A05755BB1755CBC75552B
:109912004E755620029A927557057558B17559C7FA
:10992200755A05755BB1755CBC029A9275570575DF
:1099320058B17559D9029A927557057558B175592A
:10994200E3755A05755BB2755C00029A927557050C
:109952007558AD7559EB755A05755BB2755C190290
:109962009A927557057558B27559307B057AB27956
:1099720052E553FD7C00129EBF755A02755B01755C
:019982005C88
:10998300C8029A927557057558B27559677B057A5F
:10999300B2797BE553FD7C00129EBF755A02755B5D
:1099A30001755CC8E4F555F556029A92755705752D
:1099B30058B2755989029A927557057558B27559F7
:1099C300A775551F755640029A927557057558B27B
:1099D3007559C2755A05755BB2755CDF755D0575A2
:1099E3005EB2755FF67555037556E8029A92E553B4
:1099F300B4FF0B7557057558B37559108035E5538A
:109A0300601E7557057558B37559287B057AB0796B
:109A130017FD7C00129EBF7F6B7D46120782801369
:109A23007B057AB37947E4FDFC129EBF7F517D32FB
:109A3300120782E4F555F55680557557057558B3E9
:109A430075594A7B057AB3795CE553FD7C00129E18
:109A5300BF755D02755E01755FC875553A75569899
:109A6300802D7557057558B3755971802275570543
:109A73007558B3755986755A05755BB3755CA2E461
:109A8300F555F55680097557057558B37559B87F5F
:109A930002AB57AA58A9597564771206AB7D2DAB53
:109AA30057AA58A9591205A87F02AB5AAA5BA95C09
:109AB3007564771206AB7D3CAB5AAA5BA95C1205B1
:109AC300A87F02AB5DAA5EA95F7564771206AB7DC2
:109AD3004BAB5DAA5EA95F1205A812033FAF56AE5A
:059AE3005512935D2205
:109AE8008F528B538A54895590681FE0B552047F72
:109AF8000180027F00901DF7EFF07566057567B36A
:109B08007568D285536985546A85556B7B027A01DD
:109B180079C812EF5B7F0CE55275F011A42408FD9B
:079B280012059E1293562264
:109B2F00E49001B9F0A3F0A3F09001BBE0C3943C23
:109B3F005019E4FF1293989001BAE02FF09001B9F9
:109B4F00E03EF09001BBE004F080DE9001B9E0FE52
:109B5F00A3E0FF7C007D3C12EB499001B9EEF0A32E
:109B6F00EFF0E4A3F09001BBE0FFC3940B502FEF95
:109B7F0025E0246FF582E434CBF583E493FC740184
:109B8F0093FDD39001BAE09D9001B9E09C500790EE
:109B9F0001BCEFF080089001BBE004F080C790019A
:109BAF00BCE0FFD3940250077B057AB379D922EF3B
:109BBF00C3940840077B057AB379E0227B057AB31B
:039BCF0079E62212
:109BD2009003A1E0D394005003029C92906615E09A
:109BE20060057E007F00229003A1E075F063A4244B
:109BF200BFF582E5F0341DF583E0FFE4FCFDFE12C3
:109C0200EE257F007E407D007C0012EC2912EE25BD
:109C12009003A1E075F063A424BEF582E5F0341D43
:109C2200F583E0FFE4FCFDFE12EE257F007E007D61
:109C3200087C0012EC2912EC0212EE259003A1E03E
:109C420075F063A424C0F582E5F0341DF583E0FECF
:109C5200A3E0FFE4FCFD12EC029001BF12EDD890EC
:109C620001BF12EDBC12EE257FEB7E517D007C0020
:109C720012EC8B12EE44C374649FFF7E009001BD10
:109C8200EEF0A3EFF0D39464EE940040087F6422D8
:0E9C92007E007F64229001BDE0FEA3E0FF2271
:109CA000EF602C146003029D4D1200069002D474E4
:109CB00088F09002D67420F09013AF12EDBC8F4F55
:109CC0008E4E8D4D8C4C7F04129FFD12006F227FB3
:109CD000057B027A66791112A0BE7F817EB17D4F2D
:109CE0007C0112EE2590661112EDBC12ED07405A70
:109CF0007FC07EF37D5E7C0112EE2590661112ED31
:109D0000BC12ED076002504290661112EDBC901338
:109D1000AF12EDD8E4FFFE906611E0FD12E0B07FD7
:109D2000017E00906612E0FD12E0B07F027E00909E
:109D30006613E0FD12E0B07F037E00906614E0FD44
:0E9D400012E0B0C2AF12E0C2D2AF12351F2245
:109D4E008B608A6189629069C5E07059FF12023F8B
:109D5E00E4901DF7F0FFFDAB60AA61A9621205A8A1
:109D6E00906991E064017031906C4BE06408702949
:109D7E00906999E0647B6021901A43E064616019F8
:109D8E007F017B027A6979997567EF1205507D0222
:109D9E007B027A6979991204C5E4FF7D0C7BEE751E
:0B9DAE00667E120945E49069C5F022B2
:109DB900300C2290020BE075F00AA4FE90020AE032
:109DC90075F064A42EFE90020CE02E9001C3F0B54C
:089DD90007037F01227F002235
:109DE100E4FFFE12E09E906611EFF07F017E00120B
:109DF100E09E906612EFF07F027E0012E09E906678
:109E010013EFF07F037E0012E09E906614EFF09056
:109E1100661112EDBC9013AF12EDD87F047E0012D3
:109E2100E09E906611EFF07F057E0012E09E906645
:109E310012EFF0906611E0FFA3E09065FFCFF0A371
:109E4100EFF09065FFE07002A3E0600FD390660031
:109E5100E0943C9065FFE0940040089065FFE4F0D9
:109E6100A304F07F087E0012E09E906611EFF07F60
:109E7100097E0012E09E906612EFF07F0A7E0012CA
:109E8100E09E906613EFF07F0B7E0012E09E9066DD
:109E910014EFF090661112EDBC9065F412EDD8222A
:109EA1008B588A59895A8B668A6789688F6C8E6B41
:0E9EB1008D6A8C697B027A0179C812EF5B2200
:109EBF008B608A6189628B668A6789688C698D6A13
:0A9ECF007B027A0179C812EF5B22D2
:109ED9008B608A6189628B668A6789688F6C8E6BF1
:0E9EE9008D6A8C697B027A0179C812EF5B22C8
:109EF7008B588A59895A8F5E8E5D8D5C8C5B85582D
:109F070066855967855A687F3F7E007D007C001211
:109F1700EE25AF5EAE5DAD5CAC5B12E3B812E677E3
:109F27008E698F6A7B027A0179C812EF5B902D8464
:089F3700E06004E4F080C722A1
:109F3F008F577F007E007D007C0012EE2590664ECD
:109F4F0012EDBC12E5EA70089001C4F0A3F0801F77
:109F5F007F457E617D007C0012EE2590664E12EDEE
:109F6F00BC12E53B12E6779001C4EEF0A3EFF09040
:109F7F002D84E06004E4F080B9E55760087B057A32
:109F8F00B379EC80067B057AA779D98B668A6789C6
:109F9F00689001C4E0FAA3E0FB7C007D3CFFAE02B9
:109FAF0012EB498E698F6A7C007D3CAF03AE0212C3
:109FBF00EB498C6B8D6C7B027A0179C812EF5B22B7
:109FCF00AB07EDAE047807CEC313CE13D8F9547F89
:109FDF00FF74D32BF582E43402F583EFF0ED547F59
:0E9FEF00FF74D42BF582E43402F583EFF022E8
:109FFD00AB07AF4FAE4EAD4DAC4C781C12ED5712BA
:10A00D00EE257F0F7E007D007C0012ECD574D32BE6
:10A01D00F582E43402F583EFF0AF4FAE4EAD4DACAB
:10A02D004C781512ED5712EE257F7F7E007D007C5A
:10A03D000012ECD574D42BF582E43402F583EFF0E5
:10A04D00AF4FAE4EAD4DAC4C780E12ED5712EE2516
:10A05D007F7F7E007D007C0012ECD574D52BF582C0
:10A06D00E43402F583EFF0AF4FAE4EAD4DAC4C780E
:10A07D000712ED5712EE257F7F7E007D007C0012CA
:10A08D00ECD574D62BF582E43402F583EFF07F7FA7
:10A09D007E007D007C0012EE25AF4FAE4EAD4DAC77
:10A0AD004C12ECD574D72BF582E43402F583EFF026
:01A0BD002280
:10A0BE008F4A74092FF582E43402F583E0FFE4FC45
:10A0CE00FDFE781512ED6B12EE257408254AF58209
:10A0DE00E43402F583E0FFE4FCFDFE781C12ED6B28
:10A0EE0012EC0212EE25740A254AF582E43402F5CA
:10A0FE0083E0FFE4FCFDFE780E12ED6B12EC021213
:10A10E00EE25740B254AF582E43402F583E0FFE474
:10A11E00FCFDFE780712ED6B12EC0212EE25740CAC
:10A12E00254AF582E43402F583E0FFE4FCFDFE12DD
:06A13E00EC0212EDA0226C
:10A144007F1BE4FDFB1296BBC2AF7E007F287D001F
:10A154007B027A7C795712EE9D907CB37478F090F0
:10A164007CB27401F0907CB47439F0907C7F741FDD
:10A17400F0A37486F0E4FFFD12D42D9001C6EFF035
:10A18400FD907CB37404F0907CB27402F0907CB4C3
:10A194007441F0907C7F7419F0A3749AF07F0112DB
:10A1A400D42DD2AF907C57E07002A3E0700A7F1CDC
:0BA1B400FDFB1296BB7F00227F012202
:10D27200005EBCE2613FDD83C29C7E20A3FD1F41B4
:10D282009DC3217FFCA2401E5F01E3BD3E6082DCA4
:10D29200237D9FC1421CFEA0E1BF5D0380DE3C6294
:10D2A200BEE0025CDF81633D7C22C09E1D43A1FF84
:10D2B2004618FAA427799BC584DA3866E5BB590774
:10D2C200DB856739BAE406581947A5FB7826C49A64
:10D2D200653BD987045AB8E6A7F91B45C6987A2454
:10D2E200F8A6441A99C7257B3A6486D85B05E7B944
:10D2F2008CD2306EEDB3510F4E10F2AC2F7193CD34
:10D30200114FADF3702ECC92D38D6F31B2EC0E5023
:10D31200AFF1134DCE90722C6D33D18F0C52B0EE13
:10D32200326C8ED0530DEFB1F0AE4C1291CF2D7303
:10D33200CA947628ABF517490856B4EA6937D58BF3
:10D342005709EBB536688AD495CB2977F4AA4816E3
:10D35200E9B7550B88D6346A2B7597C94A14F6A8D3
:10D36200742AC896154BA9F7B6E80A54D7896B35C3
:0ACE2600E4907C09F0907C32F022C9
:10CE3000E4907BEDF0A3F0C3907BEEE09FEE648086
:10CE4000F8907BEDE0648098500EA3E004F070064B
:09CE5000907BEDE004F080DF228C
:10CE5900C2B57F507E0012CE30D2B57F0612CE30D9
:10CE6900A2B5E433907BEFF07F4612CE30907BEF92
:03CE7900E0FF22B5
:10CE7C00C2B5D2B5E4907BF0F0907BF0E0C39403A4
:0DCE8C005005E004F080F2A2B5E433FF226F
:10CE9900C2B5EFB40102D2B57F0D7E0012CE30D2F9
:02CEA900B522B0
:10CEAB00E4907BF2F0907BF1F0907BF1E0C394087F
:10CEBB00502F12CE7CEF601A907BF2E0FF907BF14B
:10CECB00E0FE7401A806088002C333D8FC4F907BA8
:10CEDB00F2F07F107E0012CE30907BF1E004F080F8
:07CEEB00C8907BF2E0FF227A
:10CEF200AD07E4907BF3F0907BF3E0FFC39408501E
:10CF02001EEDA807088003A2E713D8FB907BF4F07C
:10CF12005401FFF012CE99907BF3E004F080D87FA9
:07CF22000D7E0012CE30224B
:10CF29008F4C907BF67404F0E4907C33F0FE7F28FC
:10CF3900FD7B027A7C790A12EE9DC2AF12CE59EFBF
:10CF49007068907C09F0907C32F012CFB8EF605590
:10CF5900907C33E004F0E4907BF5F0907BF5E0C33E
:10CF690094085032E0FF2434F582E4347CF583E000
:10CF7900FE907C33E075F008A4240AF582E4347C41
:10CF8900F583E5822FF582E43583F583EEF0907B16
:10CF9900F5E004F080C512CFB8EF6009907C33E06A
:0FCFA900C3940A40ABD2AF7F0122D2AF7F0022E8
:10CFB800907BF77401F0E4A3F0A304F0E4A3F0A3DA
:10CFC800F0129356E4907BFDF0907C08F012CE5955
:10CFD8007E00907BFEEEF0A3EFF07006907C32E0CE
:10CFE8006007E4907C09F0FF227FF012CEF21293E2
:10CFF80056E4907BFAF012CE7CEFB40106907BFAEF
:10D008007402F07F107E0012CE3012CE7CEFB40195
:10D0180007907BFAE04401F0907BFAE0FF6403702C
:10D028000302D110EFD394004009EFC313907BFCA7
:10D03800F0804E907C09E0FF907BF7E0FEC39F50A4
:10D0480026A3E02434F582E4347CF583E0FD907B6C
:10D05800F9E0FCED5CD3940040047D0180027D0082
:10D06800907BFCEDF0800FEEB507047F0180027F16
:10D0780000907BFCEFF0907BFCE07005907BFBEE72
:10D08800F0907BFCE0FFB40121907BF8E02434F5BC
:10D0980082E4347CF583C083C082E0FE907BF9E0B3
:10D0A800FDEE4DD082D083F08020907BF8E02434D0
:10D0B800F582E4347CF583C083C082E0FE907BF97E
:10D0C800E0F4FDEE5DD082D083F012CE99907BF72C
:10D0D800E004F0907BF9E0FF25E0F0701C907BF80D
:10D0E800E02434F582E4347CF583E0FF12D14790E4
:10D0F8007BF8E004F0A3E004F0129356907BF8E08C
:10D10800C39408500302CFF9907BF7E0C3944140E1
:10D1180006907C08E06007E4907C09F0801B907B17
:10D12800FBE0907C09F070047F0180027F00907C16
:0FD1380032EFF0907BFD7401F0907BFDE0FF2261
:0FD14700907C08E06F90D27293FF907C08F022EA
:10D15600AC0712CE59EF6005D2AF7F00227F551281
:10D16600CEF2E4907C00F0907C00E0FFC39408507F
:10D1760025EC75F008A4240AF582E4347CF583E5F1
:10D18600822FF582E43583F583E0FF12CEF2907CA0
:09D1960000E004F080D17F0122C9
:10D19F00AA07A905C2AF12D156EF7002FF227F0F67
:10D1AF0012CEF2AF0112CEF2E4FF12CEF2AF0312A3
:10D1BF00CEF2AF0212D156EF7002FF227FAA12CE2B
:10D1CF00F212CEAB907C01EFF012CEAB907C02EF5F
:10D1DF00F012CEAB907C03EFF012CEAB907C04EF4D
:10D1EF00F0AF0212D156EF7002FF227F5512CEF22E
:10D1FF00907C01E0FF12CEF2907C02E0FF12CEF2A3
:10D20F00907C03E0FF12CEF21293567FBC7E021287
:10D21F00CE3012935612CE59EF6005D2AF7F002257
:05D22F00D2AF7F0122D7
:10D23400AC07AB0512CE59EF60037F0022C2AFAF3B
:10D244000412D1567FF012CEF2AF0312CEF2E4FFF5
:10D2540012CEF212CEAB907C07EFF012CE59EF60F3
:0ED2640005D2AF7F0022D2AF907C07E0FF2200
:10E0800025642E20253575202825732900414E54FE
:0EE090002B53706F7274005375756E746F00B1
:10CE0300417C8901417C8A07417CB607487CAAB9E9
:10CE1300A521FBBD72C345487C81B9AD3228757E1F
:02CE2300C74DF9
:10D3720012D41A7F647E0012E03CE4907C3CF09070
:10D382007C3CE004F012DF5FEF64016009907C3CBA
:10D39200E0C3940A40E91293567F647E0012E03C97
:10D3A20012D41A7F647E0012E03C129356E4907C01
:10D3B2003CF0907C3CE004F012DA20EF640160095A
:10D3C200907C3CE0C3940A40E97FD07E0712E03CA7
:10D3D200E4907C3CF0907CB3E0B4780DE4FF7B02F7
:10D3E2007A7C79AA12D9538012907CB3E0B4040BF0
:10D3F200E4FF7B027A7C798112D953907C3CE00471
:10D40200F012DD76EF6009907C3CE0C3940A40C5DF
:08D412007F647E0012E03C2261
:10D41A005328BF908000E528F0000000432840E52B
:03D42A0028F022C5
:10D42D008F4A907C40EDF012D372E4907C3DF090E9
:10D43D007C3DE0FFC39408400302D56DE4FDFC1272
:10D44D00DE68E4907C3EF0907C3EE004F0E4A3F0D6
:10D45D00907C3FE004F0907C3DE0FF7D5112D8EBD5
:10D46D00EF64016009907C3FE0C3940A40E2E490D0
:10D47D007C3FF0907C3FE004F012DDEBEF64016047
:10D48D0009907C3FE0C3940A40E9907C3DE0FF1297
:10D49D00DBEC907C9FEEF0A3EFF0129356907C9F07
:10D4AD00E07002A3E07009907C3EE0C39432409797
:10D4BD00907C3EE0C39432400302D56D1293567FAB
:10D4CD00057D4B7BE9756679120945907C9FE0FEE1
:10D4DD00A3E0FF907C40E0FD25E02457F582E43485
:10D4ED007CF583EEF0A3EFF0748B2DF582E4347CA4
:10D4FD00F583E54AF07566057567E0756880ED049E
:10D50D00756900F56A907C9FE0FEA3E08E6BF56C6B
:10D51D00E54A70087B057AE0798D80067B057AE017
:10D52D0079978B6D8A6E896F7B027A0179C812EFBC
:10D53D005B907C40E0FE1313543F75F064A42414FB
:10D54D00FFEE540375F00AA42450FD1204BB120320
:10D55D003F907C40E004F0907C3DE004F002D43C30
:09D56D0012D372907C40E0FF2211
:10D576008F4F8D5012DD89EF7002FF22E55024FE99
:10D58600605A14700302D62F2402600302D67B125F
:10D59600DC11EF64A5703F907C89E0640170377FF1
:10D5A6000112DCC5EF640160037F00227F4112DCBB
:10D5B600C5EF640160037F0022AF4F12DCC5EF6444
:10D5C6000160037F0022E54F64E5FF12DCC5EF64CE
:10D5D6000160067F00227F00227F012212DC11EF0C
:10D5E60064A5703F907C89E0640170377F0112DC8E
:10D5F600C5EF640160037F00227F4B12DCC5EF6438
:10D606000160037F0022AF4F12DCC5EF64016003A7
:10D616007F0022E54F64EFFF12DCC5EF6401600670
:10D626007F00227F00227F012212DC11EF64A570A9
:10D636003F907C89E0640170377F0112DCC5EF649E
:10D646000160037F00227F4C12DCC5EF640160039A
:10D656007F0022AF4F12DCC5EF640160037F00221A
:10D66600E54F64E8FF12DCC5EF640160067F002227
:06D676007F00227F01226B
:10D67C008F4F8D508B5112DD89EF7002FF2212DC1F
:10D68C0011EF64A5705D907C89E0640170557F0397
:10D69C0012DCC5EF640160037F00227F4212DCC5FF
:10D6AC00EF640160037F0022AF4F12DCC5EF640111
:10D6BC0060037F0022AF5012DCC5EF640160037F72
:10D6CC000022AF5112DCC5EF640160037F0022E53C
:10D6DC004F64E465506551FF12DCC5EF64016006D0
:09D6EC007F00227F00227F012251
:10D6F5008F4F8C508D518B5212DD89EF7002FF22B6
:10D7050012DC11EF64A5600302D795907C89E06473
:10D7150001600302D7957F0512DCC5EF6401600344
:10D725007F00227F5112DCC5EF640160037F002278
:10D73500AF4F12DCC5EF640160037F0022AF51E5F6
:10D745005112DCC5EF640160037F0022E550FF1232
:10D75500DCC5EF640160037F0022AF5212DCC5EF28
:10D76500640160037F0022AF5312DCC5EF640160E2
:10D77500037F0022E551E54F64F16551FDE5506DEC
:10D7850065526553FF12DCC5EF640160067F002218
:06D795007F00227F01224B
:10D79B008F4F8C508D5112DD89EF7002FF2212DCFE
:10D7AB0011EF64A57064907C89E06401705C7F0369
:10D7BB0012DCC5EF640160037F00227F4312DCC5DE
:10D7CB00EF640160037F0022AF4F12DCC5EF6401F1
:10D7DB0060037F0022AF51E55112DCC5EF6401609D
:10D7EB00037F0022E550FF12DCC5EF640160037F6D
:10D7FB000022E551E54F64E56551FDE5506DFF12E3
:10D80B00DCC5EF640160067F00227F00227F0122CE
:10D81B008F4F8D5012DD89EF7002FF2212DC11EF5A
:10D82B0064A5704E907C89E0640170467F0212DC27
:10D83B00C5EF640160037F00227F4412DCC5EF64F7
:10D84B000160037F0022AF4F12DCC5EF6401600360
:10D85B007F0022AF5012DCC5EF640160037F002212
:10D86B00E54F64E36550FF12DCC5EF640160067F92
:08D87B0000227F00227F012240
:10D883008F4F8D5012DD89EF7002FF2212DC11EFF2
:10D8930064A5704E907C89E0640170467F0212DCBF
:10D8A300C5EF640160037F00227F4512DCC5EF648E
:10D8B3000160037F0022AF4F12DCC5EF64016003F8
:10D8C3007F0022AF5012DCC5EF640160037F0022AA
:10D8D300E54F64E26550FF12DCC5EF640160067F2B
:08D8E30000227F00227F0122D8
:10D8EB008F4B8D4C12DD89EF7002FF2212DC11EF92
:10D8FB0064A5704E907C89E0640170467F0212DC57
:10D90B00C5EF640160037F00227F4D12DCC5EF641D
:10D91B000160037F0022AF4B12DCC5EF6401600393
:10D92B007F0022AF4C12DCC5EF640160037F002245
:10D93B00E54B64EA654CFF12DCC5EF640160067FC2
:08D94B0000227F00227F01226F
:10D953008F4B8B4C8A4D894E12DD89EF7002FF226B
:10D9630012DC11EF64A5600302DA1A907C89E0648B
:10D9730001600302DA1A907C4274A5F07F0912DC7D
:10D98300C5EF640160037F0022907C42E06409F0EC
:10D993007F4612DCC5EF640160037F0022907C4266
:10D9A300E06446F0AF4B12DCC5EF640160037F0017
:10D9B30022907C42E0654BF0E4907C41F0907C4106
:10D9C300E0FFC394085040AB4CAA4DA94E8F82751B
:10D9D300830012EAF2FF12DCC5EF640160037F00EB
:10D9E30022907C42E0FFAB4CAA4DA94E907C41E0D3
:10D9F300F58275830012EAF2FEEF6E907C42F0909E
:10DA03007C41E004F080B6907C42E0FF12DCC5EF7D
:0DDA1300640160067F00227F00227F012257
:10DA200012DC11EF64A5703C907C89E064017034D5
:10DA30007F0112DCC5EF640160037F00227F4A1280
:10DA4000DCC5EF640160037F0022E4FF12DCC5EF58
:10DA5000640160037F00227FEE12DCC5EF64016089
:0ADA6000067F00227F00227F0122D2
:10DA6A008F548B558A56895712DC11907C43EFF0FC
:10DA7A00907C89E06401600302DBE9907C43E0FF6B
:10DA8A00245C600302DBE9907C45EFF012DC119024
:10DA9A007CA9EFF0907C89E0B40112907C45E0FF0C
:10DAAA00907CA9E0FEEF6E907C45F080037FFF2218
:10DABA0012DC11907CB6EFF0907C89E0B4011290F0
:10DACA007C45E0FF907CB6E0FEEF6E907C45F080EE
:10DADA00037FFF2212DC11907C8AEFF0907C89E0B0
:10DAEA00B40112907C45E0FF907C8AE0FEEF6E90D4
:10DAFA007C45F080037FFF22E4907C44F0907C44D4
:10DB0A00E0FFC39408501474A12FF582E4347CF525
:10DB1A0083E4F0907C44E004F080E2E4907C44F0FA
:10DB2A00907CA9E014FF907C44E0C39F503E12DC35
:10DB3A0011907C44E0FE24A1F582E4347CF583EF65
:10DB4A00F0907C89E0B40119907C45E0FF74A12E25
:10DB5A00F582E4347CF583E0FEEF6E907C45F0803C
:10DB6A00037FFF22907C44E004F080B4907C45E07F
:10DB7A00FEC00612DC11D0E06F907C45F070609018
:10DB8A007CA9E064037010907CB6E0B44006907CF7
:10DB9A00A2E0FF227FFF2274F4FF7E0112E03C9094
:10DBAA007CA7E0FF907CB5E06F6031EFF0AB55AA3F
:10DBBA0056A957AE02AF01EF4E601E907CB3E0B497
:10DBCA007809907CA8E012EB21800E907CB3E0B437
:10DBDA000407907CA1E012EB217F42227F40227F42
:02DBEA004122D6
:10DBEC00907CB6E0B45107907C8AE06F60057E00B3
:10DBFC007F0022907CA2E0FE907CA1E07C002400BF
:05DC0C00FFEC3EFE22CA
:10DC1100907C467401F0E4A3F0907C8904F012D466
:10DC21001AE4907C48F0907C48E0C39408400302D9
:10DC3100DCB61293565328FB908000E528F00000D3
:10DC41000000000000000000432804E528F0E490F3
:10DC51007C49F0A3F0907C4AE004F07006907C4986
:10DC6100E004F012935620950FC3907C4AE0941083
:10DC7100907C49E0942740DDC3907C4AE094109069
:10DC81007C49E094274009907C897402F07F00224E
:10DC9100908002E0F52A30E109907C46E0FFA3E0A4
:10DCA1002FF012D41A907C46E025E0F0907C48E0F9
:10DCB10004F002DC27432801908000E528F0907CE5
:04DCC10047E0FF2217
:10DCC5008F54907C4B7401F0907C89F012D41AE447
:10DCD500907C4CF0907C4CE0C39408400302DD70CE
:10DCE500129356907C4BE05554600B43280290806C
:10DCF50000E528F080095328FD908000E528F053C1
:10DD050028FB908000E528F00000000000000000DE
:10DD15000000432804E528F0E4907C4DF0A3F09042
:10DD25007C4EE004F07006907C4DE004F0129356B2
:10DD350020950FC3907C4EE09410907C4DE0942785
:10DD450040DDC3907C4EE09410907C4DE0942740DC
:10DD550009907C897403F07F002212D41A907C4BC1
:10DD6500E025E0F0A3E004F002DCD9907C89E0FF37
:01DD7500228B
:10DD760012DDEBEFB40109E4FFFBFAF912DA6A22CD
:03DD86007F0222F7
:10DD8900908002E0F52A20E008E4FFFBFAF912DAB4
:10DD99006A5328FE908000E528F0129356E4907C9F
:10DDA9004FF0907C4FE0D394C85018908002E0F572
:10DDB9002A30E00F00000000129356907C4FE004D7
:10DDC900F080DF907C4FE0C394C840134328019052
:10DDD9008000E528F07F027E0012E03C7F00227F70
:02DDE900012215
:10DDEB00129356432801908000E528F0E4907C5074
:10DDFB00F0A3F0C3907C51E094E8907C50E0940346
:10DE0B00501C908002E0F52A30E013129356907C60
:10DE1B0051E004F07006907C50E004F080D5C39084
:10DE2B007C51E094E8907C50E0940340037F002207
:03DE3B007F012242
:10DE3E008B458A468947129356432801908000E508
:10DE4E0028F0908002E0F52A20E00C7F01AB45AA75
:0ADE5E0046A94712DA6A227F41222A
:10DE68008F4B8C4C8D4DE4F54EAF4BE4FDFB12D639
:10DE78007C054E12DD76EF6007E54EC3941440E949
:10DE8800E54EC3941440037F0022E4F54EAF4BAD3A
:10DE98004DAC4C907CB3E0FB907CB2E0F55312D6CD
:10DEA800F5054E12DD76EF6007E54EC3941440DDAC
:10DEB800E54EC3941440037F0022E4F54EAF4B9027
:10DEC8007CB4E0FD12D883054E12DD76EF6007E5DD
:10DED8004EC3941440E7E54EC3941440037F0022D8
:10DEE800E4F54E907C80E025E0FD907C7FE033FCFB
:10DEF800AF4B12D79B054E12DD76EF6007E54EC398
:10DF0800941440DFE54EC3941440037F0022E4F5E7
:10DF18004EAF4B7DF012D81B054E12DD76EF600731
:10DF2800E54EC3941440EAE54EC3941440037F00C1
:10DF380022E4F54EAF4B7D0212D576054E12DD7602
:10DF4800EF6007E54EC3941440EAE54EC3941440CD
:07DF5800037F00227F01227C
:10DF5F00129356432804908000E528F0432801E5EA
:10DF6F0028F05328FDE528F0D2955328FBE528F03B
:10DF7F00E4907C52F0A3F0C3907C53E094FA907C31
:10DF8F0052E09400500EA3E004F07006907C52E033
:10DF9F0004F080E35328FE908000E528F0E4907CA5
:10DFAF0052F0A3F0907C53E004F07006907C52E0A6
:10DFBF0004F0129356908002E0F52A20E00FC390F0
:10DFCF007C53E09430907C52E0947540D7C3907CA2
:10DFDF0053E09430907C52E0947540037F0022E42C
:10DFEF00907C52F0A3F0907C53E004F07006907C8C
:10DFFF0052E004F0129356908002E0F52A30E00FC1
:10E00F00C3907C53E09430907C52E0947540D7C31A
:10E01F00907C53E09430907C52E0947540037F00E5
:0DE02F0022432804908000E528F07F0122A4
:10E03C008E588F59E4907C55F0A3F0C3907C56E039
:10E04C009559907C55E095585029E4907C54F0906B
:10E05C007C54E0C39419500B129356907C54E004FA
:10E06C00F080EC907C56E004F07006907C55E00457
:04E07C00F080C82246
:10E09E00E5D220E0FB75D2028F828E83E0FFE4F59D
:02E0AE00D2227C
:10E0B000E5D220E0FB75D2028F828E83EDF0E4F58D
:02E0C000D2226A
:10E0C200C2AFE5D220E0FB75D25075D2A0D2AF220A
:10E0D200E4907CB7F0907CB7E0C39F500600E00468
:04E0E200F080F222B6
:10E0E600AE07EE7003430501C2C27F0C12E0D2D226
:10E0F600B312E0D2907CB87401F0907CB8E0D3946F
:10E1060008501FED1392B47F0C12E0D2D2C212E077
:10E11600D2C2C212E0D2EDC313FD907CB8E004F087
:10E1260080D8EE64017039907CB804F0907CB8E039
:10E13600D39408501FEB1392B47F0C12E0D2D2C2D4
:10E1460012E0D2C2C212E0D2EBC313FB907CB8E05D
:10E1560004F080D87F0C12E0D2C2B312E0D2805510
:10E16600EE7052907CB904F0E4FB907CB804F09019
:10E176007CB8E0D39408502E7F0C12E0D2D2C212A3
:10E18600E0D2D2B430B406907CB9E02BFB907CB9D7
:10E19600E025E0F07F0C12E0D2C2C212E0D2907C01
:10E1A600B8E004F080C97F0C12E0D2C2B312E0D20C
:08E1B600C2B4AF03227F002276
:10E1BE00EF75F00A84C454F0FEEF75F00A84EE2574
:03E1CE00F0FF223D
:10E1D100EF5DFEC4540F75F00AA4FEEF540F2EFF3D
:01E1E100221B
:10E1E200C2AFEF700302E26B14600302E30B7F0124
:10E1F2007D8EE4FB12E0E69066A3E0FF12E1BEAB87
:10E20200077F017D8412E0E69066A2E0FF12E1BE84
:10E21200AB077F017D8212E0E69066A1E0FF12E18A
:10E22200BEAB077F017D8012E0E69066A4E0FF129C
:10E23200E1BEAB077F017D8612E0E69066A5E0FFB6
:10E2420012E1BEAB077F017D8812E0E69066A6E090
:10E25200FF12E1BEAB077F017D8C12E0E67F017DFC
:10E262008E7B8012E0E602E30BE4FF7D84FB12E08A
:10E27200E6907CBAEFF030E70EE0FF7D1012E1D1BC
:10E282009066A3EFF0800F907CBAE0FF7D3012E140
:10E29200D19066A3EFF0E4FF7D82FB12E0E6907C72
:10E2A200BAEFF07D7012E1D19066A2EFF0E4FF7D4B
:10E2B20080FB12E0E6907CBAEFF07D7012E1D19023
:10E2C20066A1EFF0E4FF7D86FB12E0E6907CBAEFF8
:10E2D200F07D3012E1D19066A4EFF0E4FF7D88FB7F
:10E2E20012E0E6907CBAEFF07D1012E1D19066A5C3
:10E2F200EFF0E4FF7D8CFB12E0E6907CBAEFF07D5C
:0CE30200FF12E1D19066A6EFF0D2AF222E
:10E30E00020C51E493A3F8E493A34003F68001F2C8
:10E31E0008DFF48029E493A3F85407240CC8C33310
:10E32E00C4540F4420C8834004F456800146F6DFDF
:10E33E00E4800B010204081020408090CBAEE47EF6
:10E34E00019360BCA3FF543F30E509541FFEE493D4
:10E35E00A360010ECF54C025E060A840B8E493A39B
:10E36E00FAE493A3F8E493A3C8C582C8CAC583CAC6
:10E37E00F0A3C8C582C8CAC583CADFE9DEE780BE7E
:01CE2500000C
:0300000002E38E8A
:0CE38E00787FE4F6D8FD75817E02E3493B
:10E39A00DA0CD902800BD906300701B3500502E71F
:10E3AA002C920702E718D9F680F9D2068002C20633
:10E3BA0012E75D300606C86002B207C89206DAD0D4
:10E3CA00D9E4B8000A12E7A4A206920702E701609C
:10E3DA00FBB53100400F12E7A4A20692F7A20792FA
:10E3EA0006A2F79207C398F40424E740DF2419AD84
:10E3FA002DAC2CAB2B7A00C394084008CDCCCBFAB9
:10E40A00E4CD80F424086010F9C3ED13FDEC13FC8D
:10E41A00EB13FBEA13FAD9F1A206300701B3403035
:10E42A008A35E52E2BF536E52F3CF537E5303DF5F7
:10E43A0038501A13F538E53713F537E53613F5363C
:10E44A00E53513F5350531E5317002053202E6B7D7
:10E45A00E4C39AF535E52E9BF536E52F9CF537E5AD
:10E46A00309DF538500DB207C378357F04E496F62F
:10E47A0008DFFA7A047019E531C39408F5315002BD
:10E48A001532E4C535C536C537F538DAE802E75836
:10E49A0020E7BAE5317002153215317835C37F04A9
:08E4AA00E633F608DFFA80E812
:10E4B200DA03B8000302E72CD9028002D9F702E797
:10E4C2001812E75D300701B392077004D9E780059F
:10E4D200DADEB8000302E758D9E2C3947E5002158F
:10E4E200322531F531500205327833760008B839D9
:10E4F200FA782B7933E608FAE8FC782E8AF0E608F7
:10E50200A427F709E5F037F7500989F00907E76012
:10E51200FBA9F0B831E61919ECF8B82ED802E6B723
:10E5220002E743B8FFFA02E72CD9FB02E718DAF652
:10E53200B800F002E75812ECE812E75D300701B3C9
:10E5420092077007D9E3B800E280DBDAE1B8000293
:10E5520080E1D9D5C8C39850021532247F500205F4
:10E5620032F531783876007A1A7B80C3E52E952B06
:10E57200E52F952CE530952D4016C3E52E952BF50C
:10E582002EE52F952CF52FE530952DF530E64BF63F
:10E59200DA0302E6B7EB03FB30E703187600C3E5C4
:10E5A2002E33F52EE52F33F52FE53033F53040CA03
:05E5B20030E7DD80B63A
:10E5B700D908A207300601B3400A12E72C7480225B
:10E5C700DAF8D9ECA2069206D082D08312EE4CC0BC
:10E5D70083C082A206E492E1B2E11422D9DCA20749
:10E5E700B380E312E75D9206DAD6D9F0A2073006C8
:10E5F70001B35005A207B380CDFEFFC3985004AF07
:10E6070031F404C3136009C3EE983007B9B380B679
:10E61700EFF539B206EED083D08212E3CCC082C0C8
:10E6270083E8600EC539C3953994145005A207B322
:04E6370080A3E422B6
:10E63B007920800C7910800479087D007E007F00A2
:10E64B003392D530D50312ECF9EC33400FEF33FF97
:10E65B00EE33FEED33FDEC33FCD9EE22EECCF5F0D0
:0CE66B00747E29A2D513FF92F7AEF022B6
:10E67700EF8EF0A2F7D2F73392D5C3947F5006E41A
:10E68700FFFEFDFC229420400474FF80F304CCFEBF
:10E69700E4FFFAE5F0CC6012C3CC13CCCD13CDCE9A
:10E6A70013CECF13CF0450EEDAEC30D5D702ECF906
:10EEFC00E57A2466F8E6057A22786330180278669B
:10EF0C00E475F00112EE1502EAD72011EB7F2ED238
:10EF1C00118018EF540F2490D43440D4FF30150BCB
:10EF2C00EF24BFB41A0050032461FFE57B60021587
:10EF3C007B057EE57E7002057D20195830180D7812
:10EF4C0063E475F00112EE15EF02EB2102F6AD74DD
:10EF5C0003D2188003E4C218F57A8B638A6489653E
:10EF6C00E4F57BF57DF57EE57B60077F2012EF37BE
:10EF7C0080F5F57CC212C211C213C214C216C2179C
:10EF8C00C21912EF05FF700D3018057F0012EF4B00
:10EF9C00AF7EAE7D22B42550C2D5C21512EF05FF4F
:10EFAC0024D0B40A00501E75F00A20D50DC57BA4E0
:10EFBC00257BF57B7002D21480E0D211C57CA42590
:10EFCC007CF57C80D524CFB41A00EF5004C2E5D276
:10EFDC001502F21CD21280C0D21180BCD21380B8A0
:10EFEC00D2D580B612EEFCFF12EF3702EF73D217B8
:10EFFC0080A6D21680A212EEFCFB12EEFCFA12EEE8
:10F00C00FCF94A4B700679077AF37B05201333E53C
:10F01C007B602FAF7CBF00011F7E008E827583004A
:10F02C0012EAF260050EEE6F70F1C2D5EBC0E0EAA9
:10F03C00C0E0E9C0E0EE12F277D0E0F9D0E0FAD00F
:10F04C00E0FB12EAD7FF60A3EBC0E0EAC0E0E9C046
:10F05C00E012EF37D0E02401F9D0E03400FAD0E030
:10F06C00FBE57C60DDD57CDA8081D213809E12F2C8
:10F07C005C60F7E57C12E7BAA97C600BE57C12F2C8
:10F08C00FAEF7003D57CF5EA30E702F404C399502B
:10F09C0077EAF4257C0430E701E404F57C800D125A
:10F0AC00F25C60C6EA057C257C12E7BAEA7879F650
:10F0BC0030E701E4257C04D57C042016011412F2FF
:10F0CC0077E4C0E012F2FA7879E6601320E70714CF
:10F0DC00F612EF1F802204F6D0E014C0E07F00127D
:10F0EC00EF1FE57C600712EF16157C800B301603C2
:10F0FC0012EF16D0E002EF73D0E00480C512F25C80
:10F10C0060A0E57C0412E7BA7879EAF6E57C042085
:10F11C001602600104240412F27774FF04C0E0129A
:10F12C00F2FA12EF1FE57C201602600312EF16D0E4
:10F13C00E0B57CE87F4512EF297879E67F2B30E744
:10F14C00047F2DF404C0E012EF37D0E075F00A8490
:10F15C00C0F012EF20D0E012EF2002EF7379108094
:10F16C000C79088008D2D5790A8006790AC2D5C2F2
:01F17C00177B
:10F17D00E4FAFDFEFF12EEFCFC7B0820121312EEEA
:10F18D00FCFD7B1030110A12EEFCFE12EEFCFF7B33
:10F19D0020EC3382D592D55013C3E43011069FFF76
:10F1AD00E49EFEE42012039DFDE49CFCE4CBF8C23A
:10F1BD0012EC700CCFCECDCCE824F8F870F380179C
:10F1CD00C3EF33FFEE33FEED33FDEC33FCEB33FBDE
:10F1DD00994002FB0FD8E9EB301205F8D0E0C44896
:10F1ED00B212C0E00AEC4D4E4F78207B0070C2EA9F
:10F1FD00C0E012F279D0F0D0E0201204C4C0E0C417
:10F20D00B212C0F012EF20D0F0D5F0EB02EF731276
:10F21D00EE77F00253F16958EFE44CEFE042F16DF7
:10F22D004FF17144F17149EFF043F17755F0AB4671
:10F23D00F10945F07A47F31950EFE82DEFEC2EEF79
:10F24D00FA2BEFFE23EFEA20F3142A0000EFF4105F
:10F25D001103757C0612EEFCFC12EEFCFD12EEFCA9
:10F26D00FE12EEFCFF787202E7E7790AA2D52014B0
:10F27D0014301609B910020404B9080104A2D520EE
:10F28D0017025001042013619213B57B005032C058
:10F29D00E07F203014177F30A21372177216500DB5
:10F2AD0012F2CEC213C217C2167F30800F30160372
:10F2BD00E9C0E012EF37301603D0E0F9D0E0B57BAE
:10F2CD00CE3016177F30B9100C12EF377F5830152E
:10F2DD00077F788003B9080312EF373013057F2DB0
:10F2ED0002EF377F2B2017F822921380D47F00B4C2
:10F2FD00070050052472F8E6FF22286E756C6C2904
:10F30D00002D4958504443D21902EFA412EEFCB41B
:10F31D0006004001E490F30E9312EF28743A12EFB9
:09F32D0028D214757B0402F16979
:10F336009E92DA331160B135FEE57F378984213933
:10F34600FFC3AE3A5B951D3C4758633DF0FD753EE5
:10F356001872313F0000803F02E95302E963D9FB8E
:10F3660050F602E95E12E938D9F412EE257C3B7DAF
:10F37600AA7EB87F3F12E4C312E93892D5247B50A7
:10F3860010A2D570DB500AE5F024045004A2D58003
:10F39600CF12E92F12EE2512E677EFF582F404FC80
:10F3A60012E64312E3B8C08290F336740912E900FC
:10F3B60012E938D0F092D525F0A2D57001C313FF1B
:05F3C600EE92E7FE22BB
:10F3CB00DA48923ECDCCCC3EABAA2A3F000000409F
:10F3DB000000803FF037983FF304B53FFC44D73F24
:10F3EB001772313E1772B13E9115053FD95BDE3E68
:10F3FB0002E963D9FB02E953D2108002C21012E971
:10F40B0038D9F040EBD360EDC5F07F3FFEF8ED7AD5
:10F41B0000C39496C8948B40230AC89469C8941A65
:10F42B00401A0AC89468C8941F40110AC8945AC855
:10F43B009425400805F07A00CEC2E7CEC0F08C418F
:10F44B008D428E438F44EA2323C0E024DBF5827583
:10F45B0083F35002058312EE25C083C08212EDC8E0
:10F46B00D082D08312E3B4EFB2E7FF12E92F12ED93
:10F47B00C812EE25AC41AD42AE43AF4412E3B81215
:10F48B00EE2512E92612E5388C418D428E438F44CE
:10F49B0090F3CB740312E8F612EE25AC41AD42AEFD
:10F4AB0043AF4412E4C3D0E0601424E7F5827583C4
:10F4BB00F35002058312EE2512EDC812E3B812E9E0
:10F4CB002FD0E0C3947FFDE49400FC12E63F12EED4
:10F4DB00257C187D727E317F3F12E4C312EE25121C
:10F4EB00E92612E3B830100E12EE257CD97D5B7E37
:07F4FB00DE7F3E12E4C32294
:10F5020083FA703AE4E9AABCF8E0813EE6E99DBFDD
:10F512000000803F1A3C2839666999BBE335A33D58
:10F52200E75D25BFDB0FC93FCCDB8D41EE3649C419
:10F532003F91C9453DF8B0C50000803F34F517C37F
:10F5420073FA2F45DDFD0AC612F5F104A2E192110C
:10F552001420E01590F502740412E8F6802912F5E1
:10F56200F130E102B21120E0EB8C4C8D4D8E4E8FCA
:10F572004F90F516740412E8F612EE25AC4CAD4D20
:10F58200AE4EAF4F12E4C3301104EF6480FFEE338E
:10F59200EF337001FF2212F5F1C0E08C4C8D4D8EDD
:10F5A2004E8F4F90F53A740312E8F612EE25AC4CEA
:10F5B200AD4DAE4EAF4F12E4C3ECC54CFCEDC54DA4
:10F5C200FDEEC54EFEEFC54FFF90F52A740312E81B
:10F5D200F6D08212EE25AC4CAD4DAE4EAF4FE58269
:10F5E20030E00712E53BB211809D12E5388098EEBB
:10F5F20033EF3324605007D0E0D0E002E963EFA29A
:10F60200E7547F9211FF12EE257C837DF97E227FE3
:10F612003E12E4C3EE33EF332481501012EE251272
:10F62200E67712E63BEFB2E7FF12E3B8EE33EF33D1
:10F63200602A2403F8C313FFEE92E7FEE82481E474
:10F64200501A12EE2512E677EF04C2E0FCC0E01277
:10F65200E643EFB2E7FF12E3B8D0E003FAEE33EF8E
:10F6620033600B148FF0A2F713FFEE92E7FEEA224B
:10E6B700E53820E7137835C37F04E633F608DFFA39
:10E6C700E531700215321531E5353378367F03E6CB
:10E6D7003400F6500E08DFF77538800531E53170E4
:10E6E700020532E53220E7547027E531604E0460B9
:10E6F7002085383085372F85362E5320F0AC2EAD48
:10E707002FA207E53113FFE53092E7FEA83102EEAD
:10E717004CE4F530F52FF52EF5327531FF5320F027
:10E7270043200580D874FFF530F52FF52E7532009C
:10E73700F531D2075320F043200980C15320F0431D
:10E747002003E4F530F52FF52EF532F531C20780B9
:06E75700AC5320F080EC41
:10E75D0079017A018530F0E531A2F73392077532F0
:10E76D0000F5316002D2F785F030A831B8FF080905
:10E77D00E530C2E76001098C2B8D2C8EF0A2F7EFEE
:10E78D003304700A0AC2F705F00AD5F0011A1460B5
:07E79D0002D2F785F02D22E6
:10E7A400C88831C530C52DC530C52FC52CC52FC56A
:06E7B4002EC52BC52E222C
:10E7BA00F91420E72524FA50037907E4F42402FB2C
:10E7CA0018DBFDE624FB5011E4F618E604F6B40A59
:0DE7DA0008E4F6D9F57401F60A22C2D52232
:10E7E700EE33EF3392D5FB602AB4FF33EEC2E77BFB
:10E7F7000560067AE8790CE4227AE8791520D504D1
:10E807007AE87910224E614E002B494E46002D4979
:10E817004E4600E47A08F608DAFC7B0074072212F9
:10E82700EE258882EBFF75F010A4FAABF08FF07439
:10E837004DA42BFBACF050010CC3EA94F0FAEB9417
:10E847003AFBEC9426FCE530C2E7FF75F056A4F4DA
:10E857002414C5F0F434C58FF0A42AE5F03BE43C5A
:10E86700F620E70B12E9A312EE6412E53B800BF4E6
:10E877000412E9A312EE6412E4C3EE33EF33C39438
:10E887008240097050EED2E794A0504912EE4CA88E
:10E8970082E6FAEEA2E7D2E7FEEF332482FBE4C377
:10E8A700CC33CCCD33CDCE33CE33DBF3F6087B0779
:10E8B7008CF0740AA4FCAFF08DF0740AA42FFDAF9E
:10E8C700F050010F8EF0740AA42FFEE435F0F6081D
:10E8D700DBDE740722A882E604F620E70812E9A324
:0FE8E70012E53B80AAF40412E9A312E4C380A057
:10E8F600C0E012EE2512E4C38002C0E012E92F1236
:10E90600EDC8A3D0E0C0E012EE2512E92612E4C35A
:10E9160012EE2512EDC8A312E3B8D0E0D5E0E62248
:10E92600AC3BAD3CAE3DAF3E228C3B8D3C8E3D8F2D
:10E936003E2279018EF0A2F7EF3304700A09C2F77E
:10E9460005F009D5F0011A146002D2F72274FF13FC
:10E95600FF7E80E47805800BE47803800474FF78FA
:0DE9660009FFFEFDFCE52054F048F52022DD
:10E973000000803F000020410000C84200007A44AC
:10E9830000401C460050C347002474498096184B2E
:10E9930020BCBE4CCA1B0E5A1CC25367AEC59D7425
:10E9A300FB600654076014232312E9C4EB54386058
:10E9B3002A12EE2512E9BE12E4C322EB54380324D3
:10E9C3001CAA83A98290E973FF93FCEFA393FDEF45
:0CE9D300A393FEEFA393FF8A83898222A6
:10E9DF00E709F608DFFA8046E709F208DFFA803E1A
:10E9EF0088828C83E709F0A3DFFA8076E309F608C3
:10E9FF00DFFA806EE309F208DFFA806688828C8383
:10EA0F00E309F0A3DFFA805A89828A83E0A3F6082C
:10EA1F00DFFA804E89828A83E0A3F208DFFA804210
:10EA2F0080AE80B480BA80C480CA80D080DA80E49F
:10EA3F0080378023805389828A83ECFAE493A3C8BA
:10EA4F00C582C8CCC583CCF0A3C8C582C8CCC5834A
:10EA5F00CCDFE9DEE7800D89828A83E493A3F60891
:10EA6F00DFF9ECFAA9F0EDFB2289828A83ECFAE058
:10EA7F00A3C8C582C8CCC583CCF0A3C8C582C8CCF7
:10EA8F00C583CCDFEADEE880DB89828A83E493A347
:10EA9F00F208DFF980CC88F0ED14B4040050C324E1
:10EAAF001E83F582EB14B4050050B724158325821D
:10EABF00F582EF4E60ACEF60010EE58290EA2F73A6
:08EACF00000402000C06001215
:10EAD700BB020689828A83E0224003BB0402E72245
:0BEAE700400789828A83E49322E32227
:10EAF200BB020CE58229F582E5833AF583E02240E8
:10EB020003BB0406E92582F8E622400DE58229F5D9
:0FEB120082E5833AF583E49322E92582F8E22233
:10EB2100BB020689828A83F0224003BB0402F722DA
:04EB31005001F3227A
:10EB3500EFF88DF0A4FFEDC5F0CEA42EFEEC88F025
:04EB4500A42EFE22DA
:10EB4900BC000BBE0029EF8DF084FFADF022E4CCB0
:10EB5900F875F008EF2FFFEE33FEEC33FCEE9DEC79
:10EB6900984005FCEE9DFE0FD5F0E9E4CEFD22EDBF
:10EB7900F8F5F0EE8420D21CFEADF075F008EF2F09
:10EB8900FFED33FD4007985006D5F0F222C398FDFA
:05EB99000FD5F0EA2297
:10EB9E00C2D5EC30E709B2D5E4C39DFDE49CFCEE92
:10EBAE0030E709B2D5E4C39FFFE49EFE12EB493075
:0AEBBE00D507C3E49FFFE49EFE228A
:10EBC800BB0210E58229F582E5833AF583E0F5F08A
:10EBD800A3E0224003BB0409E92582F886F008E691
:10EBE80022400DE5832AF583E993F5F0A3E9932202
:0AEBF800E92582F8E2F5F008E222B8
:10EC0200EF2531FFEE3530FEED352FFDEC352EFCD4
:03EC120002EE4CC3
:10EC1500C3EF9531FFEE9530FEED952FFDEC952E6A
:04EC2500FC02EE4CB3
:10EC2900EFF88531F0A4FFE531C5F0CEF9A42EFE49
:10EC3900E435F0CDFA88F0E530A42EFEED35F0FD8F
:10EC4900E433CC8531F0A42CFCE5308AF0A42CFC0B
:10EC5900E52F89F0A42CFCE52E88F0A42CFC89F082
:10EC6900E530A42DFDEC35F0FCE52F88F0A42DFD51
:10EC7900EC35F0FC8AF0E531A42DFDEC35F0FC0211
:02EC8900EE4C4F
:10EC8B00E4CCF8E4CDF9E4CEFAE4CFFB75F020C385
:10EC9B00E53133F531E53033F530E52F33F52FE53D
:10ECAB002E33F52EEF33FFEE33FEED33FDEC33FC5D
:10ECBB00EF9BEE9AED99EC98400CFCEF9BFFEE9AD4
:0AECCB00FEED99FD0531D5F0C622DB
:10F67200C2D5EC30E70FB2D5E4C39FFFE49EFEE4AF
:10F682009DFDE49CFCE52E30E705B2D512F69712FB
:10F69200EC8B30D515E4C39531F531E49530F53076
:0BF6A200E4952FF52FE4952EF52E22A5
:10ECD500EF5531FFEE5530FEED552FFDEC552EFC71
:03ECE50002EE4CF0
:10ECE800CFC531CFCEC530CECDC52FCDCCC52ECCDE
:01ECF80022F9
:0EECF900C3E49FFFE49EFEE49DFDE49CFC222C
:10ED0700C3EF9531F8EE953048F8ED952F48F8ECBC
:10ED1700952EA2E748F830D201B392D5D082D0839E
:0BED270012EE44E8A2D5C083C0822297
:10ED3200C3EF9531F8EE953048F8ED952F48F8EC91
:10ED4200952E48F892D5D082D08312EE44E8A2D50F
:05ED5200C083C0822215
:10ED5700E86010ECA2E713FCED13FDEE13FEEF13D2
:04ED6700FFD8F022BF
:10ED6B00E8600FEFC333FFEE33FEED33FDEC33FC06
:03ED7B00D8F122AA
:10ED7E00BB020789828A8302EDBC4003BB0405E90E
:10ED8E00F802EECC400789828A8302EDC8E9F802C8
:02ED9E00EED8AD
:10EDA000BB020789828A8302EDD84003BB0405E9D0
:0CEDB000F802EEE4400122E9F802EEF067
:0CEDBC00E0FCA3E0FDA3E0FEA3E0FF22CA
:10EDC800E493FCA3E493FDA3E493FEA3E493FF225E
:0CEDD800ECF0A3EDF0A3EEF0A3EFF022AE
:10EDE400A8828583F0D083D08212EDFB12EDFB1252
:10EDF400EDFB12EDFBE473E493A3C583C5F0C58377
:10EE0400C8C582C8F0A3C583C5F0C583C8C582C878
:01EE140022DB
:10EE1500FAE6FB0808E6F925F0F618E6CA3AF622FE
:10EE2500E53A053A6010D0F0D0E0C02EC02FC030D2
:10EE3500C031C0E0C0F08F318E308D2F8C2E22AFC7
:10EE450031AE30AD2FAC2EE53A146010D0F0D0E0E5
:0FEE5500D031D030D02FD02EC0E0C0F0153A22EF
:10EE6400D0F0D0E0C02EC02FC030C031053AC0E091
:03EE7400C0F022C9
:10EE7700D083D082F8E4937012740193700DA3A32A
:10EE870093F8740193F5828883E47374029368603E
:06EE9700EFA3A3A380DF3E
:10F6AD00EFB40A07740D12F6B8740A309811A899C0
:10F6BD00B8130CC2983098FDA899C298B811F630BD
:07F6CD0099FDC299F5992295
:10F6D4008B538A548955E4FFFEAB530555E555AA6F
:10F6E400547002055414F912EAD760070FEF700141
:04F6F4000E80E6227C
:10EE9D00EF4E6013EDBB021089828A83EF60010E85
:10EEAD00EDF0A3DFFCDEFA2289F04003BB0407F787
:0FEEBD0009DFFCA9F02250EFF309DFFCA9F022D6
:0CEECC00E6FC08E6FD08E6FE08E6FF2272
:0CEED800E2FC08E2FD08E2FE08E2FF2276
:0CEEE400ECF608EDF608EEF608EFF6225A
:0CEEF000ECF208EDF208EEF208EFF2225E
:00000001FF
